:100000000100000000000000000400000094511AEC
:100010001CF09FE51CF09FE51CF09FE51CF09FE5A0
:100020001CF09FE51CF09FE51CF09FE51CF09FE590
:1000300028440E02F4440500784405007C44050081
:10004000D4440500D8440500DC440500E044050024
:10005000ED440500000000EA954F01EA28008FE218
:10006000000C90E800A08AE000B08BE001704AE24A
:100070000B005AE18E4F010A0F00BAE814E04FE27C
:10008000010013E303F0471013FF2FE15C63050049
:10009000AC6305000030A0E30040A0E30050A0E303
:1000A0000060A0E3102052E27800A128FCFFFF8A44
:1000B000822EB0E13000A128003081451EFF2FE1E3
:1000C00004309FE503308FE013FF2FE1114205005C
:1000D000F8B5050001F0B7FE0027FF43002804D162
:1000E000686902F0FEFA00282DD02A89501941795A
:1000F00003790906091419430C180E3288180606EC
:10010000360E280001F092FE002807D1617D227D85
:100110000802083610433606360E03E0607B217B6A
:100120000002084301F058FE00280CD02200A11D57
:1001300028002E8102F025FC002804D0280000F0C1
:100140007AFB0020F8BD3800F8BD002070470000A1
:10015000404870B5042B046840680ED14C610B898F
:100160005B18DC799D7923022B43E52B01D1162303
:1001700000E0042354F094EA03E0012B01D14C6128
:10018000F8E7002070BD70B50C00324D1600052B4D
:1001900016D120890019C17882780802104303D152
:1001A000200000F048FB04E02000FFF791FF00284A
:1001B00001D1012070BD32002100286805230DE027
:1001C000032B06D1200001F02EFE32002100032374
:1001D00004E0022B04D1A8683200210054F060EA48
:1001E000002070BD10B51B4C206800280CD101F018
:1001F00024FE2060184A2021A06054F056EA174AD5
:100200006068202154F050EA10BD10B5114C2068F0
:10021000002808D00022132154F046EA206854F048
:1002200048EA0020206010BD70B5040000F07CF8A2
:10023000050001202073200054F03EEA280000F061
:1002400078F870BD0200034810B50068682154F0CA
:100250002CEA10BD28640500410100007701000070
:1002600010B554F0A4E954F02CEA002010BD10B5EC
:10027000FF48006800022CD5FE4CFF4A0020C11C3C
:100280006163A36B81005350031D6363A36B8918E3
:10029000801C0C284B60F2DBF848FFF7D3FF04F01A
:1002A00073FEFF21F64A2D3102E0401C8842FCDB40
:1002B00050780028F9D0F3486063F348A063C00782
:1002C0006063F248A063EF480E3860630520A063C6
:1002D00005E0EA48401CFFF7B5FF04F055FE012099
:1002E00010BDE74910B5486004F07EFD10BD70B543
:1002F00004000D00202801D304F046FEE44EA400C3
:100300003059002801D004F03FFE0020355170BD67
:10031000DF4A00218000115008007047DD48006866
:10032000002800D001207047802010B554F0CCE99F
:1003300010BD10B554F0C8E910BD02688368C168EB
:100340001000184770B5052804D2D34D84002B59EE
:10035000002B01D0012070BD2C23CF4E4343DC3E47
:100360009B192B5135000401F03528516019C260EA
:10037000816000214160C94919615861002070BD48
:10038000FEB50E001700052815D2C349020114312D
:1003900055186968C04B840000290DD101220197CE
:1003A0000096029218594369026954F092E90028B4
:1003B00001D101206860FEBD18591D0054F08CE980
:1003C00028593A00310054F08CE9285954F08CE94E
:1003D000FEBD10B5040054F08CE9206010BDA849A2
:1003E00070B50878401C0006000E08700121490411
:1003F0004018FFF727FFAA4D6C6AE00705D054F0BC
:100400007CE904F083FEA8176862A64E9ABCD26706
:1004100001000000FC030000000400005AEF5E131E
:10042000A0070CD5A86A02218843A8622020F060AA
:10043000491F6962B1680143B16004F069FE600759
:1004400005D5A86A04218843A86204F0F2FE2007BB
:100450000AD5A86A08218843A8628020F060C943B1
:100460006962B1680143B160012070BD924870B506
:1004700004688C4EA10706D500210161B26D0120F0
:100480009047022084432006000F03D0E0208443DD
:100490001020044300250AE0E00706D0A8003258E7
:1004A000002A02D021002800904764086D1C002C0F
:1004B000F2D1002070BD70B5FF257F4C6D1CE5604A
:1004C0007E480068002801D0002102E07C4800211D
:1004D000006854F020E9A0682843A060012070BDA6
:1004E00070B50124744D8440EC6020F07DF9A8685B
:1004F0002043A860012070BD6F480121C90310B5D9
:10050000C160704A136A6F4C0023403C2360136241
:1005100082680A438260012010BD674801210904F6
:1005200010B5C160674A536A664C0023403C636063
:10053000536282680A438260012010BD70B50124B5
:100540005D4E8440F46004F041F8050003F03CFB8C
:10055000002805D0680509D52A2018F0F1F905E032
:10056000680703D504F020FA04F087FA280004F0A5
:1005700038F8280004F03AF8B0682043B060012051
:1005800070BDFEB5404D4035EC68E00702D0A817BD
:10059000E8600440600704D50420C043E8600420FC
:1005A0008443200606D58020C043E8608020844331
:1005B00054F0B4E8200709D50820C043E8600820BB
:1005C000844322F00BFD082002F0A0FFA00606D510
:1005D0002020C043E8602020844303F0A0F92004D9
:1005E00007D50126F603300054F098E8F043E860A0
:1005F000B4436003400F06D00720000421000140EF
:10060000C943E9608443244F2002000F002671375C
:1006100000282FD0200221D51B494039C8688A0103
:100620001043C86028480068002803D188048078F7
:10063000800702D401200005044304F007F80028D5
:1006400004D0012003F038F903F054F9BE7480207F
:1006500004F05BF80120C00554F060E80F200005AD
:100660002040019002F07CFE0198C043E8600F201A
:1006700000058443E000400F30D007208006204072
:10068000009023E00029008040200080087601C00F
:10069000400001003C6405000F000080FF0C0000DA
:1006A000070080FFB447000478FC00040C7B0500C1
:1006B0002B03000000300080002800802864050023
:1006C000286A050080E80080006A050002F0B7FD96
:1006D0000098C043E860072080068443E00610D5F8
:1006E0001020C043E8601020844304F0CFF80028B5
:1006F00007D00EF07EF9002803D0BE74102002F05F
:100700002FFC600003D52748E860C0438443A00065
:1007100003D52548E860C0438443002C23DA012038
:10072000C00702F0A7FD2148E860214800780128B1
:1007300019D12048006800281CD01F48C1688201D8
:100740001143C16003F082FF002804D0012003F0B0
:10075000B3F803F0CFF8BE740920000502F000FEE4
:10076000002004F0F5FA154988680122920510432B
:100770008860FEBD01200005F0E7104B01229205C4
:1007800010B5DA60FFF7FDFE012010BD70B5012540
:100790000A4C2D07E5600DF010F8A0682843A06012
:1007A000012070BDFFFFFFBFFFFFFFDFFFFFFF7FE7
:1007B000A2640500006A0500002000800028008077
:1007C00010B50400002A03D0200003F01FFF00E052
:1007D0000024200010BD7CB50C0015004979237958
:1007E0000906091419430B198188426924336029C9
:1007F00014D9603920328180517EC906CA0F009217
:100800002A0001A905F0CFFAA071000AE071019851
:10081000001B2071000A607101207CBDBB5EA33FFC
:1008200001000000F80700000004000009358D7F7A
:1008300000207CBD30B5040020202081656920188F
:10084000AD7A05706469E47A44700171090A4171F6
:10085000110A8271C171190A8370C17030BD0028FC
:1008600010B507D00169002905D14189C08803224C
:100870000EF0E0F910BD53F034EF10BD10B5018952
:10088000C1220818418D0024D200914208D10100F4
:10089000062212310C3053F044FA002800D1012412
:1008A000200010BDF0B50400002085B006000390C4
:1008B00002900190208901270519A8780007800F70
:1008C000022800D000276069407A02280BD120005E
:1008D000FFF7D4FF012806D12020A6802073FF490E
:1008E0000869401C0861A08800287ED0002F2CD009
:1008F00017F083FF002828D015F010FF002824D11E
:1009000015F0F6FE002820D120890519E978C807DE
:1009100001D1A81D01E028001230F14A537C002BC0
:100920000DD01289092A0AD10078C00707D088069D
:1009300002D518F0A6F808E00120019005E00BF0C0
:1009400084FD012801D018F077F80EF0A6FF0028EA
:1009500066D0280005F0DEFA002859D1002F12D009
:100960000122200069460FF0E0F900280BD0009822
:10097000002800D0012000284AD000214F200EF08E
:100980002DFD039008E0200002A90FF0CFF8002809
:1009900000D0012000283BD00EF07FFF002846D079
:1009A000D04D01242C6118F006F817F012FF002832
:1009B0000BD118F037FA002807D1CB480660CB4896
:1009C00006800320AC7017F0C5FF0399FF200EF0DE
:1009D00084FFC74C2088002804D0C649042008564C
:1009E000401C0BD00224012000E00FE004F05EFA6E
:1009F000641E07D0287A0028F5D103E00EF039FFF5
:100A000026802E721D2017F0A5FFEE6005B0F0BD08
:100A10006B46187A00280AD12020A680207306E0B1
:100A2000002F04D00222200069460FF07EF90198C1
:100A30000028EBD01B2017F08DFFE7E7FFB581B052
:100A4000002206000D000398417800780F0207434A
:100A50002037380034300104A748090C53F06CEEFD
:100A6000040036D038001430A08020206661208138
:100A700020181421009053F064EE3B04049A1B0CE0
:100A800014212000FFF7D6FE002D12D028892E0059
:100A900028811C360B20072130567156401A0CF065
:100AA000F1FF00990873072030560CF0DEFF009923
:100AB000487334202081039920183A0053F044EE03
:100AC0002000FFF7EFFEA088002804D12000FFF7E8
:100AD000C6FE00209AE72020208117F0A3FE002800
:100AE00002D0052017F036FFFFF732FC844B0500DB
:100AF000824821001C68002200680523A0472800C6
:100B0000FFF72BFC012081E7FFB50120904083B067
:100B1000039F0406240EFF378137387A0E00150034
:100B200020422ED1FF229132462301A902A80EF0C5
:100B30002BFC002825D0387A182120433872019CDC
:100B40001034200053F0FCED0698002801D1052058
:100B500000E00D20607225722000627A0C990A3044
:100B600053F0F2ED310006220C31A01C53F0ECEDF5
:100B70000199182088720020C872029903980EF01B
:100B8000CFFB07B0F0BD1A002FE68288602A10D98B
:100B9000603A828048790A790006001410432430B4
:100BA0000871000A4871E62088710020C871012090
:100BB0007047002070471FB501AA0400009202AAE6
:100BC00003AB18F0F2FC019802040298121401041D
:100BD0000914200018F05DFE20000399C030418206
:100BE000019981820299C18220000FF009FC1FBD8A
:100BF000F1B5002486B027002600250005A853F093
:100C0000A8ED0028BDD06B46587DC10601D48006F2
:100C1000B7D56B46187D0007000F0128B1D10190B0
:100C2000384800780128ACD00EF037FE473EF42D4E
:100C300001000000F40B000000040000FD5AF8CB96
:100C4000002803D006980EF0D2FDA4E732480078C1
:100C500000280AD16B46987D05072D0F08F007F98B
:100C6000060007D06D086D0004E0012802D16B4634
:100C7000987D05091E4906980968884209DA1C48CA
:100C80000699406881420ADD1948012780680028DA
:100C900081D0012453F06AED1549C8610DE053F08D
:100CA00066ED1349C96905F053FE1C49884204D812
:100CB0000F4880680028C8D001240D488168A142EF
:100CC00001D0002F04D0002CBFD0C168B142BCD0ED
:100CD000C6608460104802A9007853F04CED6B4662
:100CE000187D2B000207120F0092220002A817E0C5
:100CF000740C0004785F01C020840500143501C025
:100D0000DC690500CC690500E0680500200D0004E1
:100D10002C6405009C67050058650500404B4C009D
:100D2000019903F07FFF36E7F8B505000C000027B6
:100D3000FFF718FB0090E168A06800232E005940DF
:100D4000584008433BD0A088A779FD4BC1194039D2
:100D50002A1A8C460100D21840315B009A4205D90C
:100D60009A1CA84201D2AE1A00E0AE18664524DDF6
:100D70008E4222DAB0420FDD801B0604360CE16899
:100D8000A068320053F0FAECE160B919A1710121B9
:100D90000843A580A06018E0301A0204120C9742A4
:100DA00000D2A2710021012053F0E8ECA268E368B0
:100DB00010431943E160A06007E00EF0D0FB002073
:100DC000A5800121A071A160E0600098FFF7CFFA33
:100DD000F8BDF3B595B0050000200790049003908E
:100DE00016980A27002879D028896E69411920228F
:100DF0000AA853F0B4EC0AA808AB0990D87AC10746
:100E0000D0486844149002D10998801D00E01498DD
:100E100005901698183053F0B6EC08AB997A000795
:100E2000C40F0A070020920F022A03D109090907FB
:100E300000D501201699204320310028139124D099
:100E4000FFF790FA01901398BF4A007E4107099876
:100E5000490F0C3004F0A8FB07000A2812D2002C1E
:100E600005D0B94839010818C168491CC160A88873
:100E7000002807D1B5493801411810AB188800097E
:100E8000FFF752FF0198FFF772FA16990B200856E8
:100E9000FFF7B8FE288920216C182038298120719D
:100EA000000A10AB6071188800092072000A607295
:100EB000B07A2070F07A6070307A06280FD108ABD3
:100EC000D87A80070BD4A07C01210843A0740D20A0
:100ED00080013018C16A491CC16204E008E1A07CAD
:100EE00040084000A074A888002802D1287B202850
:100EF0003ED108ABD87A800601D50120039008AB1B
:100F0000987A0107890F022932D10009000721D5FB
:100F10008F48007800281DD015F0BAFE002819D09F
:100F20001398007EC00615D58A480068002811D0A5
:100F30008948006800280DD016F007FE002809D067
:100F40000EF068F8012805D084480068002801D117
:100F50000120049017F070FC002809D0099804F0D3
:100F6000E3FF002804D102201DF061FC14F078F9A1
:100F700016993000FFF729FE3000C030162112907C
:100F8000415E08000CF088FD207312981221415E2A
:100F900008000CF074FD08AB6073987A0009000734
:100FA00004D51398007E4007400F00E0FF20A07298
:100FB000A888002804D0099804F0B6FF002872D051
:100FC0000027A770E770A888002802D1287B202876
:100FD00045D1A07A16F068FD002809D003980028B2
:100FE00004D0002130000AF0BCFF01E05C4807702B
:100FF00005980078C00715D107F039FF002813982D
:10100000007E07D0C006C30F049A0399300008F091
:101010004FFF06E0C006C30F049A0399300009F0A1
:1010200008FB049008AB987A03990209300016F087
:101030001EFE0498012812D14A480088C0056C7F22
:1010400001000000F00F000000040000AE802BA79C
:1010500000280BD0494800220068462153F04CEB91
:10106000002803D046490120087002E0162017F03E
:1010700085FCFFF781F90700099804F05FFF00285D
:1010800015D0404E3068002811D020001499062257
:101090001A3053F06EEBEB20A07100200200E071DB
:1010A00039483468290000680523A04702E0280079
:1010B000FFF7E9FB380023E0FFE71398007EC00943
:1010C0000DD0169A21002800FFF773FD00281CD1CF
:1010D0000020A070E0702800FFF7D5FB12E0099B0C
:1010E000169A21002800FFF762FD00280DD1A0709C
:1010F000E070FFF741F904002800FFF7C4FB20006F
:10110000FFF73FF9002017B0F0BDA888A070000AD3
:1011100022000B32E0701698D11C04F03CFE707A6D
:1011200002287ED130001CF0A1FD0B218901069020
:101130004018007A0190002008AB0890987EC00704
:1011400024D0012008900198C0076AD00198800738
:1011500067D43BE0FF0700003A0000005849000454
:10116000484A00040669050018690500146905006D
:101170006C690500056905006086050028640500A6
:10118000026905009C6705002C64050014981DF099
:10119000A2FC0028079071D0707A02286ED10798BF
:1011A000407BC0066AD50798F17AC07A81427ED129
:1011B0000A2F63D301984007019802D4C0075DD07D
:1011C00004E0C00784D00198400781D4FA48002287
:1011D0000188FA48032318F0B0FD002800904AD097
:1011E0000099A888888000F04EFE00990004000C49
:1011F0000881009908220A73009940181221019071
:1012000053F0B2EA01981421017100214171E17992
:10121000A0790902014301988171090AC1710698F8
:1012200000E02BE0406A012808D10798002805D08B
:10123000707B000702D50198A17A0173607921794A
:1012400000060014084301190198AA88143053F0CD
:1012500090EA0099306948610198F17A41700198EB
:10126000B17A01700199A8888870000AC870009846
:10127000042100F0F5FD08980028A3D017F0E6FA45
:10128000002802D0052017F079FB0A2F0BD2CC489A
:1012900039010818083003C8002358405940084352
:1012A00001D00EF066F9FFF767F8002200E024E0B5
:1012B0000290C54BC34829001D6800680523A84754
:1012C00005000298FFF75DF8012D09D10A2F07D21A
:1012D000BB483901091810AB18880009FFF72EFD2B
:1012E000A07A16F0EBFB002813D0039801280AD14E
:1012F000002130000AF03FFE0BE001980007BDD549
:101300000A2FBBD3E4E60398002802D1AF4800219E
:10131000017005980078C00715D107F0B2FD0028CC
:101320001398007E07D0C006C30F049A03993000BB
:1013300008F0C8FD06E0C006C30F049A0399300008
:1013400009F081F9049008AB987A039902093000FA
:1013500016F097FC0498012812D19D4800880028B7
:101360000BD09C4800220068462153F0C6E90028B3
:1013700003D099490120087002E0162017F0FEFA08
:101380000120C0E6FFB59FB00600080037680021C5
:10139000179121997C69002910D040301E9053F09C
:1013A000FCE9229905004118C0782031400602D49A
:1013B000B88823B0F0BD2888682801D80020F8E755
:1013C00019AA18910092219918981AAA17AB04F03B
:1013D00073FD280004F0AAFD002853D07F480021A7
:1013E00004AA01AB07C318AB7D4A00921D7910AB6C
:1013F0001A7F38002B001AA907F0F1FA05002DD149
:101400002000FF308130017A090624D5002C0CD051
:101410000B21890161184968002906D018AB1A7997
:10142000920068328B585B1C8B50017A4906490E3A
:1014300001721E9853F0B0E918AB1D7921992A0169
:10144000521B52180E320092010010AB8912563E08
:1014500001000000EC1300000004000011450E1410
:101460001B7F2A002000FFF76DFB00203060AFE7F4
:10147000356028891E99401952F03EED0088A880F9
:101480002000FF30813018AB1B7901263200017A31
:101490009A40914301721DE010AB197F00910195B4
:1014A0002A8818991898643A091D1AAB04F0A4FF09
:1014B00006001CD0200018AB1A79FF3081300123C0
:1014C000017A934099430172288808382880B888A7
:1014D0000838B880002C08D00B2080012018406804
:1014E000002802D0416E491C416630006BE7002C99
:1014F00014D00B2080012018416800290ED018ABB1
:101500001A79920068328B585B1C8B5041680A69CB
:10151000521C0A614068C168491CC1601E9853F0A2
:1015200046E9010018AB1879219A03011B1A9A1891
:101530000E320092020010AB1B7F2000FFF702FB6F
:10154000D3E700280CD00B218901411848680028F6
:1015500006D00269521C02614868C16C491CC16412
:10156000704701207047FFB583B004001E000C9F38
:101570000E9D1EF09BFC002821D0607A02281ED010
:10158000082E1CD3082F02D3012007B0F0BD38006D
:1015900006F09DFF03008000BB250019AD00119AE5
:1015A000109940196D4607C55800BF2100198900E0
:1015B00043180D9A0599049804F030FBE5E70FA84D
:1015C00007C86C462B0007C4F3E70000EA69050072
:1015D0000C0D0004484A00042C6405009C670500BB
:1015E000056905006086050028640500026905009C
:1015F00064F70500645601C0F7B592B014000F00FF
:10160000129800680D9000200A900D984569080016
:101610004030119053F0CAE80600243009902800A9
:101620001DF0E9FE21002C311091091D2037002802
:101630000F9122D0109807AA08A903AB07C36B46E5
:10164000E0790F9A0107387E090F4007400F07C362
:101650000021B078099A03092800FFF784FF0028C9
:101660000BD0002D08D00B208001281840680028DE
:10167000F8D0016D491C01658AE030886828FBD9E3
:1016800022004C3268380304111F081F0692021F03
:101690000591049003920C3938381C3A029101905C
:1016A0000092387E1B0C47077F0F1A000999300003
:1016B0003B0004F0DFFD0700300004F041FC00288F
:1016C0003ED00AA9009100200BAA01920A900D9B1E
:1016D000099A3100380004F054FA002858D0FE4A24
:1016E0000092FE4AFE4B0D98310007F0B0F800283A
:1016F00002D1129908604BE0129906000860018936
:101700000818119952F0F8EB0E900A9800284AD068
:101710000BAA009209990E982300320004F060FA97
:10172000070040D1002D08D00B2080012818406808
:10173000002802D00168491C01600E98807922E0DF
:10174000002F28D03807800F0FD0002D20D00B207D
:1017500080012918486800281AD0C26C521CC26443
:1017600048680169491C016112E0B80710D5002DD5
:1017700008D00B20800128184068002802D001689A
:10178000491C0160B079C107C90F28001BF0F0F9AE
:10179000002015B0F0BD3088143830800D980D99B8
:1017A000808814388880079C6B461A8C10990F9893
:1017B000230004F030FA002F0AD1002D08D00B20AE
:1017C000800128184068002802D0416E491C4166FB
:1017D0000120DEE7F7B582B0140000250298076803
:1017E00003980197403052F0E2EF0600C0787F691D
:1017F000400605D42037B87E400732D4012530E0BA
:10180000002C02D1002005B0F0BDA07AC00721D085
:10181000E0790007000F012805D10399220001A8F3
:10182000FFF7EAFE05E003992200042301A8FFF771
:10183000B3FD0299050001980860B079C00710D186
:10184000002D0ED0A07980070BD52100380001F0C3
:101850009BF806E00B208001381840688F328922FF
:1018600001000000E817000000040000429FDD783E
:101870008168491C81602800CFE77FB504000E0015
:101880001D00142152F0A0EF25606B46A672188946
:1018900020817FBDF0B5C36802691900114301D1F1
:1018A0000020F0BD0125002B0DD0002A21D11F21E1
:1018B0002A008A40134203D1491E0906090EF7D1B6
:1018C000CB40C3600CE0002A13D01F212B008B40BB
:1018D0001A4203D1491E0906090EF7D1CA40026116
:1018E0000289130712091B0F511809010B430381C9
:1018F000D6E700210C000F008C468E4601E0002C3C
:101900000ED101258D402A4222D0002920D04D1E23
:101910000126AE401D0035421AD001240F0017E009
:1019200001258D4016002E4212D11F2910D21E0013
:101930002E420DD00124BC406D1E641EA54364469A
:1019400025434C1E2406240E0027A6463C00AC4628
:10195000491C0906090E2029D1D3714600290CD053
:10196000CB40CA40C360026101890A070B09714676
:10197000120F591809010A4302816046F0BD70B583
:101980000400008988B006092000FFF783FF0028C3
:10199000019023D0182102A852F016EF21680622E8
:1019A000FF318B3102AD03A852F0F6EEA07A6B4600
:1019B000987428000422103001A99E8252F0ECEEA7
:1019C00004206B46D882FF209A301881102058815D
:1019D00020681423592102AA0DF089FD08B070BDBA
:1019E000080000214160CAE7F7B582B00C00FF276C
:1019F00004980026403052F0E4EE05002168029879
:101A0000814253D1A8780107890F02294ED10009DC
:101A10000DD004280AD0082802D00C2808D10126AD
:101A200004982030007E47077F0F01E00126002741
:101A3000A07AB8423AD1288B218900090909401AB5
:101A400001D420281BD360680027002802D003F0AF
:101A5000AAFC67602000FFF792FF288B218900090C
:101A60000A09801A01D4202809D3E76008072761F2
:101A7000298B000F09090901084320810020012159
:101A8000002E04D0226981400A43226103E0E2680B
:101A900081400A43E2606068002807D1002200927A
:101AA000154A1648231D210003F02BFCB5E6F0B5BE
:101AB000002599B003950295B0E10020059002F051
:101AC000B8F80D980007C00FC0000490069801896F
:101AD000081807A952F085FC1798002810D106981D
:101AE00000218180FEF7E3FE98E10000585601C016
:101AF000605601C064F70500400D0300591900004D
:101B000017980C301CF0FBFF040005D11799012039
:101B100012311DF017F80400179920000FF082FA17
:101B20000028DCD1002CDAD006994C61607A0228BA
:101B30000CD120001BF01DFF0C300290607B179A27
:101B4000C0060699C00F04F0B5F81DE0207A012800
:101B50000AD0062812D11798C078820701D4C0078E
:101B600012D0002088800FE02300179A9C330120B8
:101B700004F0AAF820001DF0D2FB05E02300179A1C
:101B80009C33012004F0C3F8069801890F18F978F6
:101B9000C90701D1BE1D01E03E0012360B218901AB
:101BA000611818914968002902D00A6B521C0A6317
:101BB0003178C90706D018994968002902D04A6BC4
:101BC000521C4A63818800296CD00499002943D1B2
:101BD0003178C90736D1B8780007800F02283BD189
:101BE0009F49200007AAFFF7FFFEB87800090C28DC
:101BF00015D0082804D110AB187D4007400F00E035
:101C0000002003900A224000009202191300FF33C3
:101C1000FF32179906987933693204F0ADF80698C7
:101C20008088002818D1200007A9FEF7ECFF06984D
:101C3000FEF73DFE18984068002802D0016A491C52
:101C40000162EBE0312109016218390004F083F8E8
:101C5000069880880028B7D0607A022827D1200013
:101C600007A913F0FBF817990298C9787F30D94E6D
:101C700001000000E41B000000040000B6F0A8CC46
:101C8000007EC906C90F884202D0200012F098FFDA
:101C900020000FF056FB200010F004FD012803D1B6
:101CA0001799200012F0E7F802984030007D0328D1
:101CB00003D006990020888099E006988088002843
:101CC000FAD03078C0070AD101F0BAFF002806D157
:101CD000069808AB8188DA7D07A808F0C5FD17983B
:101CE00004F034F8002812D00698634A8188644BC7
:101CF0004039818000920189604A091806F0BBFDD5
:101D00000028A8D006900189081817906FE017984E
:101D10008079C0075B4828D02218906A00282AD012
:101D2000617A032925D11799083005002431C97833
:101D30004030007C8909884204D153488169491C9C
:101D4000816118E0D06A00280AD008305022125C65
:101D50008A42F2D14C4905004869401C48610AE0BA
:101D600049498869401C886105E02018006B0028FB
:101D700001D005000835002D4ED0E9790807000F85
:101D8000022801D0032813D1039A1799520012197F
:101D9000FF326132128B0120002A00D0002004F0B3
:101DA000D0F8069833002A0007A91EF0F1FC17E0CE
:101DB000012801D0080729D100201EF01DFB0028B2
:101DC000FAD12A0007A906A8FFF718FD002804D1B8
:101DD000069800282CD0002181800598002806D084
:101DE000E8790007000F022808D0032806D00698DB
:101DF000FEF78AFD069807A9FFF713F808F063FFBE
:101E0000002815D0012008F0B2FF1AE01F48FEF7A5
:101E10005FFA03F0FFF8EAE7189840688168491C08
:101E200081601798BF21C07808401799C87040E7B3
:101E30000121002007AA0BF09BFA0028069000D091
:101E400045E613498020C04308610CF0B9FF002823
:101E500002D0042008F08BFF0E490020C860086102
:101E600019B0F0BD0C4A01000120914200D00020C1
:101E700070470000707B0500585601C0605601C0D5
:101E800064F7050080020000740C000402000100E9
:101E900000A5008020840500888E000002220B002F
:101EA00010B5010002730D481C22006852F03EEC90
:101EB00010BD40690069704710B540691CF0E9FF2A
:101EC00010BDB0207047010005A010B552F08AEC9B
:101ED00010BD10B5406920F08AFD10BD2C640500CE
:101EE0007364696F00000000F3B50024060025004C
:101EF000002881B014D0707A022811D002E00120AD
:101F000003F006F828006D1C022807D20022F948C9
:101F1000110052F044EC0400F1D00AE0002C08D18A
:101F20000022F5481100032317F025FF040000D11B
:101F3000FEBD6661FFF7C5FF0004000C2081082785
:101F4000051914212800277352F02CEC30001DF0E5
:101F500031FF28731420287100206871380AAF718E
:101F6000E871B07A2870F07A6870029814350560CC
:101F70002000FEBD10B504000321323052F012ECF7
:101F800020001C21353052F00EEC2034A07D0121C0
:101F90000843A07510BD70B50400FFF7EBFF2000EB
:101FA000FF30FF220421953052F020EC2000FF2169
:101FB00054304131050052F012ECFF34413401211C
:101FC00000206161A0612074280006F01BF970BD3B
:101FD0000321090270B54418A169002927D1007AAC
:101FE000002803D0032801D0042820D1FEF7E2F90D
:101FF0000500C2480021FF2299324A438258002A34
:102000000AD1FF239933594301220E184250300060
:10201000FFF7C1FFA66102E0491C0229EBDB2800A3
:10202000FEF7CDF9A069002801D102F0F3FF70BDE1
:102030000321090240188169002902D000220A60A8
:102040008261704710B50289123112189170090A25
:10205000D1700F21FFF722FF10BD0A0003210902F2
:10206000411810B58969263152F0C4EB10BDF0B5A6
:102070008FB00600149D159C1700092992E386C4B1
:1020800001000000E01F000000040000E52A7BA022
:1020900016D1382101A852F0ACEB04206B46988091
:1020A0009C48D88002A806223900801C1D8152F06D
:1020B00088EB04A82A002100801C52F082EB05E086
:1020C00023000022290001A805F0BDFD300001A970
:1020D0001FF039F80FB0F0BDFEB50C3A0D00140634
:1020E0000700240E1021102C00D82100032000022C
:1020F0003E18B0690A00FF3029006D30083152F0F7
:1021000060EBB2690094FF326D3201922B78AA1C09
:1021100009213800FFF7B5FFFEBD10B50400080027
:102120004979C90615D5010060318A784B781102CA
:1021300019430922633005F054FE002809D0032119
:10214000090261188B694278811DA4332000FFF7D2
:10215000C3FF012010BDF8B50D00060006F043F8DE
:10216000040025D029002A00AC3150322000009113
:1021700005F06AFE01206867E81DF93007008068F5
:1021800003F025F90021B9602079022812D120003E
:10219000603081784078090201432000009A633062
:1021A00005F03EFE70692100FFF7B7FF002811D14E
:1021B0000020F8BD20006030817840780A02024398
:1021C00021000098633152F0FCEAA0798006800F6C
:1021D000C03568822000F8BDF3B581B00C000198CD
:1021E00006F001F805001ED00121F8200153002659
:1021F000F42006516879C00622D5E01DF9300700A9
:10220000806803F0E4F822002100AC3150320C0069
:102210002800BE6005F018FE019829004069FFF70C
:102220007CFF002801D10020FEBD280060308178AD
:1022300040780902014328002200633005F0F0FDD8
:102240002800FEBD03210902401810B580695430F2
:1022500006F080F810BD7CB50C00150006990091C1
:102260000321079A09024018019280692A0035303B
:10227000210005F037FB7CBDFFB585B00E001D00C9
:102280000189446908180390200004A9FFF736FE6D
:10229000070002D1012009B0F0BD03200002009622
:1022A0002618B2690399130004982C33263205F0DE
:1022B00033FE0498817C012910D000220092019203
:1022C000B269010013002C33263271312000FFF770
:1022D000C2FF04996031C873000A08740799049812
:1022E0002B00012205F041FD01003800FFF7B4FE8C
:1022F0000020D0E703221202801810B58069353023
:1023000005F025FC10BD0000D80D00040C0D0004E4
:10231000847B05000404000010B504008EB06846FC
:1023200005F091FC200069461EF00DFF0EB0E9E7B4
:1023300070B50500032000022C18A06928220100B6
:10234000FF312931D83052F064EA01212800FFF72B
:10235000D1FFA3690100D83301222800FFF7DCFF79
:1023600070BD10B544692000FFF7E2FF03200002B2
:10237000201881690122C0310A618069C03040693A
:10238000002803D0817AFD22114081720020B9E734
:1023900070B5002145692800FFF7ACFF0321090251
:1023A0006C18A3690100FF335B1C00222800FFF7B3
:1023B000B3FFA0690121C0308160A069C030C2684C
:1023C000002A03D1C160280052F026EA002070BD27
:1023D000F7B584B005000E004769008903A94019CC
:1023E00002903800FFF78AFD040002D1012007B0F7
:1023F000F0BD032000220002381800928269029981
:10240000130003982C33263205F086FD3100039823
:1024100001224031002305F0A8FC0700706F00285E
:102420000BD0607B0121084360730698002801D01F
:10243000FB4800E0FB48A06109E00698002803D0B3
:10244000280000F0E5FA02E02800FFF78AFF3900D3
:102450002000FFF701FE0020C9E7FEB50E0001894C
:1024600045690F18280001A9FFF748FD040001D1B4
:102470000120FEBD0320002200022818009282697C
:10248000019813002C332632390005F031B5FEAA2D
:1024900001000000DC23000000040000CDBBFE1D95
:1024A00045FD3100019801224031002305F067FC11
:1024B000617B012211436173E049A16101002000A9
:1024C000FFF7D4FD0020FEBDF7B586B00321090259
:1024D0000698002640694518AC69069854342100D6
:1024E00005F08BFE070016D0A8693A3005F0BCF95C
:1024F000002829D0A8693A3005F0CAF90028A8694F
:1025000004D04179801D17F0BBFB02E0263004F0B7
:102510009CFE060001D10020C7E6A8693A3005F00C
:1025200091FD020021002000D431503002AB07C3DE
:1025300022004032B43901920091079A0899230091
:10254000300005F002FE01262200210006984032EC
:1025500020310023FFF79AFE002801D0002608E072
:10256000012E06D139000931200005F046FB00207C
:10257000A067300099E670B50500406903210902A3
:1025800040188669280054363100FFF72FFE0400FA
:1025900001D1002070BD20790122022800D0002244
:1025A00031002800FFF71EFF002801D0200070BD79
:1025B00021000931300005F020FBEAE770B5050085
:1025C0004069032109024018866928005436310009
:1025D000FFF7CBFD04000AD031002800FFF747FFCA
:1025E000002804D121000931300005F006FB00204D
:1025F00070BDF8B505000E000089170040198179FB
:102600000024090716D54079C00709D02800FFF734
:10261000B2FFF8BD012002F08FFC641C2406240EDA
:102620003A0031002800FFF74FFF0028F1D1072CB6
:10263000F0D3F8BD2800FFF7C1FFF8BDFEB50C00D0
:102640000600086F1700401C06D1E06E401C03D145
:10265000200005F0EBFDFEBDFDF7C0FE050002E029
:102660000021FDF73BFE764852F0E4E80028F7D160
:102670002800FDF7B8FE300001A9FFF749FC05006E
:10268000E9D00320000236180094B26901981300C3
:102690002C332632390005F093FCB0693A3005F04E
:1026A000D1FC0200B0692030417E807D0907CB0F4C
:1026B0008006C10F019805F08CFDE06E401C0128DA
:1026C000E06602D1206F401C2067210001980122A2
:1026D0004031002305F053FB01002800FFF7C6FC42
:1026E000FEBDF3B581B00600032000023518A869CD
:1026F0000400FF305530070000685434002820D013
:10270000FC20005D00901AF07BFF029A210030004F
:10271000FFF794FF0098002814D0012811D1A86970
:10272000484A2030017D0823491C0175009821008A
:1027300005F0F0FD444A4549200008237E6105F07C
:10274000D5FDFEBD3F4A00982100082305F0E2FDBB
:10275000A8692030C17C491CC174FEBD70B50E0053
:102760001100032212028418A569FF225435153284
:102770005051A06906222C3052F02CE8A0690622A4
:102780002630310052F026E8314A32492800082329
:1027900005F090FD70BD03210902401880690028F2
:1027A00003D02030407DC007C00F7047FFB581B017
:1027B000050016000A9FFFF7EEFF002812D0280040
:1027C000FFF74AFD032000022C18A0690299801D22
:1027D000320052F000E8A0693A00467104992800DE
:1027E000FFF7BCFF05B0F0BD032109024018806966
:1027F000FF30413080690006000E70470321090256
:10280000401808B58069C08E009008BD020010B560
:10281000FFF7C1FF00280BD00320000210188169C8
:1028200020314A7D520852004A758069FFF7B6FB95
:1028300072E5000061290000B3220000E1220000DF
:10284000E84A000475810000409C0000A18100005E
:1028500080969800C9810000032109024018806910
:1028600001222030417D11434175704770B506004B
:1028700086B014000D000AA807C8002901D10591EF
:1028800005A9009301AB07C303200002301880693B
:1028900023000100FF31953135302A0052C27412F5
:1028A00001000000D8270000000400009E612D7187
:1028B00004F0E3FE06B070BDF0B506000320000290
:1028C0003418A0690F0041791500801D8FB017F0F2
:1028D000E1F9002810D001002B003A0001A805F012
:1028E00012F9300001A91EF042FC3000FFF7BEFCD7
:1028F000A0690121C030C1600FB0F0BD70B5050006
:10290000032000022C18A0692030417DC90712D095
:10291000817DC9060FD5007E00220007C10F280067
:10292000FFF7CAFFA06901222030007E0007C10F17
:102930002800FFF7C1FF70BD0FB503210902401841
:1029400081696B46FF319A8881318A8281691A7A5E
:10295000FF3181318A758069197BFF308130C17503
:102960000FBD30B50324240200198469FF3481347B
:10297000257D0D70647D4C708169FF318131897DC9
:1029800011708069FF308130C07D187030BD30B566
:1029900003242402001984692034A57D0D70E47D90
:1029A0004C7081692031097E117080692030407E31
:1029B000187030BD0321090210B54418A069002821
:1029C0000BD0FF304130C069002806D002F013FD63
:1029D000A0690021FF304130C161A7E4EAE703218B
:1029E000090240188069FF306D30704703000A000B
:1029F00000B5FFF7DAFEFD21002814D00320000205
:102A000018188369C0335A6180690300C033002AF3
:102A100008D02030407DC00701D0186909E0907AC5
:102A20000840907200BD002AFCD0187B4307F6D501
:102A3000C0070028F3D100BD10B50400FFF7A5FCC6
:102A40002000FFF7B9FC002070E470B50025038971
:102A500044691B185E78002E0BD0032E14D1637AC4
:102A6000022B02D120F081F801E0FFF7CCFD012517
:102A70000AE0607A032801D0012805D118790128DD
:102A800002D108000FF05AFD280070BD10B517F0F4
:102A900023F9002010BD0000F94810B500680200BD
:102AA0008030016803680901C90EDB00DB0F1B02DF
:102AB0001943F44B9980016801231B0719430160F6
:102AC00001681F23DB0599430F23DB05C91801604B
:102AD000ED490869ED4B800502D508699843086106
:102AE00008680124E4072043086088682043886060
:102AF000D069240CA043D06108691843086110BD57
:102B0000DF4810B500680200803003680121090722
:102B10008B43DC4989880C0AE407E40823430360FB
:102B200003681F24E405C906A34309090B43036096
:102B3000D54908698B0D98430861D369080C034394
:102B4000D3618868400040088860086840004008F9
:102B5000086010BDF8B50027CA4D3C0069692869B6
:102B60003E0079407840084303D002F015FB060090
:102B70000C0024F035FC51F04EED24F03EFC696968
:102B800028697940084309D002F006FB2A69801BB6
:102B90006B69A1418018594169612861F8BDF8B598
:102BA000040001F0C3FD002843D001F0B7FDB8498F
:102BB000012080058860C01151F04AEE01F035FE19
:102BC00001F078FEB04D403DE868EE0BB043E860A0
:102BD000AC480078C00721D0AE4F062C0FD0AE49CC
:102BE0004868012210434860802001F0E2FDF001B6
:102BF00051F02EEE0320B874642023F0FFFB012077
:102C0000C007807806210840A04201D151F002EDB2
:102C100001F076FD002803D1B87401E051F0FAEC20
:102C2000E8683043E86001F008FE01F04CFE01F076
:102C30006DFDF8BDF0B5002425002600270085B005
:102C4000FDF7D6FB039000F081FD00F038FF8D48C2
:102C500008300068810702D5C10700D001240107B0
:102C600002D5410700D50125810602D5C10600D550
:102C70000126010602D5400600D501270120C00724
:102C800080780621084002907E480178C90724D048
:102C90000299490701D40124250002998078022273
:102CA0001140014315D1002E19D1002212ED4FF031
:102CB00001000000D42B0000000400006A0E58C57B
:102CC0007B48009200680822012101AB02F0A8F9BC
:102CD0000122009200221100100013000BF0BBFC37
:102CE000012821D105E07348006800281CD1002E7E
:102CF0001AD0002C18D0002D16D0002F14D0694DFA
:102D0000AC68E817E86024F043FB01007D20C001B7
:102D1000814201D824F03CFB042123F05EFB0298A1
:102D2000FFF747FFAC600DE024F032FB01007D208F
:102D3000C001814201D824F02BFB042123F04DFB7C
:102D4000FFF712FF0398FDF762FB0421002023F038
:102D500044FB05B0F0BD10B500F053FD00F027FFB7
:102D6000FFF772FF10BD10B5FDF74CFB040021F01A
:102D7000E1F821F0E6F82000FDF749FB10BD464AD6
:102D80000100083212680020914300D101207047F1
:102D900070B50400FDF736FB05003F4808300168B8
:102DA00021430160E00601D4A0062DD5C8062BD52D
:102DB000880627D501F0AAFD38498039C8683A4A03
:102DC000383A9043C86035488030416B3A4A1140E8
:102DD0004163314C607800280FD0D00780784008DC
:102DE0004000400709D40120FFF7C9FF002804D0A4
:102DF0000420FFF7C4FF002801D123F051FD00207B
:102E0000607001E001F082FD2800FDF700FB70BD5D
:102E100010B50BF09DFE002801D1284810BD2848B0
:102E200010BD10B523F06AFC26494000085A264B15
:102E30001A495843C03149680B071B0F51F016ED72
:102E4000080507060609090B0B06400810BD800897
:102E500010BDC00810BD000910BD10B5FFF7E1FF9F
:102E60001A49884201D11A4810BD1A49884201D135
:102E7000194810BD194A1A49904248D0194A90423F
:102E800001D1194810BD194A904231D11648D238A3
:102E900010BD000048650500A0640500802000808A
:102EA000000200000028008080000080C024008014
:102EB000F0710500006A05007FFFDFFF3F3D000065
:102EC0007F841E006E5B0500A0860100001BB7001A
:102ED00054150000405DC600B013000000F8240146
:102EE000540D000000366E01AA0A000080BA8C0161
:102EF000414A904201D1414810BD414A904201D11E
:102F0000404810BD404A904201D1404810BD0800E1
:102F100010BD70B50400FDF775FA05003C48016866
:102F2000A1430160E00601D4A00611D5C80601D571
:102F300088060DD43749C868374A1043C86001F085
:102F4000FDFC3649486B364A1043486323F0C2FC07
:102F50002800FDF75CFA70BDF8B52D4C083C02F076
:102F600025F9A269E369851A99410E00616900910A
:102F700020696422070051F07EEC33002A0051F0F2
:102F80007EEC00990600002538006940684008433F
:102F900009D101206561206102F008F96A1E8018DC
:102FA0005141E161A0613000F8BD194808380021A5
:102FB000016141618161C161704710B501F0FFFBA2
:102FC00010BD70B5040001F0FAFB041B23F09CFD5A
:102FD000050014490026200051F054EC33002A006B
:102FE00051F04CEC70BDC00005D509482830406850
:102FF000002800D00047704700F04902AA060000F0
:1030000000751903EB040000007C9200AA1A00006E
:10301000A864050000200080480000800021008096
:103020008000200040420F0010B504003020FFF760
:1030300070FF01F096FCE00602D51AF07DFB10BD92
:103040001AF01CFB10BD10B501F064FB002804D081
:10305000012000F095FC00F0B1FC0020FFF7E4FF38
:1030600010BD7047022910B505D0032903D00429EB
:1030700001D0052903D1B94BFF21491C9960042ACD
:1030800005D0052A03D0062A01D0072A07D1002837
:1030900005D100210A2208000B003DF050FB10BDB5
:1030A0007047042803D2AE498000085C7047FF20B7
:1030B000704710B50C000020FFF7F3FFCF865AC908
:1030C00001000000D02F00000004000039D48BA9BB
:1030D000A04201D100F068FA0120FFF7ECFFA04206
:1030E00001D100F080FC0220FFF7E5FFA04201D1F2
:1030F000FFF7B3FF10BD10B50C000020FFF7DBFF9A
:10310000A04201D100F06BFA0120FFF7D4FFA042EA
:1031100001D100F06DFC0220FFF7CDFFA04201D1EC
:10312000FFF7A9FF10BD042910B507D004DC022960
:1031300004D0032906D101E0052903D100F00DFADE
:10314000002800D0012010BD022910B505D00329A8
:1031500003D0042901D0052901D100F0AFF910BD39
:10316000022910B505D0032903D0042901D005296F
:1031700001D100F05AF910BDFF280BD07D4A002183
:103180008B00D35C834202D10806000E7047491CB5
:103190000429F5D3FF207047FF280CD0754A002181
:1031A0008B009B185B78834202D18800105C7047CB
:1031B000491C0429F4D3FF207047042804D26D4928
:1031C0008000401840787047FF207047FF280CD0DF
:1031D000684A00218B00D35C834203D188008018A9
:1031E00040787047491C0429F4D3FF207047FF281A
:1031F0000CD0604A00218B00D35C834203D188004D
:10320000801880787047491C0429F4D3FF20704748
:10321000F7B582B007000E000C2901D2092F02D3A6
:10322000002005B0F0BD00255249A8000A5CBA4252
:103230001ED14418A278B2421AD02806000E3900D6
:10324000019020F03DFF002812D0A670E07804998C
:103250004007400FC9000843E07001983200390070
:1032600020F030FF002808D0E07802210843E07009
:103270006D1C042DD8D30120D3E73E48AA00FF21BE
:1032800010188170E0784007400FE070C8E7F0B593
:1032900006000800374F002204219300FC5CB44272
:1032A00009D1DD19EC7823000B43002802D023005C
:1032B000FB242340EB70521C042AEED3F0BD2D4AB0
:1032C00000218B00D35C834206D188008018C0782F
:1032D0004007C017401C7047491C0429F1D3002047
:1032E000704770B505000C00100001F07CFA20005A
:1032F00051F082EA2800FFF74FFF022805D003288B
:1033000003D0042801D0052803D1200000F096F84E
:1033100070BD2000FFF771FE70BD10B50400C00045
:1033200005D50122120311040C20FFF7DAFF20015A
:1033300005D50122D20211040B20FFF7D2FF600154
:1033400005D50122920211040A20FFF7CAFF10BD21
:103350000120C00310B501F046FA0120C00751F06A
:103360004CEA054908698A0D9043086110BD0000C8
:1033700000280080C064050080200080F3B581B083
:103380000198FFF7F9FE04000198FFF71FFF050001
:103390000198FFF72CFF012706003F05022C02D100
:1033A000042D22D109E0002C01D0012C1DD12B1FAE
:1033B00051F066EA0403080E141B102001F013FA02
:1033C000380010E0202001F00EFA012040050AE04C
:1033D000402001F008FA0120800504E0802001F07F
:1033E00002FA0120C00551F05CEA0298002816D1CB
:1033F0000198FFF764FF002811D0331F51F040EA15
:10340000060F0F0F0F07040F0021102005E063497E
:10341000A0004018C0780021C00824F055FAFF220F
:1034200001991000FFF74FFEFEBD0800002110B506
:10343000FFF7A4FF5A490020887410BD10B504009E
:10344000C00203D501210220FFF798FFA00203D597
:1034500001210320FFF792FF600203D50121042020
:10346000FFF78CFF200203D501210520FFF786FF1F
:1034700001200007844205D04010844202D0401051
:1034800084421AD1FF208206A11808D0891804D0DE
:10349000C206891804D10C2002E00B2000E00A20AB
:1034A000FFF77AFE022805D0032803D0042801D0B4
:1034B000052802D10121FFF761FF10BDF8B5040016
:1034C0000E0017000800FFF792FE0500FDFB93F7C2
:1034D00001000000CC330000000400008611AE1A89
:1034E000002C01D0012C2AD13B1F51F0D4E9040358
:1034F0000C151E28102001F07AF9102001F083F934
:103500000120000519E0202001F071F9202001F0D0
:103510007AF90120400510E0402001F068F94020D0
:1035200001F071F90120800507E0802001F05FF9CA
:10353000802001F068F90120C00551F0A8E92B1F97
:1035400051F0A8E9060F0F0F0F07040F01211020FB
:1035500005E01749A0004018C0780121C00824F0F8
:10356000BDF9FF2231001000FFF7CFFDF8BD0100CB
:103570000020022910B518D0002901D0012913D14B
:103580000D4C00222068462151F010E900280AD194
:1035900020680022082151F00AE9002803D151F0E7
:1035A0008EE9002801D1002010BD012010BD0000CF
:1035B000C064050080000080286A0500022010B564
:1035C000FFF7BBFC01F0BAF8002804D0012000F09E
:1035D000EBF900F007FA23F0D0FC01E023F0B8FD8E
:1035E0000028FBD00021082208000B003DF0BBF8AA
:1035F00010BD022010B5FFF7DFFB10BD70B5002035
:10360000FFF763FD04000020FFF7E1FD0500012046
:10361000FFF793FC99494868022210434860984993
:103620001005886001F017F9082051F0F0E82A0031
:1036300021000020FFF72AFD70BD70B5FCF7F6FEF3
:10364000050090480068C00710D00020FFF7D6FFA3
:103650007D20C00022F0F0FE002051F034E904008B
:1036600002E0002051F02EE9A042FAD02800FCF739
:10367000E2FE70BD002010B5FFF727FD040000201A
:10368000FFF7A5FD020021000020FFF773FD10BD2C
:1036900010B5FCF7CBFE04007A480068800701D51E
:1036A000FFF7E8FF2000FCF7C6FE10BD002010B5B4
:1036B000FFF70BFD04000020FFF789FD0200210049
:1036C0000020FFF73AFD002800D0012010BD38B5DA
:1036D00001F034F8002826D1401E009069486A4C59
:1036E0000068C00711D06068401C18D0A068FFF7C0
:1036F0007CFC664951F0EAE800906168884201D399
:10370000002000E0081A009009E068463CF07DFEC9
:1037100000280CD000986060FFF763FCA06021785F
:103720000098884203D3FFF7C1FF002801D1002091
:1037300038BD012038BD534810B50068C00705D01A
:10374000FFF7C5FF002801D0012010BD002010BDEB
:10375000002010B5FFF7B9FC04000020FFF737FD8B
:10376000020021000020FFF7F9FC10BD10B5FFF7A3
:103770009DFF002804D000203DF08AF8002801D1E8
:10378000002010BD012010BD3E4810B50068800724
:103790000DD43F480078022809D1FFF7CCFF00285C
:1037A00005D0FFF7E3FF002801D0FFF7D1FF10BDE0
:1037B000F8B50020FFF789FC05000020FFF707FDA2
:1037C00034490600096817204883082051F05EE854
:1037D00001F039F801F02FF8294801214905C160AD
:1037E0002D4CC017009020680121084320603CF058
:1037F0002FFE00280BD168463CF007FE012806D1B9
:103800000098401C03D1206840084000206032002E
:1038100029000020FFF758FC18494868022290430D
:1038200048600120FFF7C8FAF8BD70B5154D28684B
:10383000C00722D1FFF74BFF00280BD1124CE068E4
:10384000FFF7D3FB1549884204D9FFF7CAFBE060B4
:1038500051F040E82868C0070FD1FFF738FF002873
:103860000BD0FCF7E3FD0400FFF731FF002801D087
:10387000FFF79EFF2000FCF7DEFD70BD40200080BA
:1038800000280080A8640500E8640500E204000048
:103890007772050054F90004FC64050080841E0062
:1038A000F8B5FCF7C3FDD74D07002868002830D1D4
:1038B00022F06CFF86211F2022F01EFF22F05CFF09
:1038C000D14E3068012109070843C9108843306090
:1038D00000F089FF040000F086FFA0427888949CE5
:1038E00001000000C837000000040000D5CB7D7641
:1038F000FBD030680921490608433060C849C869CF
:1039000008229043C861C6494031886A80229043AA
:10391000886222F045FF0821202022F002FF22F0D9
:1039200035FF012028603800FCF78FFDF8BDF8B5A1
:10393000FCF786FDB84D0090286801283AD123F0A5
:10394000F9F8002807D122F02BFF0821202022F0CF
:10395000DDFE22F01BFFB2494031886A802210430D
:103960008862AF48C1690826B143C161AB4F38686E
:1039700051050843C9108843386000F03EFF040039
:1039800000F03BFFA042FBD00A2022F05FFDA449DB
:10399000C8693043C86138680921490688433860DE
:1039A00022F0FEFE04211F2022F0BBFE22F0EEFEDC
:1039B000002028600098FCF748FDF8BD10B5040011
:1039C0000120FFF78CFB002C05D196490968CA0736
:1039D00011D0C9060FD506280DD00120C00300F074
:1039E00010FF0120C00750F05CEF8D49403108699D
:1039F0008A0D1043086110BD012010B5FFF76FFB61
:103A0000062803D000F0A4FE0028FBD110BD08203A
:103A100010B5FFF79CFA10BD082010B5FFF7D6F9D6
:103A200010BD38B5002000900120FFF758FB0400BE
:103A30000120FFF7D6FB05000420FFF788FAFFF707
:103A400076FF00F056FF202050F0EAEE00F025FF50
:103A5000684650F04EEF0121734AC906002800D095
:103A6000009891602A0021000120FFF719FB38BD62
:103A700010B5FCF7E5FC04006A480068400702D571
:103A80000020FFF7CEFF2000FCF7DFFC10BD012077
:103A900010B5FFF724FB04000120FFF7A2FB020092
:103AA00021000120FFF753FB002800D0012010BDAA
:103AB00008B5684650F020EF002803D0FFF7E7FF75
:103AC000002801D1002008BD012008BD554810B5CF
:103AD0000068400705D5FFF7EBFF002801D0012063
:103AE00010BD002010BD70B50120FFF7F8FA0400EA
:103AF0000120FFF776FB05000020FFF7F0FAA04257
:103B000004D02A0021000120FFF732FB70BD454898
:103B100010B50068000709D4FFF7D8FF002805D0CA
:103B2000FFF7B5FF002801D0FFF7DDFF10BD10B58E
:103B300000F0C5FE39484030816A3C4A114081623C
:103B40003B4908690322D202104308613448016AE4
:103B500049084900016231480168364A1140016054
:103B600010BD38B5002000900120FFF7B8FA04001E
:103B70000120FFF736FB0500202050F092EE00F008
:103B8000AFFE29490120C006C860684650F0B0EE7B
:103B9000002808D1FFF7CBFF50F0B2EE002808D084
:103BA000FFF788FE05E00098002800D0012000F013
:103BB00045F82A0021000120FFF790FA0420FFF7C2
:103BC00005F900F0C5FD00280ED013484068002814
:103BD0000AD019480068806B0001000C02D1012056
:103BE000FFF7ECFEFFF708FF38BD0E4810B5006880
:103BF00040070FD4FFF75CFF00280BD0FCF720FC38
:103C00000400FFF755FF002801D0FFF7AAFF2000AE
:103C1000FCF71BFC10BD0000F8640500402100808B
:103C200040200080A864050000280080FDFF7FCCB4
:103C300040220080F5FFFFBF4865050070B500F029
:103C40002CFE1A48816A1A4A11400722D2051143F4
:103C500081621648C0300169164A1140016122F0A4
:103C600069FF154D154E002802D1286A304328629D
:103C7000134C2078FF2809D122F092FD122022F067
:103C80003AFD04210840207022F080FD20780028B1
:103C900002D1286A30432862044940390868094A39
:103CA0001040094A8018086070BD00008021008023
:103CB000FDFFFFCFFEC7FFFF402000800100010095
:103CC00000650500F0FFFF9F0E000040FF484068C0
:103CD0007047FF49C869401CC8617047FC49886A41
:103CE000C96A704710B528F0B4FC002809A15A38F9
:103CF00001000000C43B00000004000021A408C231
:103D000009D0FCF7A7FBF64A117C002901D0491E17
:103D10001174FCF7A4FB10BD70B502201AF0FFFD72
:103D200007E0200036F0E9FFE27AA17A200019F0DE
:103D30008AFF0400F5D11AF0F2FD002801D036F018
:103D4000DCFF00F01BFFE84908690222904308618C
:103D5000E34C0025A561E5482574606128F09CFCD2
:103D6000656170BDF3B5040083B050F0D8ED0090EC
:103D7000DB48DB4D2038007E0E00603D0027002828
:103D800044D1D8492A69886AC96A6B69121A8B4179
:103D90001ED2009A28696969801AD54AB1418518EE
:103DA000E0697941010604D5A581E58124F0A6F9F1
:103DB00006E0800605D5A581E58124F09FF9400045
:103DC0002D1AE069012189020843E061606885805D
:103DD0000498C549800040394018006B3A2780029A
:103DE0000190BF48E75F4069009AFB17C117801830
:103DF0007141C01B019A99410023801A9941616168
:103E0000206160880121C9030843608005B0F0BDCE
:103E1000F8B504000D0050F082EDB34BAA00403B12
:103E2000D218136B6268002692781507AD0F022D29
:103E30000ED11709042F0BD1A94A9D02603A92694D
:103E40000B009788310038185941401BB1410FE0F1
:103E5000012D14D112090E2A11D19B020200180063
:103E60000D00101A2B00B341642219008018714113
:103E70006161206160880121C90308436080F8BD49
:103E8000F3B50C0083B00027C869C00403D5208DAA
:103E900081054D0E1BE0E06A0026350001900EE022
:103EA0000199A8004118042202A850F0D0EC6B46FA
:103EB000D87A6D1C0007000F86190E2D02D260788B
:103EC000B042EDD26B4618898005450E187AC007BE
:103ED00000D00127E069290002040398120C2CF09D
:103EE000ADF90600012F02D10E352D062D0E6068AA
:103EF00001230288E0690104090C280050F012ED4A
:103F00007C498019096B081860877FE7F8B50220A3
:103F10001AF005FD0500FF21774800222D3150F0F1
:103F20008EEC06007ED00221B0203173341830812F
:103F3000A078F32280088000104008300007000FAE
:103F40004030A070E0784008400008431040CF2186
:103F50000840BF210840E0703120000129180622E6
:103F60000D00A01D50F072EC2000062229000C303C
:103F700050F094EC200006222900123050F066EC3C
:103F800000211C202180351830817421280050F038
:103F900076EC534A2F00162060372C66603A78730F
:103FA0005088A87010004030017E002904D0C188DC
:103FB000A1808089A87002E09069C088A080A8686C
:103FC000FF21491C0843A86002201AF0A8FC706178
:103FD0004A48007E800607D4A878002804D0A86844
:103FE000012189070843A86007203873A8680521C4
:103FF00089020843A86020F026FA0124002804D092
:10400000012000F01EFB3748046030002CF0F2FD68
:1040100035480169022211430161314801001C3118
:10402000846100E004E04868401C48600120F8BD5D
:104030002B491C314869401C48610020F8BD2949C2
:1040400010B50A69002482421ED10020086124486C
:104050008069002803D1FFF759FF04000AE02848CF
:1040600001694069814205D0264807220068012184
:1040700000F0FAFF1A492039087E002804D0002CED
:1040800003D12D2014F0E8FC10BD0128FCD1022042
:10409000087610BD10B5134C6169814204D13020FF
:1040A00014F0DAFC0020606110BDF8B500250600B0
:1040B0000B48856150F032EC0A4CE162A06220F0BE
:1040C000C2F92168084303D0002000F0BAFA256045
:1040D000002E04D002481C300168491C016013E026
:1040E000187F050008650500C0A20080FFFFFF7F64
:1040F000A60E000040A60080480D00040F25CD67E5
:1041000001000000C03F000000040000727EDBAE32
:104110001067000400A00080A06C0500FF4D287E01
:10412000022811D1FE49C86802221043C8606069A4
:1041300001F09DF908220092EA88FA48FA4B002122
:1041400001F043F903202876F8BDF8B502201AF0F3
:10415000F0FB050050F0ECEBF34C07000E00143CB4
:10416000803508E0688BA26B8002E36BC117801872
:104170005941E163A063A26BE36BD21BB341F1D35E
:10418000E16BA06BF8BDFEB550F0D2EB0C000090D7
:10419000FCF76AF9E14DE449203501901439287C97
:1041A000096A084325D1DD480026017E0700403F0B
:1041B000002904D080887B6D3A6D31000AE028F038
:1041C00008FA002801D168690AE0B8697B6940886B
:1041D0003A6931008018009A5941801AA1416861FA
:1041E000002806DD2CF041FF002802D0287C401C6E
:1041F00028740198FCF73DF9FEBDF8B5012000F0E8
:10420000A1FC50F096EBC54AC74D403A5165143DAC
:104210001065286901F02BF9C04CC44F207E00289E
:1042200068D050F086EB2A6B6B6B801AC04A9941BC
:1042300000263300121A8B4101D2E6612FE0E069BB
:1042400001282CD120F044F9BA4E032816D820F0CA
:104250002AF9002812D1E088FF30F5300004000C64
:10426000B842E08000D9E780A088FF38F538000424
:10427000000CB042A0803DD2A6803BE0E0886438CC
:104280000004000CB042E08000D2E680A088AA4979
:1042900064300004000C8842A0802BD915E020F087
:1042A000DCF8002813D050F044EB07000E00FFF7B5
:1042B0004CFFC01BB1416A68A9685318834203D9F7
:1042C0004A08801AE08000E0E280A18012E0E869FC
:1042D000002801D0EE6109E0984982008A58002A3E
:1042E00004D1401C0728F8D3E78001E06089E08012
:1042F0002089A0808C4B08220092A288904800213F
:104300001B1F01F062F801202076A8698D4E02275C
:1043100001280DD1FCF7A8F80021A96171693022AC
:1043200091437161884A516AB9435162FCF7A1F81F
:104330007A49A088203148613069B8433061FFF77D
:1043400022FFF8BDF8B50400744E203670680028CE
:1043500036D0FCF789F8714D0700287E002C1ED05E
:1043600000282AD12868002827D07068002824D087
:1043700028F02FF9002820D120F063F8002803D17D
:1043800020F06BF8002818D06549C8680122520552
:104390009043C86050F0D4EAFFF72FFF0DE00028EB
:1043A0000BD0614C143C606901F061F8206901F0A8
:1043B0005EF8FFF7BBFC002028763800FCF759F8C0
:1043C000F8BD59491439CA6882420DD10020C8602D
:1043D000012088615B4841693022114341615A499B
:1043E000486A0222104348627047F8B55748446B48
:1043F000002550F09EEA00194B4C6941143CE163E2
:10440000A06328F0E6F8454E403E00280FD0B06883
:1044100000280CD0E06801F02AF808220092192246
:1044200023004B48520100210C3300F0CEFF3B4FDC
:10443000387E002810D003280FD120F00EF8002875
:1044400004D03749C86802229043C860606901F00F
:104450000EF8302014F00AFBF8BD0128FCD150F012
:1044600068EA326D736D821A9941B8880B00290091
:10447000801A9941374D00040014A842ECDA2069F3
:1044800000F0F5FF284B082200922D482A00002159
:104490001B1F00F09AFFF8BDF8B5204C224D2034C8
:1044A000143D2D287ED00CDC212809D00126B6022F
:1044B0002A285AD02B280DD02C2801D100F0D6F86C
:1044C000F8BD2E284BD02F284BD03028F8D1FFF73D
:1044D00094FEF8BD60680028FBD0FBF7C5FF040020
:1044E00028F077F8002817D00020FFF72BFF50F0B6
:1044F00028EA0B49C868012252051043C8601249D6
:104500008039886AFF2292041043886245DF81A8BF
:1045100001000000BC43000000040000708703B8E5
:10452000300000F003F9300000F0F3F820001DE047
:10453000F87E050000A70080593F00001C650500BB
:10454000D859000020A10700B80B00005046000019
:10455000F47802C0033F0000C0A20080C0A8008021
:1045600000A600807342000034080000FBF78BFFB8
:10457000F8BD012000E00020FFF7EEFEF8BD5D4F22
:10458000F888002804D138002430B861B88803E0E6
:1045900058491C31401EB961F8800120B8603000D4
:1045A00000F0B7F850F0CEE97961386105F0EDFF21
:1045B000286900F066FF00E025E008220092B86953
:1045C0004E4B02884C48002100F009FFA8694C4E70
:1045D00001280ED1FBF752FF0021A9617169302239
:1045E0009143716147494A6A02239A434A62FBF741
:1045F0004AFFB869408860613069022188433061B0
:10460000FFF7CBFDF8BDFF26F5366661FFF7C5FD68
:10461000286900F036FF082200923748374B3200F5
:10462000002100F0DCFEF8BD10B5324C6034A0680B
:1046300000280DD0E06800280AD028F02EF80128C4
:1046400006D160602E2014F01BFA2B2014F018FA0B
:1046500010BD2C2010B514F013FA2F2014F010FA0E
:10466000244900206031486010BD0322264912050C
:104670000028086901D0104300E0904308617047AA
:104680001C4870B560304068002831D0FBF7F6FE5A
:104690001A4C0600103C206900F0F3FE002525614D
:1046A00005F08BFFE06800F0ECFE1548E56041691D
:1046B0003022914341611348416A02229143416291
:1046C00010488038816AFF22920491438162440D30
:1046D000200000F02BF8200000F023F8054885604A
:1046E000FFF72EFB3000FBF7CEFE0120FFF734FE74
:1046F00070BD0000B87E0500033F0000186505008E
:10470000C0A20080C0A8008000A700800948C0693E
:10471000704708490A6902430A618A6902438A614B
:104720007047044A11698143116170470149C043D0
:10473000C8617047802100800849084840394268B4
:104740005204FCD44A68002AF9D1704710B523F00E
:104750006FF810BD10B522F0D7FF10BD40E8008003
:10476000DC48006800680004000C7047D948006805
:10477000416801221205114341607047D548006825
:10478000416801221205914341607047D148006899
:10479000806BC005C00F7047CE4800684168012299
:1047A0005204914341607047CA4800684168012241
:1047B0005204114341607047C6480068816B09018B
:1047C000090C01D000207047816B002904DA816B4D
:1047D0000906090FFBD100E0806B01207047BD483E
:1047E0000068816B0906090FFBD17047B949096858
:1047F0008A69120C120402438A617047B548006846
:10480000816BC907FCD041680122D203914341600A
:104810007047B04909680A6B086348680122D203EF
:10482000104348607047AB480068406A7047A94829
:104830000068C06A7047A7480068406B7047A54988
:104840000968CA698243CA617047A2490968CA698E
:104850000243CA6170479F4909680A6A02430A62B3
:1048600070479C4909680A6A82430A6270479948FE
:104870000068806B8007C00F704796480068806BA7
:104880000007C00F704793480068C0304168372266
:104890009143416070478F480068C03041680822EA
:1048A0009143416070478B480068C03041680822DE
:1048B00011434160704787480068C0300168012299
:1048C00011430160704783480068C030016849089F
:1048D0004900016070477F480068416801229204E6
:1048E000114341608168121191438160FF30401C87
:1048F0004168490849004160704776480068C11D19
:10490000F9314A6801231A434A6041689A04914385
:104910004160816812111143816070477F76719EFA
:1049200001000000B847000000040000235DD0D45F
:104930006D480068FF30401C41680222914341608D
:10494000704769480068FF30401C416802221143EB
:104950004160704764480068FF30401C01680122D4
:1049600011430160704760480068FF30401C0168D7
:1049700049084900016070475B4800688030416821
:1049800049084900416070475748006880304168D5
:10499000012211434160704770B5534D2868803043
:1049A00001680122114301600168504C490205D59C
:1049B0000168A14301600A204FF0A6EE286880300C
:1049C00001682143016070BD4748006801008031E3
:1049D0000A68520852000A60816BC900FCD4704713
:1049E0004148006880300068C007C00F70473E48EB
:1049F0000068803001683D4A9143016070473A4841
:104A000000688030C068704730B5374C21680A694B
:104A100001252D042A430A610A00803215691061BC
:104A2000506953619069F0209061886810221043AA
:104A3000886088682023984388602068416B426BB7
:104A40008A42FCD0FFF7DBFF0028F6D1206881689E
:104A5000194381604168012252031143416030BD16
:104A6000214800688030006970471F4800688168ED
:104A700020221143816070471B4800688168202212
:104A80009143816070471849096880310A681F2383
:104A9000DB05C0069A43000902430A600868012248
:104AA00012071043086070470F48006880680003D1
:104AB000C00F70470C48006881680122D20411437E
:104AC000816070470848006881680122D2049143E0
:104AD000816070470448006880300168FF22521CE2
:104AE0001143016070470000486505000000400068
:104AF0003F488068002800D00120704710B504F0BE
:104B00004CFA00280ED0FFF7F3FF00280AD03948EE
:104B1000C16802229143C16035484068C00FC00798
:104B200027F036FF10BD10B5314CA16881420ED17F
:104B3000FFF7E4FF60684004400CFFF7FCFD60688D
:104B40004004400CFFF7FCFD0020A060606010BD39
:104B500008B5274B5A6802435A60082200920A009F
:104B600025480021083300F044FC08BD70B505005D
:104B700000240420FFF7E4FD1E488030C06A400096
:104B800013D422F00AF800280FD00420FFF7CBFD41
:104B9000002D01D10124E407200004210843144919
:104BA0000968FFF7D5FF002070BD1249C8680222CE
:104BB0009043C860012070BD0E48C16802221143B5
:104BC000C16070470B48C06802210840704704204C
:104BD00010B5FFF7B0FD0420FFF7B2FD044CA0684C
:104BE000002804D000F057FC0020A060606010BDD9
:104BF0004C65050000A70080AF490000CA490822A3
:104C00000028C86801D0104300E09043C860704796
:104C1000C64800214160FF2101707047F0B50325AF
:104C20002D03C148C24CC030C20D9302870C00292D
:104C3000BD4E016A0AD011430162016A99430162C3
:104C4000606B284360633068384309E09143016238
:104C5000016A19430162606BA84360633068B8431E
:104C60003060F0BD38B50500002468464FF010EE06
:104C7000002802D1002D1AD10BE0002D0BD16B467C
:104C80005878C10713D0400611D598780007000F57
:104C90000BE001240BE0012D09D16B465878810708
:104CA00005D5C00903D0987800090128F1D020006B
:104CB00038BD73B56B4605005C79600708D59B4E1F
:104CC0007068002804D19B482CF0F2FF012070602E
:104CD0002800FFF7C7FF0106090E2800FFF79EFF17
:104CE000600703D46B461879000900D00120FFF754
:104CF00085FF7CBD33B56B460028997902D1080742
:104D0000000F02E0012813D108098B4A8649D443D9
:104D1000803100280DD0894B894D01280DD00928FC
:104D200010D00F2804D1C817C860086102D4388396
:104D300001000000B44B000000040000D732A56061
:104D4000C86108623CBDCA600A61CC6102E0CB6008
:104D50000A61CD610C623CBDCB607F480861CD61CA
:104D60007E48EEE7F0B50028047A45780679477961
:104D70002ED001290FD1059901290CD1012A09D181
:104D8000002C00D140246540D90700D06640990727
:104D900000D567402C00724B1968914200D01A6010
:104DA00001782A0609040A4321020A43634922437F
:104DB000C0314A628279C37812041B021A4332431B
:104DC0008A62C279807812043B021A430243CA62A3
:104DD000F0BDF0B50026050087B06B46187D3700A2
:104DE00034001E75002D06960ED145205875987D0D
:104DF0000120987518720221587299720421D97293
:104E000018735873997310E047206B465875987D56
:104E100090209875092018720A22587211219A72EE
:104E2000D97218735A73997312216B46D973187417
:104E300005992800FFF747FF05992800FFF764FF51
:104E4000069823000207120F00923A00310002A8D0
:104E5000FFF788FF012007B0F0BDFEB5070008F09E
:104E60002DFCFFF709FF002825D1344D6C46E435B1
:104E700007CD6B46324E07C40C3D187999780C3C2F
:104E8000002F0BD0884216D05A7A1B7A9A4212D041
:104E90007170B3706B4698701A720AE088420AD13A
:104EA0006B46587A197A884205D170789870B07834
:104EB000187207CC07C5FEBDF0B5002507002048D5
:104EC0002E0001782C00B94285B035D0077004A8B7
:104ED0004FF0E8EC002804D13800FFF77AFF05B066
:104EE000F0BD6B46187C0007000F012805D838007C
:104EF00001A94FF0E0EC002801D10020EFE7049970
:104F00003800FFF7E0FE04993800FFF7FDFE6B461E
:104F1000587CC10601D4800600D501256B46187C5B
:104F200023000207120F00923200290001A8FFF7A8
:104F300019FF0120FFF791FF0120D0E700A70080B3
:104F4000586505000021008000A0008011DD55DDBE
:104F50001FDF5FDFEF2FAF2FF1FDF5FDFEF2FAF25D
:104F60007C0C000438B500240D4D01E08047641C22
:104F7000A00028580028F9D13BF024FE4FF002EDA4
:104F800008480A4902680092074A0948094B4FF04D
:104F9000FEEC09480168002901D00020884738BD8F
:104FA00008C102C0B46A050018520004180D0004BC
:104FB0000C0D0004009002C060650500FEB50D00F8
:104FC0001600089F0A9A0999002800D1FEE7046894
:104FD000002C00D1FEE7029201913200290020004E
:104FE000009722F089FAFEBD10B54FF0D4EC000610
:104FF000000E10BD10B54FF0D2EC0006000E10BD33
:10500000002810B501D04FF0CEEC10BD38B514001B
:105010006A464FF0CCEC00982070002038BD10B5E7
:1050200004004FF0C8EC2060002010BD10B54FF018
:10503000C6EC10BD7CB50D001600079A0699002835
:1050400000D1FEE70468002C00D1FEE70192009138
:1050500032002900200022F02DFB002800D16563DA
:105060007CBD10B5416B22F03CFB10BD7CB50C0043
:105070001500069A002800D1FEE70068002800D13C
:10508000FEE70021019200912A00210022F062FA3D
:105090007CBD10B522F07DFA10BD10B522F084FA67
:1050A00010BD002810B500D1FEE70068002800D12F
:1050B000FEE722F082FA10BD10B522F088FA10BD8A
:1050C00038B51400049A0092220022F0A5FA38BDE7
:1050D000002810B500D1FEE70068002800D1FEE7E7
:1050E00022F0CEFA10BD10B522F0D4FA112800D16A
:1050F000122010BD10B522F0D5FA10BD01C08FE20C
:105100001CFF2FE170B5242149484FF0E0EBFBF77D
:10511000C9F90121464BC90700200A781A54491CD5
:10512000401C0A28F9DB434900200A781C18491C56
:10513000401C0A28A272F8DB3E482030E00381E1DF
:1051400001000000B04F00000004000084E8760C6D
:10515000017A1975017C5975017D9975017ED975A2
:10516000007F394A18766032110000200C781D1833
:10517000491C401C0B282C76F8DB0020D178EE2946
:10518000FCD1017891703049401C6431CB1D04780A
:105190000C70401C491C9942F9D3032149048842F0
:1051A00003D101208006AA210CE02849884202D1BF
:1051B0008005BB2106E02649884202D10020CC218F
:1051C00000E0FF21D170D9E71F486030C078EE2899
:1051D00000D1A1E7704770B5FDF71FFE1D48002202
:1051E00000680D214FF028EB1B4D6C6804E06068EF
:1051F000002800D080472468002CF8D1FFF7E4FF96
:105200002878401C0006000E2870FBF7E3F8FDF735
:10521000FCFDEAE7114810B54FF0CAEB10BD10B520
:105220000400FBF749F90C4B59680A0000E00968D3
:10523000002902D0A142FAD101E022605C60FBF7B4
:1052400040F910BDB08105000001008000A70004F6
:10525000003003C0286A050064650500507F050022
:1052600070B580204FF0F8EA10498D69104900268A
:105270004A680C68954200D800E0641C4FF0ECEAE4
:105280006D1C684231008019614170BD0848016899
:10529000491C01600021C94341607047034880698F
:1052A00003494A68904200D8486070470030008047
:1052B0006C650500EA48006AEA494968081A7047BF
:1052C000E7480169820C91430161E6494968C16080
:1052D00001690B221203114301617047E048016923
:1052E000820D91430161E04A4021D1600421C9430C
:1052F0004162704770B50400FFF7E2FFC82C00D28E
:10530000C824D8494868844200D30400D448042201
:10531000D2434262D44A936840252B439360846011
:10532000026905235B021A430261C86880472000B6
:1053300070BD01684A69026000200861C9480068C0
:1053400082684A6181607047002307E082688A4270
:1053500002D3521A826000E0836040690028F5D1D0
:10536000704770B5040000200BE04E680D690B68B3
:105370002000FFF7DEFF002B02D031002800984705
:1053800001202168002902D08A68002AEDD070BD72
:1053900010B5026802E0100052691430002A03D0F0
:1053A0008B689468A342F6D84A61016010BD10B5BD
:1053B000AC4C20680069002803D02069401C2061A3
:1053C00010BDFFF78BFFFFF775FF0300FFF778FFB6
:1053D0002168CA689A4201D960681B184868190098
:1053E000FFF7B2FF2068001DFFF7BBFF2068416890
:1053F00000290FD0FFF75EFF21684A680100100006
:10540000FFF7A2FF206840688068FFF773FF2168FC
:10541000C86010BD0021C16010BDFFB581B000247F
:105420001D00FFF75BFF80204FF016EA8D4E0090C5
:10543000306800278168002921D00C00496981600B
:105440000168491C016001D10121016001982060BF
:105450000298606030680068206103986761A0600E
:105460000A982073FFF726FF31684A680100100090
:10547000FFF76AFF30682100001DFFF789FF3068E1
:105480004168002907D00069002804D18868FFF727
:1054900031FF3168C860002C07D02069002804D093
:1054A000002D00D02860012403E0002D00D02F60E3
:1054B000002400984FF0D0E9200005B0F0BDF8B509
:1054C0000025070067482E000468241D002F20D007
:1054D00080204FF0C2E9030007E00169B94202D120
:1054E00001252E0001E0040014342068002801D0BA
:1054F000002DF2D0002E02D02000FFF71AFF5948ED
:1055000000684068002801D1FFF7E8FE18004FF05E
:10551000A4E93000F8BD70B580204FF09EE9514CF1
:105520000500216801200861486800280FD0FFF7B6
:10553000D5FE4FF026EA2268D1619061FFF7BAFEEE
:10554000010020684068FFF7FFFEFFF79702F7AB06
:1055500001000000AC530000000400003B2D53BFCD
:10556000B9FE28004FF082E970BD70B580204FF081
:105570007EE9414D060028680169002916D0002106
:1055800001614068002811D04FF004EA2C68A2693C
:10559000E369801A994101006068FFF7DFFE28681F
:1055A00040688068FFF7B0FE2968C86030004FF09F
:1055B0005EE970BDF7B582B000250E00FFF7B5FFBC
:1055C00080204FF054E901902B4800270068446880
:1055D0000CE0002E02D0207B304206D0A5684FF0B0
:1055E000DAE9029A4019794103C26469002C01D0BA
:1055F000002DEED001984FF03AE90498002801D12F
:10560000FFF7B3FF002D06D0FFF75EFE854201D302
:105610002D1A00E00125280059E7F8B506000027FB
:105620003D0080204FF022E90090134801684C684B
:1056300017E0207B400711D5A068B0420ED80020AB
:10564000002DA06006D0606928600B4800684168A2
:1056500061614460FFF789FF012702E0250064696A
:105660001435002C01D0002FE3D000984FF0FEE855
:105670003800F8BD00300080746505000028008007
:1056800030B50022FD4C256807E018235343C35C66
:10569000002B0BD1521C1206120EAA42F5D36268DF
:1056A000002008E00301CB5C002B01D0012030BDBD
:1056B000401C0006000E9042F4D3002030BD182399
:1056C000584340180169491C01617047F7B515003E
:1056D0000600EA4F002417E018206043295C0029E7
:1056E0000FD041194878B0420BD10198091D06220C
:1056F0004EF0D5FB002804D11821614349190861F7
:10570000FEBD641C2406240E38688442E4D3FEBD2A
:10571000F7B515000E00D94F002411E02001295CD7
:1057200001290AD140194178B14206D10099C01C23
:1057300006224EF0B4FB002805D0641C2406240E7B
:1057400078688442EAD32000FEBD0300080010B54B
:1057500014001900FFF7DCFFC8494968884203D2EA
:10576000002100010019C16010BDF7B51500070048
:10577000C24E002412E018206043295C01290AD19E
:1057800041194878B84206D10198091D06224EF009
:1057900086FB002805D0641C2406240E3068844251
:1057A000E9D33068844202D10020C043FEBD1820F6
:1057B000604340190069FEBD0300080010B51400E5
:1057C0001900FFF7A5FFAD494968884203D20001DF
:1057D0000019C06810BD0020C04310BDF7B515000A
:1057E0000600A648002440681CE02101695C0029ED
:1057F00015D1301D4FF07AE827017C1960700198AF
:105800003100A070E01C062214314FF05CE801204A
:10581000E8550020E06001200003608104E0641C82
:105820002406240E8442E0D3944880688047FEBD5D
:105830001823594310B58C18904A61691269904732
:10584000002802D0E17823F036FC10BDFFB583B00C
:105850000F008A4D0C9EE968039888470D3001219E
:10586000814000242800019100683BE01821614339
:10587000715C002933D1381D4FF038E8182161439D
:1058800002918D19687005983900A870281D0622AC
:1058900014314FF018E80299012070540698E8700E
:1058A000380008304FF022E8002802D10920000219
:1058B00002E0C3001818000268616969019881421A
:1058C00001D9019868610020286128730120000334
:1058D0006881039832002100FFF7AAFF04E0641CEE
:1058E0002406240E8442C1D364488068804707B0F0
:1058F000F0BDFFB581B01E0000273C0016E020017E
:10590000315C00290FD085190298E91C06224EF05F
:10591000C6FA002807D168780199884203D1039814
:10592000A97801270170641C2406240E534840689E
:105930008442E4D3380005B0F0BDF7B51600002767
:105940003C0014E018206043315C00290CD085191C
:105950000198291D06224EF0A2FA0028C60106BDB4
:1059600001000000A85700000004000068F780D381
:1059700004D169780098814200D10127641C240673
:10598000240E434800688442E6D33800FEBDFFB5CC
:1059900081B01E0000273C0016E018206043315CF7
:1059A00000290ED085190298291D06224EF081FA91
:1059B000002806D169780198814202D10398012715
:1059C0000470641C2406240E314800688442E4D329
:1059D0003800BAE7F8B50D0007002D4E00240CE0A2
:1059E00018206043285C002804D02A0021003800D9
:1059F000FFF728FF641C2406240E30688442EFD38E
:105A0000F8BD70B500248300CC50214D210008E082
:105A10004B009E187678864200D1D454491C090662
:105A2000090E2B689942F3D370BD80000858704767
:105A300070B50021164D0C0007E04A004B1D1618EA
:105A4000491C09067370090E84542A689142F4D3E4
:105A500070BD0F4902000968002004E04300D35CD8
:105A6000002B02D0401C8842F8D3704730B5002389
:105A7000074C24680FE05D00455D002D0AD101252B
:105A80005C00055520180B6040781070002030BD78
:105A9000906505005B1CA342EDD30120F7E7234B83
:105AA00010B51B68040000209C4208D218236343F1
:105AB000D45C002C03D09818C0780870012010BD69
:105AC000FFB581B080200A9E4EF0DAEE00901748B4
:105AD000002420E018276743F05D002818D0BD1986
:105AE00068780299884213D10199281D06224EF048
:105AF000E0F900280CD11820604303998019C07880
:105B000008700499A87808700020F055286106E014
:105B1000641C2406240E054800688442DAD30098E9
:105B20004EF0AEEE0148806880470EE790650500B4
:105B3000FF480188828891421FD101898289914260
:105B40001BD1018A828A914217D1018B808B8142BD
:105B500013D1F74820300188828891420DD1018904
:105B60008289914209D1018A828A914205D1018BB1
:105B7000808B814201D1012070470020704730B5F1
:105B80005B070C785B0FE408E4001C439F23039D34
:105B90001C400C7054040AD5920408D5C269FF2435
:105BA000641C2243C2610878184020300870002D20
:105BB00003D0087880221043087030BD0122120300
:105BC00002430F200002824308021043704710B5C1
:105BD000038D9B055B0E032B11D900290CD0C169E5
:105BE00020248023002A09D0CA0502D421439943E6
:105BF00001E01943A143C161012010BDF9E7002074
:105C000010BDFFB581B00E001F0001890A9D0C1860
:105C1000242120004EF05CEEA421002F02D00120B0
:105C2000000300E000200843608003208003054358
:105C3000280A257160712000062231000C304EF0D8
:105C40004CEE03990622A01D4EF046EE200005B052
:105C5000F0BD70B5040016001D000622801D4EF038
:105C60003CEE2000062231000C304EF036EE2000D3
:105C70000622290012304EF030EE70BDFFB581B023
:105C800004000E0017000B9D20214EF022EEA0789C
:105C9000F3210840B10008430007000F3901084311
:105CA000A0700A9A04992B002000FFF7D2FFCEE7DC
:105CB00003000820002905D0002B01D0C82004E0F3
:105CC000482002E0002B00D08820002A02D00121C9
:105CD000490308437047F8B500240028079E069D35
:105CE0000AD00407A40F04D09249586989688847EC
:105CF00019E0800717D5012408880C38088040383F
:105D00000004000C9880CF787F0710D40F7E3F07E7
:105D10000DD0002C09D00888683A8118082230007C
:105D20004EF0DAED03E00020F8BD0838988001203D
:105D30002C60F8BD7CB50E000588069C083D0580EA
:105D400095881900083D9580320024316B4626F075
:105D5000F6FB00982168884205D101986168884265
:105D600001D101207CBD00207CBD0280277ED5773B
:105D700001000000A45B0000000400009C98F5678F
:105D80000B607047F0B5012A069D059C13D0022ACE
:105D900015D0042A2DD14A780E78120292194E7924
:105DA0000F793602F619CF7812043602120CF61962
:105DB0008978360212E00A788E78120202E04A7878
:105DC0000E7812029219CE798F793602F6194F7930
:105DD000120436020979120CF61936027118266877
:105DE0008E4202D11F88974203D2771C03D08E4285
:105DF00001D90120F0BD002801D01A8021602A803D
:105E0000079801600020F0BD002804D0D0788207F8
:105E100001D4C00701D1002088807047002810B548
:105E20001CD0D078840719D4C00717D1907C1C7877
:105E3000A04213D1D07C5C78A0420FD1107D9C7819
:105E4000A0420BD1507DDC78A04207D1907D1C7917
:105E5000A04203D1D07D5A79904201D000208880A1
:105E600010BD70B50D001400190000280BD0E278A9
:105E7000900708D5D00706D1200006220C304EF03E
:105E800022F8002801D00020A88070BD817809097F
:105E9000042901D00C2903D1C178BF221140C1705F
:105EA000C0784006C017401C704710B504000800B9
:105EB0001100C278D30708D1920706D50622123006
:105EC0004EF001F8002800D1A08010BDF0B50026EA
:105ED0000C8B178825090C7E2407240FAF4214D1A0
:105EE000C9780A0706D5490704D4002C00D003E07E
:105EF0008680F0BD002C03D01988491CA142F7D13F
:105F000005998C42F4D21C80F0BD002CF0D1158094
:105F1000F9E7F8B505002030007D0E00C006170037
:105F2000800F022801D0032814D128000124183042
:105F30004EF0F0EC000600D50524287DC10906D0FE
:105F4000022103E040A00080A86505000C43400644
:105F5000400E01E0E87E002434703870F8BDFFB5D3
:105F60008BB01C00050003261498002826D00822B8
:105F7000210001A84EF0BAECA049062201A84DF07C
:105F8000A2FF002818D09D490622891F01A84DF0C4
:105F90009AFF002812D1994901AF02220A39B81D8F
:105FA0004DF091FF002809D0944902220839B81D0C
:105FB0004DF089FF002801D0083402260D992022D7
:105FC00003A84EF094EC0E3C022E03D1A8880838AA
:105FD000A88006E0A988080A090208432073000A7D
:105FE00060736B46D87B864FC0076F4403D106228F
:105FF00004A9891C01E00622390020004EF076EC4D
:106000006B46D87B810702D4062206A907E0C007A9
:1060100003D0062209A9891C01E006223900A01D2F
:106020004EF064ECA8880E30A8800C980460300014
:106030000FB0F0BD70B51E000378049C1370437858
:10604000537083789370C078800903012070181A08
:106050004018407B002802D01025012001E00825CF
:10606000002030700020ED1E08E0267833019B1BD5
:106070005B181B1816189B7B401CF370A842F4D3C6
:1060800070BD002810B50ED0C87840070BD55D4C08
:1060900002E001204EF0AEECE0684EF0BCECE168AE
:1060A00049888842F5D010BDC178490702D4007EE6
:1060B000000700D00120704780780107890F02296E
:1060C00006D10009042801D00C2801D10120704715
:1060D000002070474C4B02000800596991435961F8
:1060E00000E0401E9969114201D00028F9D17047A3
:1060F000F7B584B00024250043480194434E41691C
:10610000049A43061A43114341613F4A80321169A0
:1061100007231B04194311613B4BC0331968082244
:10612000914319603A4B1968914319608069029054
:10613000FFF7B4F8009033480F002AE0FFF7AEF8FD
:10614000009A0023801A2F4AB94151611061314AE7
:10615000121A8B4109D22B480168491C01602A4957
:106160004869049A9043486116E027486D1C80698D
:106170000290294800697F2149050840B54BAEFBD4
:1061800001000000A05F000000040000CF42260BC9
:1061900003D001214905411A03D1864201D1641C73
:1061A00000E00024060006988442D1D31A4E3068DD
:1061B000002809DD06988442706801D3401C02E083
:1061C0000121090440187060FFF772F8009A801AE4
:1061D000B9417161306102990498884301D001206E
:1061E0000190104A11680820014311600B49C03129
:1061F0000A6802430A60094A8032106907210904CB
:106200008843106105980560019807B0F0BD000053
:106210000E5B05001E000000A865050040A200807E
:106220004523010000A70080A086010080A800800F
:10623000FE48FF4A016904E0002000E0401C88425B
:10624000FCD3506BC007F7D1704730B5CA780B78D4
:10625000120613438A784C78120424022243134313
:10626000F44A1360CC790B79240623438C794D7959
:1062700024042D022C4323435360CC7A0B7A24064A
:1062800023438C7A4D7A24042D022C4323439360BC
:10629000CC7B0B7B240623438C7B497B24040902A3
:1062A0000C432343D360E24902684A604068886037
:1062B0000020086030BDE048C269032109028A431A
:1062C000C261C2690A43C261D8488068004730B5DC
:1062D0000100C4781231E207002A01D1821D00E0DA
:1062E0000A000300A5070C33002D01DB190003E0B1
:1062F000E40701D001001A31C8780C780006044385
:1063000088784D7800042D0228430443C948C462AC
:106310004C79097924020C430463D478117824065B
:1063200021439478557824042D022C432143416263
:1063300051791279090211438162DA7819781206CB
:1063400011439A785C7812042402224311430161BC
:1063500059791A7909021143416130BDFFB581B005
:1063600004001600B1480C9F00680B9D8047009008
:1063700039002800FFF769FFFFF75AFFAC4D0020F6
:106380002860E86AA86A286BAA4F20002830B86302
:106390002088F863A7490298403108602000FFF781
:1063A00096FF0A987863E078400701D408202860B7
:1063B000049930040843F861300C38622020B86139
:1063C000207E0007286801D09C4900E09C490843D2
:1063D0002860964DE8688047FFF72AFFE07840077D
:1063E00001D4FFF768FF69680098884705B0F0BDE1
:1063F000FFB581B006000D008C480A9F006800249C
:10640000804700900B993800FFF71FFFFFF710FF40
:10641000874800210160C16A816A006B854FBD63B6
:106420000398F8638348403005603000FFF74FFF62
:1064300004987863F078400700D40824307E814DBA
:10644000000711D00C980068A8610D980068E861F9
:106450000E98006828620F980068686210980068BB
:10646000A8627648001F01E07548001F704F044382
:106470003C606E4CE0688047FFF7DAFE7F6B0E20D1
:106480000740F07840070ED529690C9801606969CA
:106490000D980160E96A0E980160286B0F990860F9
:1064A000696B10980160FFF706FF616800988847E4
:1064B00038009BE7FFB581B005001C005B480A9ED1
:1064C000006880470090FFF7B3FE5948C16A002773
:1064D0000760E278217812061143A27863781204EB
:1064E0001B021A4311438161E2792179120611439B
:1064F000A279637912041B021A431143C161012E70
:1065000015D1E27A217A12061143A27A637A120433
:106510001B021A4311430162E27B217B12061143E5
:10652000A27B637B12041B021A4311434162217850
:10653000297061786970A178A9700B998901E97057
:106540003C498F61029A8A633A4A2D1D4032156098
:10655000039ACA63B101491C042211430160334C00
:10656000E0688047FFF764FEFFF7A5FE61680098CA
:1065700088473BE7FFB581B01C002C4E0A9F30686E
:1065800080470090FFF754FE294DE86AFD25DA6345
:10659000010000009C63000000040000E7D3A3B6E4
:1065A00000202860E178207809060843A178627805
:1065B0000904120211430843A861E1792079090610
:1065C0000843A17962790904120211430843E86182
:1065D000012F15D1E17A207A09060843A17A627A5F
:1065E00009041202114308432862E17B207B09065B
:1065F0000843A17B627B09041202114308436862CD
:10660000114802998163104A01994032116003993F
:10661000C1630B99B801C978401C490701D408210E
:1066200008432860F0688047FFF70CFE686B40075E
:10663000C417641CFFF749FE7168009888470DE095
:10664000C065050000B1009000B0009040200080BF
:10665000470002004700030080B000902000CFE612
:10666000FFB581B000250F00002827D041780378BE
:106670000E021E43082A01D0052A03D104002C343F
:106680000C2519E0042A19D10400203414E02078E4
:10669000B8420CD10498002806D00A9A0499A01C8C
:1066A0004DF025FC002802D1200005B0F0BD607837
:1066B000AD1C4519A41C0419B542E8D30020F4E729
:1066C000FFB5002085B004001D000E9E04900698C2
:1066D000007803900698477880204EF0F0E802900A
:1066E0000398DD2803D1069CA41C06200490049A7C
:1066F00000920399059823000822FFF7B1FF0400D8
:106700000021002808D1079C002F297007D102988A
:106710004EF0D4E809B0F0BD6078801C287007986E
:106720002A78001B801A0206FA4B120E002F06D19F
:10673000317028785B6801192000984715E0BF1C6C
:106740003806000E30702978884203D909199B68F1
:10675000001904E0884203D05B68091900199847C2
:106760003278069920004EF0D6E8059841780278F4
:10677000080229781043401A3178401805990870AA
:10678000000A4870C3E7002810B509D02A24520037
:106790000A430470012499000A4344708270032064
:1067A00010BD0322027001224270817003207047E5
:1067B00010B50C000021217001002022A01C4EF019
:1067C00042E96070801C0006000E10BDF8B50D0097
:1067D0000600170000240E214EF038E9082803D9DE
:1067E00008380406240E0820002F04D101210200DD
:1067F0002970310005E0002C0BD0322129703118AE
:106800002200A81C4EF01EE96870801C0006000ED5
:10681000F8BD0020F8BDF7B582B015000C00029855
:10682000077846780420042E00D23000019017E04B
:106830002078DD280FD1DD2F0DD1617801988142BC
:1068400000D2080002000298A11C801C4DF04FFBF2
:10685000002807DB01E0B84204D26078A41C0419C8
:10686000AC42E5D3AC4208D2A919891C03E02878D0
:106870006D1E0870491EA542F9D20299B21C200073
:106880004EF048E8B01C10E7FFB581B000260C9F21
:106890000B9C002F0DD002990498081A9D49052AD7
:1068A00003D0082A05D1098800E049880D1A002D77
:1068B00022DC0020F9E66178BF1EB9421EDC207898
:1068C000019A904214D130281AD0DD2810D1891CA9
:1068D000A94213DC02980A998219049841182000F1
:1068E000FFF799FF0004000C31180E04360C2D1A26
:1068F0006078A41C3F1A0419022FDCD23000D4E6C1
:106900006678B61CAE4205DC0298320021004EF0DB
:1069100002E8F3E70026F1E770B504000800110073
:106920001D00002C01D1002070BD62782378120276
:106930001A43A318203318705B1C1D705B1C0220C7
:10694000002906D02A0018004DF0E4EFAD1C2806FF
:10695000000E617822780902114309182170090A92
:10696000617070BDFEB50400401820300190D01851
:106970001500002627002037009012E0607821786B
:1069800000020843C21901992800FFF744FF61780B
:1069900022780902114309182170090AE682065279
:1069A000010000009867000000040000B40970DADC
:1069B00036182D18617000988542E9D33000FEBD6D
:1069C000F7B50600057847780C0010E02078A8425B
:1069D0000AD16278BA4207D1DD2D0BD1B11CA01CBF
:1069E0004DF08FFA002805D06078A41C0419029895
:1069F0008442EBD3029884420CD20298BF1CC51B80
:106A00002A1BE11920004DF090EF390028004DF0CD
:106A100088EF00E000273800FEBDFEB505004018F5
:106A200020300190D018140000262F00203700904D
:106A300014E06878297800020843C21901992000FF
:106A4000FFF7BEFF69782A7809021143091A2970F5
:106A5000090A361869706078A41C041900988442E9
:106A6000E7D33000FEBD002801D00021018070472F
:106A7000F8B5002506000F002C000DE0305D010682
:106A800007D54006400E04D04DF0EEEF01218140C5
:106A90000D43641C2406240EBC42EFD32800F8BD2D
:106AA000427901008B7890039B0707D5497AD2057C
:106AB0001043C90702D00121890508437047F8B582
:106AC000002406000F0025000BE0305D4006400E5C
:106AD00004D04DF0CAEF012181400D43641C24060F
:106AE000240EBC42F1D32800F8BDF8B515001F00F4
:106AF000069E0024002802D0FFF7E1FF0400002DCD
:106B000004D039002800FFF7DAFF0443002E03D039
:106B10003000FFF7C5FF04432000F8BD0200401A13
:106B20008A4200D2401E7047D4650500FEB51400AD
:106B3000060008001900099B089A002E01D0002BBE
:106B400001D10020FEBD1D890091ED1801000192C8
:106B5000FF4A2F002300280022F07DFF340020345C
:106B6000A078617800023D00084320352872000AB1
:106B70006872607DA872A07DE8720C352900300033
:106B8000FFF720FE44193000002221003730FFF7C4
:106B900027FE0019FEBD10B52C22525C04002C31DA
:106BA000032A03D14DF0C0EEE41C05E0022A03D114
:106BB00007224DF0BAEEE41D200010BD70B50300B1
:106BC0000C001500002816D018002030017AC27978
:106BD0000902114303D16421C1710021017218001F
:106BE0004B300E2106004DF03CEF020028703100C2
:106BF00020004DF09AEE70BD70B50500080016003B
:106C00001C00002D08D006214DF08AEE202229001C
:106C100030004DF022EF207070BD70B505000C0003
:106C2000002853D0002C51D05A2128004DF078EE86
:106C300020002030017A0200C079090201432800B7
:106C400020304170090A8170022101702100403119
:106C50004B7A4375897A8175517AC1702000603012
:106C600006004DF076EE290054314DF018EA7079A7
:106C7000327901022800114350300172090A417231
:106C800020000E214B304DF0ECEE0300002208E016
:106C9000A0184030A9182031521CC07A1206120EDA
:106CA000C8759A42F4D32100280007223A312C30CB
:106CB0004DF03AEE2022A11D28004DF036EE2100C5
:106CC00028000822413124304DF02EEE70BD0068BE
:106CD000406820300172090A417224E738B50C007F
:106CE0000068002240680092082206210023FFF776
:106CF000C1FC002802D0210A8470C17038BDF0B5F3
:106D0000002877D0002A75D0D7780478CF25BE0721
:106D10002C40B60F012E04D00326FF43BF0700D03E
:106D2000002636013443A606B60F047062D0A707CA
:106D30003026002F1FD1012905D0022903D00329B5
:106D400001D0042902D12C40103404700A2905D046
:106D50000B2903D00C2901D00D2902D1047834432A
:106D60000470002B3ED1082901D009293AD10178BD
:106D70003143017036E0A3079B0F012B32D17429F8
:106D800039D011DC8B079B0F2CD18B10093B4DF0B8
:106D900004EE143235323532353235292929292984
:106DA00029292932353235298C2919D00ED5F249B5
:106DB00001000000946B0000000400004066056EB6
:106DC0000CDC802924D004DC782921D07C2913D143
:106DD0001BE0842919D088290ED119E09D2914D0EF
:106DE00004DC952911D0992906D111E0A1290FD0F1
:106DF000A52901D12C400470D17800788908890038
:106E00008006800F0143D170F0BD2C401034F2E7B2
:106E10003443F0E710B5016A002910D08A7894074E
:106E2000E40F9C420BD05208DB075200DB0F1A43E1
:106E30008A70FD210A40006A59000A43827010BD21
:106E400070B5040012304DF08EED2578002805DC79
:106E500020002A304DF086ED002802DD2020054379
:106E600001E0DF200540A01C25704DF07CED0028DE
:106E70000BDC20000A304DF076ED002805DC200008
:106E800022304DF070ED002803DD207810210843FA
:106E900002E02078EF210840207070BDF0B50400BA
:106EA000323085B00D0003904DF05CED002814DD0C
:106EB0002000363006004DF056ED01002800FFF7A7
:106EC00037FE070003984DF04EED0399C01B4DF0BF
:106ED000F0E8310028004DF0ECE820003A30029054
:106EE0004DF040ED002814DD20003E3006004DF04E
:106EF0003AED01002800FFF71BFE070002984DF055
:106F000032ED0299C01B4DF0D4E8310028004DF05D
:106F1000D0E82000423001904DF024ED002814DD2F
:106F20002000463006004DF01EED01002800FFF75E
:106F3000FFFD070001984DF016ED0199C01B4DF0C3
:106F4000B8E8310028004DF0B4E820004A30009045
:106F50004DF008ED002817DD20004E3006004DF002
:106F600002ED01E0E865050001002800FFF7E0FD03
:106F7000070000984DF0F6EC0099C01B4DF098E822
:106F8000310028004DF094E820001A3006004DF042
:106F9000EAEC002814DD20001E3004004DF0E2EC85
:106FA00001002800FFF7C4FD070030004DF0DAECC7
:106FB000C01B31004DF07CE8210028004DF078E83E
:106FC00075E4FEB504000D00801C4DF0CCEC0028EB
:106FD00012DDA01D4DF0C6EC01002800FFF7A8FD52
:106FE0000600A01C4DF0BEEC801BA11C4DF060E81B
:106FF000A11D28004DF05CE820000A3002904DF001
:10700000B2EC002814DD20000E3006004DF0AAEC92
:1070100001002800FFF78CFD070002984DF0A2EC5C
:107020000299C01B4DF044E8310028004DF040E8C3
:107030002000123001904DF096EC002814DD200065
:10704000163006004DF08EEC01002800FFF770FDB1
:10705000070001984DF086EC0199C01B4DF028E81F
:10706000310028004DF024E82000223000904DF03F
:107070007AEC002814DD2000263006004DF072EC7A
:1070800001002800FFF754FD070000984DF06AEC5E
:107090000099C01B4DF00CE8310028004DF008E8C5
:1070A00020002A3006004DF05EEC002814DD2000A0
:1070B0002E3004004DF056EC01002800FFF738FD9B
:1070C000070030004DF04EECC01B31004CF0F0EFEB
:1070D000210028004CF0ECEFFEBD010010B50400CB
:1070E000223100204CF0E4EF21002A3100204CF046
:1070F000E0EFA11C00204CF0DCEF21000A31002061
:107100004CF0D6EF2100123100204CF0D2EF2100DC
:107110001A3100204CF0CCEF2078CF2108402070AD
:1071200010BDF8B504000E0015000F2B09D8210082
:10713000079822314CF0BCEF2100069826314CF024
:10714000B8EF002E0CD03078800609D421000798C3
:107150002A314CF0AEEF210006982E314CF0A8EF0A
:10716000002D26D0A87826000A36C107371D002931
:1071700008D00798A11C4CF09CEF0698A11D4CF07C
:1071800098EF01E0800707D5079831004CF090EFA9
:10719000069839004CF08CEFA878400709D52100FB
:1071A000079812314CF084EF2100069816314CF00C
:1071B00080EFF8BD000901D00020BEE47201E1BEFD
:1071C00001000000906F00000004000013BCD60214
:1071D0000120BCE4FEB51400060008000021284D83
:1071E0001F00082E0291019101D1E96800E0296990
:1071F00001AA00920A00390002ABFFF77FFA802053
:107200004DF07AEB3978042906D26B46217B1A7A45
:10721000891A1A79891821733978052906D26B469B
:10722000617B1A7A891A1A79891861736B46E18928
:107230001A7A891A1A798918082EE18106D11A7AE0
:10724000E968891A1A798918E96006E06B461A7AA2
:107250002969891A1A79891829614DF04EEBFEBD0A
:1072600001210170002141708170C1700181817222
:10727000C1720161416101834183018467E40000BF
:10728000D4650500F8B500252C009A4E28E00021B1
:107290007156884207D142206043B168401840309F
:1072A0004178491E4170002D17D142276743B068CD
:1072B00041213818095C00290FD1050042214DF009
:1072C00044EB002030567168814201DD401C307073
:1072D000B1683078791840314870641C2406240E57
:1072E00070688442D3DB2800F8BDF0B500281ED0BA
:1072F000804A4030012100274156D757B94216D065
:10730000002113009C6855680EE042224A43012682
:107310001319403301229A568657B24201DD521E9C
:107320005A70491C0906090EA942EEDB4770F0BDF0
:10733000F1B5002426006F4F17E042256543B86879
:1073400001222818010040318A56002A0ADD0978F6
:10735000FF2907D1009906224CF0E7FD002801D152
:10736000B8682E18641C2406240E78688442E4DB76
:107370003000FFF7BAFF3000F8BDF3B50024260057
:1073800081B05C4F17E042256543B86828180100BA
:1073900040314A78002A0BD00A7802998A4207D1F4
:1073A000029A01994CF0C1FD002801D1B8682E184D
:1073B000641C2406240E78688442E4DB3000FFF766
:1073C00094FF3000FEBD10B50024FFF7B1FF002888
:1073D00001D004002034200010BD70B506000D005F
:1073E000FFF7A6FF040009D1FFF74CFF04000622B7
:1073F00031004DF0AEEAFF2140200155002D04D0B0
:1074000020222900A0184DF0A4EA70BDF8B50D00A7
:1074100007001600FFF7B1FF040008D1FFF732FFA5
:1074200004002A0039004DF094EA40200555002E52
:1074300004D020223100A0184DF08AEAF8BD10B522
:10744000FFF776FF002806D042214DF07EEA294959
:107450000878401E087010BD10B5FFF78EFF002899
:1074600006D042214DF070EA22490878401E08708B
:1074700010BD612801D3573804E0412801D33738C3
:1074800000E030380006000E7047FFB581B01400F0
:1074900006001D0017D0002C15D00020215C00290B
:1074A00002D0401C4028F9DB0100083938290CD2F1
:1074B000104FF8688047029A2B003100200023F01B
:1074C0004BF83869804705B0F0BD4028FBD100215A
:1074D000605CFFF7CEFF020160184078FFF7C9FF3C
:1074E0000243C80F401840104019891C40290270FF
:1074F000EEDBE8E7F46505007CB505000E006946A3
:1075000001A84DF0CAEA00984DF0CAEA002403E051
:107510004DF0CAEA2855641CB442F9D37CBD70B55D
:1075200086B00A9E14000D000A00002E05910490FA
:1075300002D181794E07760F01005131022E08D019
:10754000032E11D10B000100200024F0C9F806B071
:1075500070BD10220093029201912300012205A91F
:1075600004A824F0BFF9F2E700912200290024F0DA
:1075700045F9ECE7FFB583B0040015001E000C9838
:107580000D9F00900020107018700C98B9004DF0FD
:10759000DCE9049800214170049908200870201843
:1075A000FE49042202904CF0C0FC002802D1287849
:1075B00004211FE0F94902980422091D4CF0B5FC92
:1075C000002802D12878082114E0F449F2F583E973
:1075D000010000008C73000000040000AC79F3B1DE
:1075E00002980422091F4CF0AAFC002802D1287836
:1075F000012109E0EE490298042208314CF09FFC79
:10760000002803D12878022108432870607B217B61
:1076100005020D431BD020000E30E54904220190E5
:107620004CF08DFC002802D13078042109E0E049BB
:1076300001980422091D4CF082FC002803D1307807
:107640000821084330706D1E01D0241DE3E7E07C63
:10765000A17C05020D430FD0002F09D02100009816
:10766000042214314DF07EE90098001D7F1E009029
:107670006D1E01D0241DEFE7CD490C980422083976
:107680004CF05DFC002805D10498102100780843D7
:107690000499087007B0F0BD70B504000D00C4492E
:1076A000002020700422103128004CF048FC0028F3
:1076B00002D12078042109E0BD49042214312800B8
:1076C0004CF03DFC002804D12078082108432070AC
:1076D00070BDB74904220C3128004CF030FC002862
:1076E00002D120780121F1E7B149042218312800A4
:1076F0004CF025FC0028EBD120780221E6E7F7B515
:10770000040000200F00050020701CE00298A90072
:107710000E18A7493000042210314CF010FC00284C
:1077200002D12078042109E0A1490422143130005B
:107730004CF005FC002803D1207808210843207074
:107740006D1C2D062D0EBD42E0D3FEBDFFB583B0EE
:10775000050010000E9F0D9E00224A7020220A7024
:107760006A78A91C5418291D0835FFF795FF287859
:107770006B461872687858721889AA1C81008D1897
:1077800001060698090EFFF7BAFF28786B461871B4
:107790006878AD1C587100959888B1008000451933
:1077A0000C984DF0DCE86B469888B04200D330006E
:1077B000820000990C984DF0D6E8A54207D2280027
:1077C000AD1C002F03D00178397040787870A54245
:1077D00006D22800AD1CA54202D20088000145193E
:1077E000A54207D20F982900002803D00F98042241
:1077F0004DF0B8E84EE7FFB581B004000D00002061
:107800000B996070A0702071E0702078F122104018
:107810000007000F207028781E006B461B7B820635
:107820000827002A1FDA9A061DD50422601D4DF094
:107830009AE860782021084360700C98002808D0EE
:1078400020780421084320700C98017861764078F4
:10785000A0760D98002831D02078384320700D98FC
:107860000078E0762AE0C20619D5DA0617D5504925
:1078700004220839601D4DF076E860781021084335
:107880006070A878000705D53078000702D5E07849
:10789000384302E0E07804210843E0700EE002077C
:1078A00008D51A0706D50422601D4DF05CE8607803
:1078B000384302E0C00701D0012060706078010702
:1078C00001D480061FD5E878000706D50A9800780D
:1078D000000702D52079384302E0207904210843CB
:1078E0002071A878010705D53178090702D5E0781D
:1078F000384307E0410708D53178490705D5E078D6
:1079000004210CE0E07005B0F0BD800705D53078AB
:10791000800702D5E078022101E0E07801210843E8
:10792000F0E7F0B505000E0017009C4621A00EC838
:107930008DB00AAC0EC404A81D490C3C1E310EC902
:107940000EC02B0007ADD0C51022202061466C462A
:1079500007C4032204A907A823F0CEFF0DB0F0BD91
:10796000FFB587B00E00170015480022FF21006800
:10797000D243F5314CF0EEEF018904000D180DA053
:107980000490082001900620029003902B00032011
:1079900001AA04A90596069724F07AFD0A981022F8
:1079A00029004CF0E0EF20004CF0A8EF0BB0F0BD48
:1079B000225B0500504D4B204E616D6500000000BC
:1079C000646C0500032210B5FF494CF0B8FA00289A
:1079D00001D1012010BD002010BD10B5828B3A49A5
:1079E000010000008877000000040000FFA320DDF4
:1079F0000400FFF7F1FF002806D0E078062801D048
:107A0000052801D1012010BD002010BDF34910B59B
:107A100004000322C91E4CF09CFA002806D0EF494E
:107A2000032220004CF095FA002801D1012010BD5E
:107A3000002010BD10B50400FFF7E8FF002807D0B4
:107A4000E1780120022904D0062902D0042900D0BF
:107A5000002010BDFFB581B01C0000260700039870
:107A6000FFF7E8FF002817D13800FFF7C0FC05003A
:107A700012D00398FFF7BBFF002806D0029A23001C
:107A800039002800FFF776FF05E0029A230039004D
:107A90002800FFF750FF012630003EE7FFB581B018
:107AA0000C000500002069780A9E8A060127002A3A
:107AB0007EDA302121701221200061700422691DBC
:107AC00010304CF05AEF01200022A070E2702072BA
:107AD0006272A073E2732879010720000A3000293E
:107AE00003DABE4904221F3102E0BC4904221B31E3
:107AF0004CF042EFE878010703D5B84904221F3162
:107B00000EE0410703D5B54904221B3108E0800788
:107B100003D5B2490422233102E0B04904221731CF
:107B2000201D4CF02AEF0B982F000937002821D098
:107B30002878800702D40398002802D1002E19D09B
:107B400001E0002E09D01022310038004CF014EF73
:107B500028780221084328700CE0049903983B0020
:107B60006A1DFFF777FF2978C007FD22800F1140BB
:107B7000014329702878410703D4810701D4000705
:107B800030D5687E2075A87E60756078801C607036
:107B90002878810701D4000778D50020A075E0750A
:107BA0006078801C6070287880070ED5012000E086
:107BB00019E0A0750020E07520001022390018306F
:107BC0004CF0DAEE607810306070287800075DD5F0
:107BD0002900200004221B3128304CF0CEEE6078C2
:107BE000001D607052E0CA0601D4090750D5DD219E
:107BF00021701621617079490422C91DA01C4CF026
:107C0000BCEE390AA771E171390A27736173390A29
:107C1000A7742000E1740422691D14304CF0ACEE0E
:107C20006878C10620000E30861F002911DA6B49E2
:107C30000422C91C4CF0A0EEE878410703D567493F
:107C400004220B311FE0000720D5644904220F31C4
:107C500019E02979090703D5604904220F3102E0B0
:107C60005E4904220B314CF088EEE8780107ECD431
:107C70004107E4D4800703D558490422133102E0B8
:107C800056490422C91D30004CF076EE6078801C05
:107C90000004000C41E6F8B504000E0015001F00BA
:107CA00038214CF066EE002F01D0052000E00620C0
:107CB000A070000A002DE0700AD010223100A01D33
:107CC0004CF05AEE0220207000206070102016E068
:107CD00010223100A01D4CF050EE01202070002039
:107CE0006070103620000822310016304CF044EE4F
:107CF0002000082231001E304CF03EEE2020207182
:107D0000000A6071F8BD02002020002904D011791A
:107D1000090700D510207047D1780A07FAD48A07DE
:107D200001D50D207047C907FCD0052070477CB5F0
:107D3000002405000E00042201A84CF01EEE0422CF
:107D4000311D68464CF018EE0198FF220100120226
:107D50000306114009025918060013021E40360A94
:107D60008919000E081800990A400E060B401202ED
:107D7000B2181B0AD218090E51186A6E82420BD330
:107D800082420AD12A6E8A4206D38A4205D108432A
:107D900003D1A86E002800D1012420007CBD7CB551
:107DA00004000D00042201A84CF0E6ED0422291D78
:107DB00068464CF0E2ED0198FF22120201001140EA
:107DC000030609025D18010013021940090A691827
:107DD000000E091800980506024001E0175B050037
:107DE0001202AD1802001A40120AAA18E5998C91E5
:107DF00001000000847B0000000400000BCC5569EA
:107E0000000E101861660143206601D10120A066B2
:107E10007CBDF8B50D00040017001E0038214CF0A1
:107E2000B2ED002F01D0022000E001200421102D2E
:107E30000BD102222270002208436270A070000A57
:107E40002A003100E070A01D33E0202D19D101225D
:107E50002270002208436270A070000AE0701022B5
:107E60003100A01D4CF092ED3100200008221831A5
:107E700016304CF08CED31000822103120001E30FD
:107E800017E00D2D01D0052D18D1002222700843D6
:107E90006270A070000A002FE07003D00120A27170
:107EA000E07102E0F08CA071E27120002A00310044
:107EB00008304CF06CED280A25716071F8BD70B582
:107EC0001500040006224CF062ED06222900A01DD8
:107ED0004CF05CEDFC492173080A607370BD70B50D
:107EE0000D0001000400513186B010220E0002A8DE
:107EF0004CF04CED102130004CF044ED002200928B
:107F0000E078A178000208430102000A0143091D3C
:107F10000904090C2A0020001023FFF71EFB102281
:107F2000300002A94CF01FF8002802D0002006B053
:107F300070BD0120FBE7F8B5002824D004006034B0
:107F4000257C2600E47B2D0225432C005F3424048D
:107F50008273240C0322C2732202270A3A4302745A
:107F6000120A42742A022D0A2A43F273120A327448
:107F7000221D009313041B0C0A0019000E3010235D
:107F8000FFF7EBFA2000F8BD10B50178DD290CD120
:107F900004004078072808D9CC490322A01C4BF0E4
:107FA000E2FF002801D1200010BD002010BD70B5F7
:107FB00004000D001600002816D013E02078DD28FC
:107FC0000BD12000FFF7E0FF002802D04179B14239
:107FD0000BD06078002800D102256078A41C2D1AEF
:107FE000AD1E0419022DE9DC002070BD70B516002D
:107FF0000122FFF7DCFF04000AD06278A51D921F62
:10800000A91C30004CF0C2EC28788007800FF08467
:10801000200070BD7CB50400150002004032130042
:108020009278603412028A845B781A438A84002230
:10803000D2430A62A1786278090211430A02090A4E
:108040000A431604360C310A6670A1708179E31C6C
:108050004907490F022901D0032911D10021F20853
:108060000091521E0221280001934CF040EDA078AF
:1080700061780002084308386070000AA0707CBD77
:10808000FF22521C0100019210223131280000967B
:1080900022F005FA7CBD70B505000C0000281DD04B
:1080A000002C1BD0210009312800FFF74AFE0028D0
:1080B00014D06079C00713D0A079000707D520003D
:1080C0002022290011304BF04EFF002806D1290054
:1080D00040312000FFF703FF002801D1002070BDD0
:1080E000012070BDFFB581B004000D0016000A9F8D
:1080F000002840D0002D3ED0722120004CF042ECF0
:10810000049A31002000FFF7DAFE2879A074267D5A
:10811000F7200640A87901210007C00FC0000643E0
:108120002675E07C0843FD21E074084069798907E1
:10813000C90F49000843E074280009304CF03AECBC
:10814000210017314BF0DCEF28000D304CF032EC01
:1081500021001B314BF0D4EFA979F0084907C0008A
:10816000490F0843002F207505D020002022390038
:108170001F304CF00CEC9AE4FFB581B004000E0007
:1081800017000A9D002838D0002D36D0722120001B
:108190004CF0F8EB049A39002000FFF790FE207DA8
:1081A000F7210840F107090F08432075E07C0F21F3
:1081B0000843E074286FFF263602010031400206B2
:1081C00009025118020037023A40120A8918000EBB
:1081D0000818210017314BF094EFE86E0100314090
:1081E00002060902521801003940090A5118000E0E
:1081F000081821001B314BF084EF58E44EC5E3957D
:1082000001000000807F0000000400005816860571
:1082100010B50400FFF7F4FB00280AD0E078062828
:1082200005D0052803D0042801D0032801D101205E
:1082300010BD002010BDFFB581B0150006000A9CDE
:108240000F0006224BF099FE002807DA06223100C3
:1082500020004CF0A6EB0622390006E00622390089
:1082600020004CF09EEB06223100A01D4CF098EB54
:108270000499202228004BF080FE010020000C30E1
:108280002C34002906DA202229004CF08AEB0499CC
:10829000202205E0049920224CF082EB20222900C4
:1082A00020004CF07EEB0CE4F0B585B00A9C0C9EEF
:1082B0002500C8350095FFF7BEFF002E09A31DD08D
:1082C000FF2281324C2003921A0001900B9820214A
:1082D00016230095029424F015F9EFE4888E00002F
:1082E000175B05005061697277697365206B65796A
:1082F00020657870616E73696F6E000040224C20BB
:1083000003921A0001900B982021162300950294E5
:1083100023F092FBD2E4FFB583B003980D9F0F9D2D
:1083200000283AD0002F38D0002D36D08E480022B9
:10833000FF210068D243F5314CF02AEB0189109AF5
:108340000C18039902920191060000940C9B069A66
:1083500004990598FFF7A8FF1022210038004CF07F
:1083600020EB10220E98A1184CF01AEB21001022DD
:10837000203128004CF014EB210028000822303175
:1083800010304CF00EEB2100280008223831183054
:108390004CF006EB30004CF0D0EA07B0F0BD0029FD
:1083A00001D0022100E0FE218174017DC908C900CD
:1083B000002A01D0C91C04E0002B01D0891C00E078
:1083C000491C0175704770B50D0001890C1821001A
:1083D0002800FFF76AFE00280DD06079C00709D198
:1083E00021002022113128004CF0DAEA20216818FF
:1083F000FFF7AAF8200070BD002802D00021016715
:10840000C1667047020070B5080010D0C41DF93471
:10841000E1680026914209D10500E035297F022953
:1084200002D15249096888472E776660E66070BDC0
:10843000002910B50FD0CC1DF9342269824208D131
:10844000E031087F022804D1484A606992680E2111
:1084500090470020206110BD70B500290FD0CC1DC1
:10846000F934A2680025824208D1886F002805D11E
:108470003E4AA560926860690F219047A56070BD73
:10848000FFB581B00400C51DF93568680E000027EE
:1084900000280DD1A868FDF78AF8AF60049A230080
:1084A000FF330092039A093321003000FDF72DF8C5
:1084B00027666766A76668E6F8B50400FF30401CCB
:1084C00000690D0016001F00FDF771F82300FF334F
:1084D00011333200210028000097FDF716F8F8BD8F
:1084E000FFB581B00C0005001F0080204CF02CEA85
:1084F000020028002100E61D1D4D0123E031F93660
:10850000002801D10B7705E0022073600877002076
:108510006066206610004CF018EAF068FDF747F836
:108520002300FF3303980D332A0021000097FCF746
:10853000ECFF2AE670B500254567802185670D5060
:10854000C567FF30401C04004068002807D1E06880
:10855000FDF72DF8E5602069FDF729F82561A06891
:10856000FDF725F8A56070BD646C0500247A050050
:108570000087930300220A70007801224006800FD2
:10858000002806D00222012803D0032800D1087059
:1085900070470A707047030000B54CF03AEA0805CE
:1085A00007070509090B0B05032000BD022000BDCC
:1085B000012000BD002000BDFFB50400099E0A9DFA
:1085C00070788006400FFFF7E6FF0123012C20D1D1
:1085D000747864072C780DD5A40704D51E00147890
:1085E0008640344314702A78D20711D00A78834029
:1085F0001A430CE0A40704D51E0014788640B44347
:1086000014702A78D20703D00A788340629C589A63
:10861000010000007C830000000400000E3FE545DF
:108620009A430A70FFBD002CFCD12C78A40709D511
:108630001C0016788440A6431670039F3F7827409D
:10864000374317702A78D207ECD00A7883409A43D0
:108650000A7003980078184010430870FFBDF8B501
:108660000E00018917000D182C00203400206070C6
:10867000A370E070FA490822201D4CF09CE920000C
:108680003A0031000C304CF096E90C37380A2F7064
:1086900068702000F8BD10B5F24B03701B0A4370E0
:1086A000002383710924C371037184700029C3708E
:1086B00002D10221017210BD121F037213000F3389
:1086C00083701B0AC3708B784373CB788373091D47
:1086D0000F304CF070E910BD10B50289141820005D
:1086E00002222030427000228270C2703F22001DA0
:1086F0004CF060E9432121700021617010BD03003E
:1087000000B54CF090E9080B05050B070709090BAC
:10871000012000BD022000BD032000BD002000BDDF
:10872000002801D1012070470128FCD100207047AA
:10873000FFB581B004000D001700067808214CF049
:1087400036E9082E267022D2002D1DD0002F1BD016
:108750000498002801D00120607068788006400FDE
:10876000E070697830354907C90F21713978617136
:10877000A9796A7909021143A171090AE171FFF728
:10878000BEFFFFF7CDFFA070082005B0F0BD0020B0
:10879000FBE7002805D0022805D0032805D00320D8
:1087A000704702207047012070470020704738B59D
:1087B0000400ADA000680090DD20207018206070DB
:1087C0000422A01C69464CF0F6E80120A071E0717B
:1087D0000020207238BD10B50400FFF7E8FF00202C
:1087E0006072A17A9F220B091B01DB1CEF210B4059
:1087F00013405B065B0EA372E37A031D1B071B0F7E
:10880000A033E372030A20736373A37B1B091B016C
:10881000DB1D0B40134020335B065B0EA373E37B31
:10882000A423E3732074000A6074A07C0009000193
:10883000801C0840104040304006400EA074E07C90
:108840004320E074BC20207500206075A07D0009E5
:108850000001801C0840602108434006400EA075BE
:10886000E07D3220E075662020760020607610BD25
:1088700030B5827A5206940F01221300A340847B04
:108880006406A50F1400AC401C43837C5B069D0F5F
:108890001300AB402343847D6406A40FA2401A4317
:1088A0001206120E002804D04378182B01D10F2A8B
:1088B00001D0002030BD002903D0007A0007000F4E
:1088C0000870012030BD0278F9231A400B785B064E
:1088D0009B0F5B001A43F72302701A400B78DB06EC
:1088E000DB0FDB001A43130702700A781B0F12011B
:1088F0001343037042784B781207120F1B011A437F
:1089000042704B78120912011B091A434270CA784F
:108910008B78110219434180704770B503005C7871
:108920000120042C19DA1D78002D0ED0012D04D061
:10893000022D12D14D4B1B6804E0DD789E782B028E
:10894000334307D064000B5304E06400095B997063
:10895000090AD9704421116070BD002070BDF7B5BF
:1089600082B004000E004578042D01DB00200CE7E6
:1089700080204BF0F4EF01902078002823D00128CC
:1089800021D002284CD169018D196A882271120AFE
:108990006271705AA070020AE27062792379110242
:1089A00019432700461A0A37002E13D0A868310051
:1089B0004CF054E8A11D4BF0B8EBE86831004CF0E6
:1089C0004EE839000CE06801801920214CF00AE8DB
:1089D000022426E0A11D00204BF0A6EB3900002068
:1089E0004BF0A2EBA888A073000AE073E88820741B
:1089F000000A60742900200010310E2212304BF062
:108A0000DAEF0498203400882070000A607020217A
:108A100028004BF0E8EF0498002122241549444F28
:108A20000100000078870000000400005DE53629A1
:108A3000018000E0002401984BF09AEF2000AEE6A0
:108A400010B50C000021002C12D06278002A0FD043
:108A5000217838300170090A417061788170090A03
:108A6000C1706278A11C001D4BF0AEEF6178091D4A
:108A7000080010BD4C5B05006E8000000050F20243
:108A80000C66050000210182FF22416082740160B2
:108A90007047FFB585B0040015001E000698008BD6
:108AA000000904900698007E0007000F039009D18A
:108AB0000698C078400705D406980088A08020005A
:108AC00009B0F0BDA088202803D920380004000C8C
:108AD00000E0002000900E9800780128039808D14B
:108AE000002808D0AD4B61891B68E08803229847B5
:108AF00055E0002833D10E98002101702868002825
:108B00000DD1A64F02E001204BF0E2EF7D21B869C4
:108B1000002209014BF050EF00282860F3D09F4954
:108B2000002001908968286888473000FFF7AAFF75
:108B3000286830600189994B4718380020307060F0
:108B40005B68202206993800984795480068934949
:108B500049694018B06029686069486130E0308A2E
:108B6000049988420AD13068062201894118069882
:108B70000C310C304BF015FA002812D028684BF05D
:108B8000F0EE864B61891B68E0880322984730002D
:108B9000FFF778FF0E990120087000202860002060
:108BA0008EE7306801894718B07C0399401C8842E1
:108BB000E4D138880099401838807A4800680190DC
:108BC000784801680198091A0098081802900CD09A
:108BD00001990698714B41185B687068029A2031C0
:108BE000984770680299401870600698C0784007EE
:108BF0001CD40098002805D1A18838882022511A59
:108C0000401A3880F878FB210840F87029683888C5
:108C1000624B88801B686189E08803229847300096
:108C2000FFF730FF28680021296049E70498308267
:108C30000398B07456E7FFB587B00400119E4069F1
:108C400002902089109D00190390008B0009069066
:108C50000398007E0007000F05900398008868388D
:108C60000004000C04900598002832D128680028E0
:108C70000CD14A4F02E001204BF02AEF4A49B86973
:108C800000224BF09AEE00282860F4D0434928686F
:108C9000896888473000FFF7F5FE28683060018951
:108CA0003E4B47183F48202200683818203070603B
:108CB0005B680399380098470498603038803848DA
:108CC0000068364949694018B060296860694861A0
:108CD00014E0324930680B68002802D00189471837
:108CE00003D16189E088032254E0B07C0599401CDF
:108CF000884225D13988049808183880099900914C
:108D00002849019703980968049A41187068089BDC
:108D10002431121DFDF792FC002815D11F4F029837
:108D2000F96888473B686189E0880322984728688A
:108D30004BF016EE3000FFF7A5FE002028602AE079
:108D40006189E0880322F1E7144920000969884716
:108D50000398C078400710D4296838880F4B888062
:108D60001B686189E088032298473000FFF78AFE7C
:108D70002868002129600BB0F0BD06983082716828
:108D80000498064B081870600598B0741B686189D8
:108D9000E088032298470020EDE7000020660500E8
:108DA00000A600804C6C05002C060000FF49002046
:108DB000087548754039C86588650866C03188609F
:108DC000C86068398862C862086348638863C8639A
:108DD00008644864086248628864C8640865486535
:108DE0007047F0B5040085B0F7F7F2FB0090012062
:108DF000102C02D0202C00D00020EC49EB4A20316E
:108E000004918979683AA14210D1E94B810089180F
:108E10000D695E6EB54209D189689D6EA94205D182
:108E20004100891849889B88994267D0F0A31CC7E4
:108E300001000000748B000000040000A98A439D1B
:108E40004100891803914F88F90702D07D26F6006A
:108E500000E0012680008018029081686B460A04B9
:108E6000120C090C9A80D9800569A81AD44A70435B
:108E7000403A002950601AD1102C0BD1D14880689B
:108E8000002803D1D048D14968430CE0D048D149EB
:108E9000684308E0202C03D1CF48D049684302E062
:108EA000C948CD4968434BF0EEED6B46D8806B4620
:108EB000D888291AC24875437143403805608160DB
:108EC000A106890F0FD0390A02D0390A714306E092
:108ED000BC498968002901D1C14900E0C149C1628A
:108EE000C14901634163B648042180304170FFF7F6
:108EF00067FFBE49012008600498847102980169E7
:108F0000B0484166029989688166039949888180E1
:108F10000098F7F76CFB05B0F0BDA948002101757A
:108F200041757047F3B581B00D00A800A44CA54E63
:108F3000403C7178071978688D4209D132780199DF
:108F4000914205D1F16E884202D1A169002921D157
:108F50009B4A683A9169401AC10F08184110A161F3
:108F6000D069814200DC0100A161009100980321D9
:108F70004BF0E8ED00226262206200996161E061DD
:108F80008F484030C263403002707868F066757078
:108F900001983070FEBD8B4810B58078012829D02B
:108FA000FBF7B4FE8648203080798006800F21D1FF
:108FB000FCF7ECF9834A803251641064804A18321D
:108FC000D3699269801A7E4A9941403AD1681369FF
:108FD000401A5B1A834200DB18001368591A814259
:108FE00000DC0800516A081881495062884200DD9F
:108FF0000100516210BD102010B5F9F7B0FF002834
:1090000008D06F4820308088000A02D0032010F07A
:1090100048F810BD77490020086077490880032090
:1090200010F03FF803200FF0DFFD10BD644910B5CC
:1090300040398A6B82420ED100208863080060307C
:109040008179012901D0022906D10121890281807B
:1090500023200FF0C9FD10BDFFF79DFF59490120E6
:10906000887010BD564910B54039CA6B824210D184
:109070000020C8635349032088705148203081790B
:109080008906890F05D001218902818023200FF0F4
:10909000ABFD10BD70B54A4D2035A8798006800F14
:1090A00024D148488078022820D1454C1421200042
:1090B0004838042261568256914217DAF7F792FA3D
:1090C000060028F090F800280DD0207D401C207567
:1090D000A879022801D0082805D1FCF757F9384AA9
:1090E0001832516110613000F7F781FA70BD10B588
:1090F000FAF7BEFE002804D04048007E002808D0C1
:1091000005E030488078002803D0042801D00120F1
:1091100010BD002010BD70B50D00294940390A6C02
:10912000824209D100200C0060340864A0798006D6
:10913000800F02D0FFF75FFF70BD0FF0BDFF00286A
:10914000FAD00221280023F097FB0028F4D0FFF783
:10915000CEFF0028F0D0A079194C4034042809D162
:10916000FFF798FFA06B0028E6D0002128000DF043
:109170008AFE70BD0828FCD127F0D5FF002802D058
:10918000FFF788FF70BDA06B0028FBD028000DF012
:10919000A0FE70BDF8B50022094E0A4F403E716C2A
:1091A000084D803781427ED10020706430005830F5
:1091B000C36A826A416B006B841AA86A99411FE0F6
:1091C00060820500486605001027000050C30000BB
:1091D0003075000080380100204E0000409C0000E7
:1091E000983A0000A8610000B80B00009C5601C02E
:1091F0006079FEFF143501C0DC690500F87E0500CA
:10920000401CA862E1173C607960BA68FB68A01A4C
:10921000994103D279683868F960B8603A6938686A
:109220007B697968121A8B4103D279683868796151
:1092300038613A68386A7B68796A8018BD29038F7B
:1092400001000000708F000000040000FA5090F14F
:10925000594179623862AA6A00234BF00AECF9613D
:10926000B8610A27FF49A8680A007D238032DB0025
:10927000A031002810D0F06AC01AA0426FDA487DF1
:10928000002802D0401E487569E04F75E868002844
:1092900065D10120106362E0F2487D23C06ADB00E3
:1092A000C61AF04B6033A6422CDADB79ED4E9B00F8
:1092B0009B199C465B687D2600E053E076019B1B72
:1092C000A34210DA487D002802D0401E487544E0D1
:1092D0004F75E868002840D12C62E869401CE861BD
:1092E0000120106339E04F756B69DE4AC018634690
:1092F000D0625C68DC4BE318984200DB1800D06257
:1093000068622AE06A697D269446821AF600961BF6
:10931000A64222D94F750C7D002C02D0641E0C751C
:1093200017E0DB79CF4C9B001B195B68CE4E9B1975
:10933000984205D12B6962469A1A8018E06200E0D3
:10934000E262CA48E26A824200DD1000E062A86977
:109350000875C448C06A686201E0A86908752620DB
:109360000FF04CFCF8BD10B5BE4C606CFCF747F933
:109370000020606410BDBB4910B58A6C824214D1D4
:1093800000208864486C00280FD008005830C36B58
:10939000826B416C006C801A9941002806D1FFF75E
:1093A000E2FF00210800FFF7FFFE10BD0028FCDDF2
:1093B00028200FF023FC10BD10B5AA4CE06BFCF781
:1093C0001EF90020E06310BDA64910B5CA6C8242A8
:1093D00018D10020C864C86B002813D0080058308A
:1093E000C36C826C416D006D801A994100280AD1CE
:1093F00024F004FA002806D1FFF7DEFF0021080060
:10940000FFF73AFE10BD29200FF0F8FB10BD38B56C
:10941000944D296D81421BD100202865FBF786FC05
:109420002C005034002806D1FBF77AFC0822009269
:109430008F4A230008E00120FBF74CFC002807D0EE
:1094400008220092AA6A23008A480021FCF785F8C6
:1094500038BD844808B5082203000092826A854816
:1094600050330021FCF779F808BDF3B581B00D0049
:109470007D217C4EC900306880024BF06EEB040009
:109480004BF01EEB7C4FFA6A002A0BD0220000231F
:109490004BF0EEEA31002839096AA01A914202D253
:1094A000001900E02000002D07D03168A94204D344
:1094B0007D21A802C9004BF0F0EA0022694B00921E
:1094C00002006E4801994033FCF747F8FBF768FF4C
:1094D000F967B867FEBD70B5F7F78EF8614D060005
:1094E000A86B0024002802D0FCF789F8AC63E86B75
:1094F000002802D0FCF783F8EC63696C080002D006
:10950000FCF77DF86C64A86C002802D0FCF777F8B3
:10951000AC64E86C002802D0FCF771F8EC64286DAC
:10952000002802D0FCF76BF82C653000F7F769F8DB
:1095300070BD70B5F7F760F8050024F05FF904001E
:1095400007D04F4800218A008258491CA41A0729D5
:10955000F9DB2800F7F755F803F0FAF8002815D0E2
:10956000484801694069814210D1002C0ED1002089
:1095700017F064F8002809D117F060F8002805D129
:1095800041480078002801D1012400E0002405F0C2
:109590008BFE012C01D1012807D13C48006800282E
:1095A00003D13B4C2078002803D119200FF026FB73
:1095B00070BD012001F0FDFC20783649401E20706E
:1095C000FF20F5300CF01CFE70BD0A68824202D10B
:1095D00000200860ADE77047FEB52248214E60309C
:1095E000817934008A063500C079920F8034C03505
:1095F000002A72D0204F8037012860D110294FD126
:10960000FBF7CEFE3A00D36A926A801A9941019123
:1096100000901BF025F807001BF026F887426870C1
:1096200008D815482978806B814203D21AF0F9FFD7
:1096300000286CD0104F009880373A6B7B6B0199F3
:10964000801A99410AD3F96AB86A0023CA9DE725AE
:10965000010000006C930000000400004595B54235
:1096600059405840084303D008488078012858D111
:10967000002233002A7019E02082050048F4FFFF21
:1096800088130000A60E00002F9100004866050018
:109690004B8E0000F47802C000A00080940C0004FF
:1096A0006C69050007690500EB920000B06850E0A6
:1096B000080055E0202955D11AF0BAFF002805D03E
:1096C0001AF0C3FF002801D1012058E0B068B06251
:1096D00054E00028EFD11AF0A2FF002808D0FC497E
:1096E0002878C96B884203D2401C2870ECE748E018
:1096F000F748006B002836D0FBF75CFEBA6AFB6ABD
:10970000801A9941019100901AF079FF00280AD03F
:10971000EF482978006C814205D210F032FA0A280D
:1097200001D22878E0E7BA6B0098FB6B0199801AA8
:1097300099410AD3F96AB86A00235940584008434E
:1097400003D0E34880780128EBD100222A707068AA
:109750003300D96A401ADF49186189698842A7DD58
:109760001861E26364E0F16A70683200401AD94916
:1097700030618969884200DC080010610020E063E4
:1097800056E0012823D11AF075FF07001AF076FF82
:10979000874268700ED8CE482978406B814209D242
:1097A0001AF049FF002805D10120E0632878401C09
:1097B00028703DE000212970B068F060F569726999
:1097C0006B005B19D218801A3061E16330E01AF047
:1097D00026FF002804D00120E0630020706227E00B
:1097E0001AF00DFF002802D0BA48806900E07068C6
:1097F000716A3200451AF5603368B64E366A9B1BB3
:10980000AB4200DC1D00D560D76956697B00DB19CF
:10981000F318B04EEB1A1361B669B34203DA0123B1
:10982000081AE36303E00023281A0818E363506270
:10983000E06BFEBDA84AA649002810B50CD090697F
:109840000867D0694867012107204BF094E903219C
:1098500007204BF094E910BD086F9061486FD0610C
:1098600010BD70B528219B484BF0E4E89948D02101
:1098700028304BF0E0E897480421018097490161C6
:10988000974900228160924B42808280996800292A
:1098900003D194494161944902E09449416194495A
:1098A0007D24E4008461C1609249C161610001626C
:1098B0008849012520310D7103254D71C4840800AC
:1098C00088309A7002639969203001750A21827587
:1098D000417570BD10B522F05BFF002805D01AF06D
:1098E0007CFE002801D1012010BD002010BD794868
:1098F0000021E830C160704776480021E83081607F
:109900007047734838B5C16D002917D0714C006E8F
:1099100028346063E06CFBF77CFE08222300009291
:109920007548626B4C330021FBF721FEFBF742FDCB
:10993000220058329064D1645165106538BDF8B585
:10994000FBF738FD634A8032536A126A801A604A14
:109950009941156E5F4A6B00283255631469DF1711
:109960000200E6170D001800390080186941001B3D
:10997000B14101D20120F8BD0020F8BD544838B5EE
:10998000416D002917D0534C806D28342063A06CA2
:10999000FBF73FFE0822230000925848226B483311
:1099A0000021FBF7E4FDFBF705FD22005832906330
:1099B000D1635164106438BDF8B5FBF7FBFC454A30
:1099C0008032D36A926A801A424A99418832D279A7
:1099D000012A11D03E4A3F4B926D28331A63DC6A4C
:1099E0005500EF17E6170B00390028185941001BE6
:1099F000B14101D20120F8BD0020F8BD38B5354C89
:109A00002834E06BFBF705FE0822230000923C4857
:109A100022693C330021FBF7AAFDFBF7CBFC2200B7
:109A200058325162106238BDF3B587B0FFF773FB4F
:109A3000002805D108983B2802D0089835282BD15A
:109A4000244F089B2837380050300690183805906E
:109A50008C30051F04903E003C0024388511465C84
:109A6000010000006897000000040000164F662EF9
:109A700080366034292B03907BD018DC172B79D0EB
:109A800008DC022B05D00A2B75D00B2B74D0122BBF
:109A9000DFD178E2192B70D0272B6FD0282BD8D1AB
:109AA000FFF794FF002801D0FFF772FFAEE2333BCF
:109AB0004AF0EAEF0DF0F0EFEBEBEBEBEB08EEED3D
:109AC000EBECEB00074880780428EFD0FFF70CFFA1
:109AD00000286FD0A07901900CF072FF00281BD0F5
:109AE000012033E048660500F8810500C0A0008031
:109AF000204E00001027102750C30000307510279B
:109B0000803801003075307594110000E990000034
:109B100097900000998D00000CF068FF002801D09C
:109B2000022013E0306B00280FD1FF480088042882
:109B300001D110200AE0082801D1202006E00DF014
:109B400005FA002801D0082000E00420FFF771F991
:109B5000F64EB0780028A07919D18006800F0ED07B
:109B600022F080FE686800280CD101F0ACFA686031
:109B700008E0C0E13EE238E281E1B9E1EEE0012037
:109B800022F05AFE0120B070FFF75EFE1FE001993F
:109B900088421CD08006800F01980CD08006800F70
:109BA00015D122F05FFE6868002810D101F08BFA11
:109BB00068600CE03EE08006800F08D0012022F0B3
:109BC0003BFE6868002802D0049801F0A7FA002044
:109BD000A080FFF794FC00F02EFCFBF7C0F80020FB
:109BE000B865FFF70BF91AF01AFD002800D0012024
:109BF000E071A0798106890F02D1E179FFF7B0F910
:109C0000F6F70EFD0290FFF7FBFC002843D0012081
:109C1000B070FBF799F8A079012804D0022802D08F
:109C20008006800F05D0FF20401CA08023200EF06E
:109C3000F9FF83E0BD498878002826D00428FCD0AD
:109C4000FFF75DFC00F0F7FBFBF789F80020B86533
:109C5000FBF77AF86868002802D0049801F05EFAF1
:109C6000B249002088703063039A9075039A0A20E5
:109C700050758869039908750020FFF7E5FDA07904
:109C80008006800FD9D0FFF7D4F9BFE13AE12BE18C
:109C9000F8E0A3E177E10020FBF730F8002802D1DB
:109CA0000120B865E5E0B078012805D1FBF78CFB11
:109CB0009E4A8032D1629062A07920280ED1E0794C
:109CC00001280BD11AF0CBFC002807D00822009203
:109CD000BA6A9748069B0021FBF753FCFBF774FB1D
:109CE000914A8032D16190610220B070A0798006E3
:109CF000800F19D0002002F00AFD6868002802D009
:109D0000049801F00BFAE079002804D0012815D15D
:109D1000A079102812D1FFF77BFEFFF71AFE00286A
:109D20000CD0FFF7F8FD09E008220092FA6881489C
:109D3000059B0021FBF725FCFFF76AFEA0790828A8
:109D40000BD00428FCD08106890F75D0E179002959
:109D5000F6D0012970D11028FCD184E0F6F760FC20
:109D600002900020B865FFF7E0F900289AD06F480C
:109D70008078012805D1FBF727FB6C4A8032D1623D
:109D80009062A07920280ED1E07901280BD11AF039
:109D900066FC002807D008220092BA6A6448069B35
:109DA0000021FBF7EEFBFBF70FFB5F4A8032D1612E
:109DB00090615E4802218170A0798006800F19D0E1
:109DC000002002F0A4FC6868002802D0049801F08A
:109DD000A5F9E079002804D001283DD1A079102808
:109DE0003AD1FFF715FEFFF7B4FD002834D0FFF796
:109DF00092FD31E008220092FA684E48059B00214E
:109E0000FBF7BFFBFFF704FEA079042809D1FFF799
:109E10005FF9B06B00281FD0079800210DF051F8B2
:109E20001AE0082801D002281BD127F09AF900284F
:109E300003D0FFF74DF90DE017E0A079082801D114
:109E4000B06B02E0022805D1F86D002802D0079817
:109E50000DF05DF80020F865A079082803D00428EB
:109E600001D0A0796FE7002189E002985019698537
:109E700001000000649B000000040000E220139A2F
:109E8000F6F7DDFBCCE00298F6F7D9FB002009B02D
:109E9000F0BD0120B063C3E0FFF73BFBFAF769FFB9
:109EA0000020B865A079012801D0022801D1012045
:109EB0000FE0042801D008280DD100F0C6FAFFF702
:109EC00092F81F49012088700021B163A188090A16
:109ED000D8D1A080A4E08006800FD3D0A088000A4B
:109EE000E5D06868002802D101F0F7F868601448EE
:109EF00081780229C6D10321817091E0A079800682
:109F0000800FBFD0FFF76FF87BE0FFF72CFD002834
:109F1000B8D0FFF70AFD83E0F6F78CFB0290A0793A
:109F20008106890FABD0E179002903D00129A6D1A0
:109F30001028A4D1FBF752FA014E07E0F881050082
:109F4000486605002F910000618D0000B26FF36F2D
:109F5000821AE0799941012801D1756C00E0B56C55
:109F60000B000021A81A994189D2F06C00283868AA
:109F700005D0E1798900C9194968441A00E0441BF9
:109F8000002CCFD03868A04200D278E700F05DFA0C
:109F900021000798FFF787FA71E76868002802D068
:109FA000049801F0C5F8FFF7B4FA00F04EFAFAF79A
:109FB000E0FE0024BC65FFF7B3FCFFF7ACFCFAF74A
:109FC000CDFE0898332802D00898342803D1F949E7
:109FD0000420887001E0F748847003988475039921
:109FE0000A204875F348346303998069087517E0BF
:109FF000F0498878042813D10020887010E0FAF71F
:10A00000ADFEEC490120F8E7FFF783FA00F01DFAF6
:10A01000FAF7AFFE0020B865FFF782FCFFF77BFC84
:10A02000012034E710B5FFF78AF8002806D0E2488F
:10A0300080798006800F01D0012010BD002010BD66
:10A0400010B50400FFF77BF8002813D0FFF7EAFFF4
:10A05000002811D1D748807802280DD1D648152183
:10A0600020384156012901DB002C05D005F06FF99D
:10A07000002801D0012010BD002010BD10B5FFF751
:10A080005EF8002806D0CB4901208978022900D04B
:10A09000002010BD012010BD10B5FFF750F80028BA
:10A0A0000ED0C54CA0798006800F09D002F076FB57
:10A0B000002805D1A088C11FF93901D0012010BDA9
:10A0C000002010BDBC486038806D7047BA4901203F
:10A0D0006039C8657047B8486038006E7047B64947
:10A0E0000120603908667047B3490020603908666E
:10A0F0007047B148603080687047AF4801216030D8
:10A1000081607047AC486030C0687047AA48012140
:10A110006030C1607047A84868384079704710B512
:10A120000400FFF70CF800280CD0002C0AD1FBF734
:10A1300055F9A14A083A5161106110001838417D63
:10A14000491C417510BD10B5FEF7F9FF002816D067
:10A15000994CA079012801D0042806D196482038CE
:10A16000017D491E0175FEF7BDFFA0798006800FB5
:10A1700005D0FBF733F9904A083A5165106510BDD8
:10A18000FFB587B00F00FEF7DAFF00287ED08A4DBA
:10A190002E00603E3100A8791C3106910839340048
:10A1A00040340128059101D0042832D1FBF716F97B
:10A1B0000B00316A069A07000598019003920291FC
:10A1C000B2697D4800920838416900693A0022F07E
:10A1D00087FC607D401E6075F6F72CFA754C070011
:10A1E000A078032813D1B06B002803D0FBF725FA21
:10A1F0000020B063A879012805D14002A88023205F
:10A200000EF01AFD03E0FEF7EEFE0120A07038000C
:10A210004FE0022801D0082866D10A980028B5D05E
:10A2200002F089FA002831D105F05CF80128ADD0A0
:10A23000FBF7D4F80B00316A069A84460598019022
:10A2400003920291B2695C48009208384169006942
:10A25000624622F045FC207D401E20750120002F23
:10A2600000D00020554908700998002801D0002F1F
:10A2700064D000200990F6F7DDF94E4CFCFD76879E
:10A2800001000000609F000000040000B1FAC0F669
:10A290000490A078032819D1B06B002805D000E005
:10A2A00025E0FBF7D4F90020B063A879022805D196
:10A2B0000002A88023200EF0C9FC03E0FEF79DFEFB
:10A2C0000120A0700498F6F7C4F941E00498F6F76D
:10A2D000C0F90EF023FF00283AD03E48006800285D
:10A2E00036D126F052FF002802D0FEF705FF2FE0FE
:10A2F000002F2DD007980CF01EFE29E0364C80066A
:10A30000800F25D0B669F517FBF772F82700483F94
:10A310003A697B69801A99412B00321A8B411AD213
:10A32000A07D401C0006000E0A28A07508D326490F
:10A33000086D401C08650020210020390863A075C5
:10A34000FBF756F838637963386479647965386562
:10A3500009980BB0F0BD0020F1E710B5FEF7F9FE4B
:10A36000002804D0194901208988012900D1002042
:10A3700010BD164830218079084070471348808806
:10A38000000A0002704770B504000D00F6F75CF992
:10A390000600FEF7DEFE002824D00C49887920282C
:10A3A00020D1C87901281DD1002C19D0002D17D03B
:10A3B0000A4802685830824214D10120C0028880C5
:10A3C00023200EF043FC0DE0486605008082050066
:10A3D000036905006C690500C0820500D04C0004CB
:10A3E000FEF73BFE3000F6F734F970BD38B5214C6E
:10A3F000606CFBF72CF90822230000921E48E26AE9
:10A4000044330021FBF7D1F8FAF7F2FF220058326B
:10A410009062D1625163106338BD10B5154CA06CC9
:10A42000FBF715F90020A06410BD10B5114CE06CCD
:10A43000FBF70DF90020E06410BD104A506B010CD1
:10A440000C4809042838C08C014351630B4AC03AB8
:10A45000116B0904090C000408431063704710B520
:10A46000044C206C002803D0FBF7F1F80020206496
:10A4700010BD000020820500C98E0000C0A700802A
:10A4800010B5F6F7E1F8FF494A6A002A03D0F6F75B
:10A49000E0F8012010BD01224A62F6F7DAF8002048
:10A4A00010BDF94B586B020CF8481204C1680A43FE
:10A4B0005A63426809040A43F349C0390A630168D0
:10A4C00064390162002181621E2281614262C161A0
:10A4D0007047EC4910B58A6A824215D10020087095
:10A4E0008862FFF7DEFFEA480068002801D01720E5
:10A4F00008E00CF0DBFC002803D10CF03BFD002849
:10A5000002D022200EF0A2FB10BD38B5DD4CA06AAF
:10A51000FBF79DF8082223000092DE48E26A002142
:10A520002833FBF742F838BD70B5F6F78DF8060012
:10A53000D94801694069814201D0012400E000242A
:10A54000D04D2878697808431BD03000F6F781F8A1
:10A550006878002813D0002C0CD0686B0722401CB0
:10A560006863CE4801210068FAF778FE22200EF0D9
:10A570006DFB04E0A86B401CA8630120A8700120BB
:10A5800070BD04F0EEFE002808D13000F6F761F847
:10A59000E86B401CE863FFF7B8FFF0E72878401C41
:10A5A00028703000F6F755F8002070BD10B5F6F7AA
:10A5B0004BF8B4490A788B68896A1A430A4303D076
:10A5C000F6F747F8012010BDF6F743F8002010BD5C
:10A5D000AC4910B54A6982420ED1AB48C038C26856
:10A5E00002231A43C2600020486102F0AEF800283E
:10A5F00002D022200EF02AFB10BDF8B5A849096A46
:10A60000A04D0C07A968240F814231D10020286198
:10A610001AF001F89C4E9C4FC03E403F00280CD0E1
:10A62000F06880071FD5F86A400003D5052C1AD0C2
:10A63000062C18D00120286115E019F0F2FF00283F
:10A6400003D119F0FAFF00280DD0F06880070AD571
:10A65000F86A400007D52879E978884201D20121BB
:10A660002961401C28710020A86021200EF0EEFA1C
:10A67000F8BD38B5834CA068FAF7E9FF082223003B
:10A6800000928848E26800210833FAF708FF834106
:10A69000010000005CA3000000040000996B454B22
:10A6A0008EFF38BD10B5040026F079FD002825D0B6
:10A6B000FFF786FF002821D122F078F8002803D088
:10A6C0000CF062FC002801D1002C17D022F06CF8AD
:10A6D000714A0021002812D0002C06D1FFF72EFF6E
:10A6E00000280BD1FFF71BFF06E01171FFF7D2FE28
:10A6F000002803D1FFF7DFFE26F0B1FD10BD002CCE
:10A7000006D1FFF71BFF0028F8D1FFF708FF00E094
:10A710001171FFF7B8FF10BD5F49CA69824204D1C9
:10A720000020C86148620120BCE7704738B55A4C28
:10A73000E069FAF796FF0822230000925F48226A38
:10A7400000211C33FAF73BFF38BD10B5524CE069CD
:10A75000FAF787FF0020E06110BD10B54E4CA068ED
:10A76000FAF77FFF0020A06010BD38B5F9F7BCFBF9
:10A770004949002803D052488069448800E08C6928
:10A780004869FAF76EFF444B082200924D482200B8
:10A7900000211433FAF713FF38BD10B53E4C606941
:10A7A000FAF75FFF0020606110BD10B53A4CA06A57
:10A7B000FAF757FF0020A06210BDFEB50A21040081
:10A7C00001AA06F0ACFB344E00250028009062D0B0
:10A7D000FF209130005B0321890308430199096E32
:10A7E0008880200026F0EFFB0199374A88708A6044
:10A7F000364A127E920603D4002801D0344888607D
:10A8000021F0D2FF00282AD12A48006A234F0407EA
:10A81000240FC03FF86880070CD51CF0A4FA00286C
:10A8200008D01E484038C06A400003D5052CF1D03E
:10A83000062CEFD026F0CFFC002809D000984AF073
:10A84000D6E8F5F70BFF164935708D61CD6121E033
:10A85000F86802218843F860FFF787FF0AE01D4C83
:10A8600002E002201BF000FF26F0ADFC002801D121
:10A87000641EF6D2FFF753FE01207070009826F098
:10A88000BDFA00282CD100984AF0B0E8F5F7E6FEB2
:10A890003570757020E025E010670500C0A70080C6
:10A8A000F08205006C690500A3A1000000A00080F3
:10A8B000A06C050000000190CBA20000D5A3000011
:10A8C000B87E0500A1A20000020400001067000489
:10A8D0000204004070170000F5F7C5FE0020FEBD21
:10A8E0000120FEBDF5F7BAFE3570D3E7FF4870B51D
:10A8F000006AFF4E0407FE4D240F8036E86880078B
:10A900000AD51CF030FA002806D0F06A400003D5C2
:10A91000052CF3D0062CF1D0E86802218843E860CA
:10A92000FFF723FF26F09BFC70BDF8B50C00060076
:10A9300015001F0001F013FF002836D10CF024FB96
:10A94000002832D004F0E2FC01282ED0002F2CD0B9
:10A950000120002C00D00020E649087021F08DFF76
:10A96000012808D1FFF721FFF5F778FEE24A002120
:10A970001170F5F778FE0EF0DBFB002815D0DF48EC
:10A980000068002811D126F00AFC002803D000201E
:10A99000FFF788FE08E0002C07D0D948007800288F
:10A9A00003D130000CF0D1FA00252800F8BDD548BD
:10A9B000C16BD54A1143C16370471CB519F035FE10
:10A9C000002804D0694601A819F01FFE03E0CF4813
:10A9D0000190CF480090CF4CC749E068096B401AFE
:10A9E000A0600CF0D1FA002803D0A068FF38F53839
:10A9F000A060E1680198814203D12169009A9142E7
:10AA00000FD0E0600099421A22604B22D2002161EF
:10AA10008918C14A8018814200D801006160FFF79F
:10AA20004AFD1CBD70B5F5F719FE0600FFF7BDFE27
:10AA3000B14C00252570657026F01EF9032801D160
:10AA4000B64801E07D20C0002063FFF7B6FF26F086
:10AA500054FB21F0A9FE002809D0FFF776FEA44898
:10AA60006562C030416B42061143416309E0FFF764
:10AA700074FEFFF792FE9E492561C86802221043CA
:10AA8000C8603000F5F7EFFD70BD70B5FEF76BFBE9
:10AA9000002827D121F0F1FE012823D1D8434861B5
:10AAA0000100000058A7000000040000CAB196276A
:10AAB00021F084FE954E9C4C002500280AD0FFF71B
:10AAC0007EFEF5F7D5FD8F49C0314A6B4B061A4320
:10AAD0004A630CE0FFF74BFEFFF769FEFFF76FFEDE
:10AAE000F5F7C6FD8749CA6802231A43CA60357064
:10AAF000A561E561F5F7C1FD70BD8B4AD368181AF1
:10AB0000401A51680004000C814202D891688142C9
:10AB100001D20804000C7B4A116B090C09040143A3
:10AB200011637047F0B5040085B0FEF726FB0028DE
:10AB300064D121F0ACFE012860D101F01AFE00289A
:10AB40005CD10CF0C7F9002801D0FFF738FE21F0E6
:10AB500035FE00283CD00CF0BDF9002807D10CF0E0
:10AB60001DFA00282AD02034207EC00626D56E4C3F
:10AB7000A76A256AFAF750FC236822000E002832E3
:10AB80008446590810000093083801AB07C333000E
:10AB9000E169A069624621F0C1FF606A002807D020
:10ABA000A26A216A8918EA19914201DA401E04E07A
:10ABB000A16A206AFFF7A1FF1E206062F5F758FD29
:10ABC00004005048C030416B42061143416309E024
:10ABD000FFF7EDFDF5F74CFD4A490400C868022275
:10ABE0001043C8600CF076F9002804D047490020D3
:10ABF000087026F03EFB2000F5F73FFD05B0F0BDE4
:10AC000070B50500484C0026E169A06971407040AC
:10AC100008430FD0A269E3693100A81A994109D20B
:10AC20003A49086C401C0864A269E369501BB341AF
:10AC3000E361A06170BD70B5040034480D00007878
:10AC400000280AD0FAF7E8FB374AD1619061290061
:10AC5000200015F028FBFFF7D3FF70BDF7B582B0D9
:10AC60000D001600F9F74AF900280CD021F0A8FDD4
:10AC7000002817D0002D70D06C20405D062811D818
:10AC80000428F6D011E021F0CAFD00280BD021F0F5
:10AC900095FD002807D0286E80780007800F02D12C
:10ACA000FFF74EFDFBE0002DE5D030690028E2D033
:10ACB000286E80780007800F02280BD101F059FD23
:10ACC000002807D10CF06AF9002803D021F078FDA4
:10ACD00000280CD121F0A3FD002804D0286E807834
:10ACE0000007800F03D0F9F709F90028DAD01148DE
:10ACF00007681148007800020743F5F7B9FC1DE02A
:10AD00000000019000A7008003690500106705009E
:10AD10006C69050004690500C0A200801000008075
:10AD2000A60E0000E2040000F082050048F4FFFFD8
:10AD3000EE02000000A00080945601C001908348FC
:10AD4000346800781434810081484058010605D0E9
:10AD50000006000E001F384302E09CE0FC20384350
:10AD60000068A04276D1F9F7C9F8002831D0002058
:10AD7000F07560880007000F01282FD031686068E7
:10AD800060318A7B801C521E1206120E8A737ED09E
:10AD90004178090714D401780A07920F022A02D1D8
:10ADA000090908290CD06B49096B01220909D20253
:10ADB00089180A0161680B8B1B071B0F13430B8358
:10ADC000417808221143417002982100F9F766F991
:10ADD00004E030686030817B491E817330686030E8
:10ADE000807B002853D0F07D002850D1FC203843D0
:10ADF0000668380004210843FC22390049F04CE978
:10AE00003E6052485449007880000A58521C0A504B
:10AE100052490A58121D0A50F9F770F8002804D157
:10AE200060680822C1781143C17001202070F9F7D1
:10AE300065F8002804D0F9F76DF8F9F7A8FA21E0D1
:10AE400021F0BCFC002806D04548416B4206114366
:10AE5000416308E01BE0FFF7AAFC3E494031C868A7
:10AE600002221043C860FFF7AAFC3E490020087088
:10AE7000286E80780007800F01D1012000E00020BB
:10AE8000FFF71AFC0198F5F7F8FB0120B6E60198E8
:10AE9000F5F7F3FB03E002983100FFF7CCFE00204A
:10AEA000ACE670B505002F4C21290DD007635785FE
:10AEB0000100000054AB0000000400003EDEE393FC
:10AEC000222910D101F05FFC002842D10CF00CF8CF
:10AED00000282ED06078002828D122E0206901289F
:10AEE00002D1FFF7E4FB70BD01F04DFC002803D157
:10AEF0000CF05EF8002802D0FFF70CFD70BD0BF0DF
:10AF0000F3FF0028FAD0FFF72DFB0028F6D1280028
:10AF1000FFF767FC012804D149F018EE174A03C275
:10AF200070BD002128000BF0FEFF70BDFFF70BFB8A
:10AF300070BD0CF03DF80028FAD026F044F9002846
:10AF400003D00020FFF7C2FB70BD28000CF011F801
:10AF500070BD0120F6E708490020487070470000E6
:10AF6000945601C0107902C0C0A60080F47802C0D7
:10AF70002C7902C0C0A70080106705008869050011
:10AF80000022662110B5FF48006849F03CED00281A
:10AF900000D0012010BD10B502F044FB002805D000
:10AFA00001F01CFC002801D0012010BD002010BDC4
:10AFB00010B525F034FE10BD10B50C008968CA002C
:10AFC00010D5012212079143A1602178012249077F
:10AFD000490F14F08FFA0101206E028B1207120F35
:10AFE0000A43028310BD10B50C001100FFF7E4FF07
:10AFF00021F051FC00281ED0200022F06FFC200020
:10B0000026F02DF9002811D0F8F782FF002802D091
:10B01000F9F7C7F908E00BF0CBFF002802D00020B9
:10B02000FFF754FBFEF786F8012010BD200022F048
:10B030006EFC002010BD200025F0D7FE10BD0100E1
:10B04000D14810B580680722FAF726F9002010BD14
:10B05000F1B582B0CC4C606A401C6062FAF7E6F948
:10B06000CA4F0090FE6A0D00C948F862210002989C
:10B070001E221831FBF704F9002802D0606B401C37
:10B080006063FE62C34880692062FAF7CFF9009AD4
:10B09000276B861AA9410D007A1C0020E06A216BFB
:10B0A0000023484300218019694149F028EDE062FE
:10B0B000206B401C2063A06A0021801BA94100D3A3
:10B0C000A66AA662A069E169884201D9A06900E088
:10B0D000E069E061626BA16A112031F09DF8FEBD6C
:10B0E000F8B50700A84DFAF7A1F904000E00AA4927
:10B0F0003800FBF7B7F8FAF799F9041BA86BB141D0
:10B100000B000021001B994100D3AC6BAC63F8BD70
:10B11000A2480088002804D0A14901200978042908
:10B1200000D000207047202089E7F8B5F5F7AAFA8B
:10B13000954B00905869012700243D00002800D05D
:10B1400000250020390081405A690E00164202D1C4
:10B150000C000A435A61401C002C01D11F28F1DD6C
:10B16000002D08D049F04AED8E48FFF771FF3920D5
:10B170000001FFF7B5FF0098F5F789FA2000F8BD48
:10B1800070B50400F5F77EFA7F490500226848692A
:10B190009043486100210028216007D16F20FFF70C
:10B1A0009FFF49F030ED0120FFF749FF2800F5F738
:10B1B0006EFA70BD70B5040046690089051921F06A
:10B1C00038FB002818D0F8F7A3FE002814D1286E09
:10B1D00080780007800F0FD1200022F07FFB200035
:10B1E00026F022F8002803D00120FFF76FFA70BD87
:10B1F000200022F08CFB0EE0707A022806D100229B
:10B200003100200009F088FC002802D12000FFF75F
:10B21000CFFE0028EBD1200049F0FCEB70BD38B523
:10B220000522594C0021A068FAF736F85E4805223D
:10B2300000680021FAF730F802E0009849F0EAEBE4
:10B24000E068042200236946FAF717F80F28F4D1C2
:10B250005648002505705648122149F028EC5548FB
:10B2600025700560002038BD70B5040000890519FF
:10B27000286F00280FD0C0790007000F022804D1E2
:10B28000286E01881039018001E0032803D12000D5
:10B2900015F0AAFB70BD6669002E09D0707A0228ED
:10B2A00006D100223100200009F036FC0128F1D03F
:10B2B0002A0021003000FFF796FE0028E9A9317925
:10B2C0000100000050AF0000000400006D0430FFDA
:10B2D000EAD1200015F0C8F800212000F5F75CF94C
:10B2E00070BD7023374A5843E03A10B58418A088DF
:10B2F000E288824201D1012010BD8200A21892682A
:10B300000A601821401C49F018ECA180A06E401E74
:10B31000A066002010BD70B50C00417A160002290D
:10B320000AD109F03DFE012806D130001C38022167
:10B330000EF0CCFE01280CD0702122486143E03889
:10B340000C18E5881821681C49F0F6EBA0888842A3
:10B3500001D1012070BDA80020188660E180A06E98
:10B36000401CA066002070BDFFB587B00124160008
:10B370000898119D002874D0052E07D0062E05D000
:10B380000A485130F5F716F9F9F7B6FF2800603092
:10B3900006900673059619E02864050054670500B9
:10B3A000C0A60080FF7FFF7F40A20080FFFF00005B
:10B3B00060860500C9690500FF030000A06C050058
:10B3C000940C000414490004906C0500761F3106AB
:10B3D000090E702048438646FF4B109EC718FF2079
:10B3E000401C8840844610203B00089A88406C33FB
:10B3F0001C3E012A049364D10291F849634609690D
:10B4000062460B4234D10842039074D1F24B70462D
:10B41000185C00281FD12878002241070798490F9F
:10B4200014F072F86B46198800010907090F0143EF
:10B430000091187800090001187000990A981DF011
:10B4400019FD0698017B0A981DF029FFE34903982E
:10B450000A6910434EE00A430399E0481143016131
:10B460004EE079E00A9878700498F5F76AF90EE0F2
:10B47000DA4B07000F420CD0109A02990798FFF799
:10B480004AFF012803D130000021F5F785F8002498
:10B4900062E0914308431861029870264643CE4FFC
:10B4A00008E00198A9788170B95D1C38491CB9552C
:10B4B000FFF7E4FE029801A9FFF713FF0028F0D080
:10B4C00041E0089A022A47D10291C44963460969BA
:10B4D00062460B421CD10500084236D0BE4B704676
:10B4E000185C002808D105990A981DF0EFFEBB49A9
:10B4F0000869A843086128E0B8480A43AA430261E2
:10B50000109A02990798FFF706FF0028BBD1A9E718
:10B51000B24B07000F42AFD09143814319610298AB
:10B5200070264643AC4F08E00198A9788170B95D58
:10B530001C38491CB955FFF7A1FE029801A9FFF775
:10B54000D0FE0028F0D0002C06D00298702358437B
:10B55000A14A115C491C115420000BB0F0BDF8B594
:10B5600005002F0000895419401900901C202E1846
:10B570007C37002928811ED060782178000208439A
:10B580001E2801D91E3800E000202070000A6070DB
:10B590007421300049F094EA0098407CF87368699F
:10B5A000007A032803D005F0D7FB012801D105203C
:10B5B00000E00020B070E078FB210840E070607E81
:10B5C000217E000208430007000F2076000A607603
:10B5D000207E072100090001207630780843307072
:10B5E000092034663873280024F002FB002802D1B9
:10B5F0002800FFF7E9FDF8BD70B5794849F078EA11
:10B6000004001FD0208905196978287812F07EFB84
:10B61000002810D0606168792A79218900021043DE
:10B6200008180204120C01212000FFF798FF0120E6
:10B63000FFF70FFD02E0200049F0F6E969490868CC
:10B64000401C086070BD6448702110B549F038EAAC
:10B6500062490020086110BDF0B50026CBB034006F
:10B6600011960E96FFF7EFFF5B48E8304A90C12035
:10B670008002F4F79FFF0022D243584F00925A49AC
:10B68000B868082241ABF9F715FE5848F4F792FF65
:10B6900041980028EBD0400607D5002012F0C8F8EA
:10B6A000534841684206114341604198C0060AD59B
:10B6B00012F004F94F48072200681021F9F7F6FD4F
:10B6C00039200DF0EBFA4198000601D58E8BFBC0B6
:10B6D000010000004CB3000000040000D2C1154C72
:10B6E00022F070FF4198C00501D522F061FF41981A
:10B6F000810602D5454A00211170400701D5F6F7B1
:10B700005CFB4198800711D533F039FE0128B8D091
:10B7100004E01398B0220021FFF72BFFF868042201
:10B72000002313A9F9F7BDFD0F28F2D14198092193
:10B73000084275D0364801682F480068814201D020
:10B74000FFF764FF13F026FD00289AD078690028DF
:10B7500097D1FFF7F1FC002893D133F010FE0128B8
:10B760008FD038698005800F6FD00025FF20204AD8
:10B77000401CA840116903000B4267D070276F433B
:10B780001A4BDB5D002B61D181431020A840084299
:10B7900011615CD01F4920480EF0ECFC13490020D9
:10B7A0001E4A7918499118214143535C002B41D01E
:10B7B000499B891889785B7899423BD11823584373
:10B7C00080184890001D13F020FB030048980022C9
:10B7D0004178180013F0A2FE6B46998E000109070C
:10B7E000090F014308AB0D91187D1AE0344800049D
:10B7F00054670500244B0004A0670500FF09000002
:10B800000404030040A50080B86D0500C969050067
:10B810009467050011111111BBBBBBBB2849000483
:10B820008DE300090001187549980D9940781DF0C5
:10B830002BFB02E0401C0228B5D3681D0106499885
:10B84000090E40781DF035FD1AE023E01EE0F949AD
:10B85000F9480EF08FFC681D0106F848090E3818EB
:10B8600040781DF03DFD0BE0F549F3480EF082FCF9
:10B8700044981C38FFF70CFDF049C85D401CC855C2
:10B88000280044A9FFF737FD0028EDD06D1C022DDC
:10B8900000DA6BE7002E71D000200C900B90E9A02D
:10B8A00003C8099006200890E8480A910168E84812
:10B8B0000068814201D0FFF7A9FE30891222851964
:10B8C000DE482900E03049F0EEE868792979000285
:10B8D000DA4F08434019E0370D90387800281BD123
:10B8E000797812F01DFA0400007A012806D10D982B
:10B8F00013F08BFA00283BD0040040E0002837D139
:10B90000787BC00634D50D9813F07FFA00282FD02D
:10B91000417BC906F0D42BE0012801D0022827D1B1
:10B92000797812F0FDF9040024D0607A022826D13B
:10B930000D980078C0070ED0200012F031FB0028CF
:10B940000E901CD00E980B2189014018C06B002866
:10B9500015D100240EE00D9813F057FA040012F0F0
:10B960008EF9002C06D0603000780328F1D106E073
:10B97000002C04D100213000F4F718FEE0E2B549B4
:10B9800001207461087004F0F8FF78887D21890136
:10B99000884201D3F9F7BAFC16A87421159049F032
:10B9A0009AE8787BC00726D000F0EBFB0BF064F838
:10B9B000002819D0A8480078002815D120F071FF80
:10B9C00000280FD0200014F071FB00220121019209
:10B9D0000091797B02000907CB0F0121200000F0C4
:10B9E000D4FC01E0FEF7AEFB0BF030F80028C1D02C
:10B9F0000CF0CDFABEE7207A012804D0617A022942
:10BA000001D0062804D10D99200013F075FD02E045
:10BA1000200014F0DBFB15982B951430339039A8D7
:10BA20001C9015983490207A012804D0617A02295C
:10BA300001D0062804D10D99200013F05DFD02E02D
:10BA4000200014F0C3FB1290129A0092B8887B4930
:10BA500043191C9AE031200000F0AEFBF988E6297A
:10BA600001D1002000E00C207A8830AB121A1A8332
:10BA7000BA8828181018E629359001D100200890BE
:10BA800008AA09A936A86B4607C30BAA6B4D3599BE
:10BA9000E035E88814AB1CF0F5F90700002030AB66
:10BAA000D876287B082802D3002029000873607A02
:10BAB000032801D001280CD1200014F087FB0028B6
:10BAC00007D05E4D2000E035297B14F068FC287318
:10BAD00016E0207A012804D1200014F06BA203069E
:10BAE0000100000048B7000000040000811BC620D0
:10BAF00077FB002805D1607A022802D0207A062838
:10BB00000AD10D99200013F001FD002804D05048FF
:10BB1000E030007B30ABD876002F0AD0200025F033
:10BB200084FA400620AB998A800D7F22D20091438F
:10BB30000BE03820005D0025FE280BD020AB998A51
:10BB40007F22D20091434006800D014320AB0125A6
:10BB5000998211E02000FF30A1301EF019FC20ABCB
:10BB6000998A7F224006D200800D91430143998239
:10BB70001C988079C0072AD0229801210903084324
:10BB800022901C988079C00721D02298091108437F
:10BB9000202188432290607A02280AD10E98C07F23
:10BBA000002802D049F028E808E0200025F050FAEB
:10BBB00004E0002D0BD1200025F037FA400620AB21
:10BBC000998A800D7F22D20091430143998220AB54
:10BBD000988A8105490E032908D82549097F8906D5
:10BBE00004D57F21C900884328309882204901204C
:10BBF0002031097EC9060AD4617A022906D10E9A3B
:10BC00000321090251180979090700D400200F9077
:10BC1000207A00282ED1200020304790807E000717
:10BC200028D420AB988A8005400E49F00EE8050024
:10BC3000122049F00AE885421CD84798807E800788
:10BC4000C20F01211BE0000022222222BBBBBBBB92
:10BC50003448000433333333AAAA03000000000041
:10BC600094670500A0670500940C000404690500B2
:10BC7000F06600043A20005D0F998007C20F3398E8
:10BC8000FAF795F81C99FA48FA4B007B891D10AA1F
:10BC9000F9F76DFF00281BD020AB988A8005400E75
:10BCA0002FF00AFB002805D0F349C8430EF06CFAC8
:10BCB000012505E0F048F149C0430EF065FA022580
:10BCC000349801218068090708433499886015E099
:10BCD000E948EB49C0430EF057FA129800250028B6
:10BCE0000CD030ABD97E0122200013F021FC30AB08
:10BCF000198C00010907090F014319841C203081A8
:10BD000030184390159808AB4290187B089A079218
:10BD100009A9129A06910CA90590D548029503919C
:10BD20000492C08811990206120E019200913B0004
:10BD3000310014AA34A820F059FF20AB449046905B
:10BD4000D88910ABD8831498002800D01CE64698F8
:10BD50000028FBD04A9848F0C4EE420920AB988AEC
:10BD600010218005400E4590084352014A99104326
:10BD700048F05CEA01000C98002800D03290469808
:10BD80002E90002030AB19911871459810AB987621
:10BD90002E9830AB008B198C00070909000F0901A0
:10BDA00008432E9908832E9880780009082810D11E
:10BDB0004A9848F096EEAE490122C988E62900D09B
:10BDC00000220092020030ABDB7E42993398F9F7F3
:10BDD000C6FF607A032801D001280AD1A448817BDC
:10BDE000027B4B004299200014F0F3FA0028ADD0FA
:10BDF0001BE0217A012903D0022801D0062914D1A1
:10BE0000129800280DD0002D07D0429910AB994A06
:10BE100018786C31F9F733FF07E09548007BFCF7A1
:10BE2000F0FCFCF7FFFC30AB1871002F09D1207A31
:10BE3000002802D0607A03280DD12FF0F8FE0028E8
:10BE400009D0904810AB012D988304D019980E2189
:10BE5000F9F7A4FF19903399429824F068FF012D57
:10BE600011D185488849C0430EF08EF910AB814945
:10BE70001878F9F71EFD22986907084322900A20D6
:10BE800018AB18730AE080497B48C943C0430EF0E1
:10BE90007BF9339A4299200024F0CEFD7448407B10
:10BEA000000706D500F077F922980121C907084359
:10BEB00022902299189810AB08431890188F188573
:10BEC000588F5885339A4299200024F00AFF22980F
:10BED00010AB000100092290188B20AB9881439889
:10BEE000429974222C9048F010EE634F2A8C84DC27
:10BEF0000100000044BB0000000400007574B3940E
:10BF00006449FF43C94338000EF048F918993800D6
:10BF10000EF044F930AB197938000EF03FF9429930
:10BF2000439A019130AB00921A7910AB1B7829002B
:10BF30002000FFF737FA002816D03000FFF7BCF9D1
:10BF4000002603F0CDF800280ED0FFF741F80028B6
:10BF50000AD10420FFF79BF801F08CFB002819D0D0
:10BF60000120FFF794F815E041980821084202D01B
:10BF700022F00DF80BE04A4848F0D8ED002804D133
:10BF8000484848F0D4ED002801D004210173060090
:10BF900000D095E4444900200870FFF786FB401F5D
:10BFA00010B50406240E022C14D2702035496043CB
:10BFB000E0394018702148F0A2ED3C4A0120116997
:10BFC000A04008431021A1400143FF20401CA04095
:10BFD0008143116110BDF8B5441F022C25D2F4F73E
:10BFE00079FB0600314DFF20401C2969A040084222
:10BFF0000AD003E000981C38FFF75EF9200069467C
:10C00000FFF78DF90028F5D0FF2112312869A140F2
:10C010008843286170201B496043E0394018702133
:10C0200048F06CED3000F4F75AFBF8BDF8B5441F4A
:10C03000022C26D2F4F74EFB06001C4DFF20401CBC
:10C040002969A04008420BD004E0009800211C3868
:10C05000F4F7C0FA20006946FFF761F90028F4D030
:10C06000FF2112312869A1408843286170200549C9
:10C070006043E0394018702148F040ED3000F4F79B
:10C080002EFBF8BD144900042849000444444444EC
:10C090005555555566666666FF7F0000777777775A
:10C0A000FC4A0004E84A0004940C000454670500AC
:10C0B000F8B500242500424EFF277F1C7020604306
:10C0C0004049355438000969A040084202D0012097
:10C0D000FEF7DDFF641C022CF0DBD2E7F8B50400AC
:10C0E0000D000026052801D0062C33D1354A601FEB
:10C0F00001211769814039422CD070214143304AD7
:10C10000535C002B01D05B1E5354FF235B1C834008
:10C110003B4205D0505C002802D10120FEF7B7FF5A
:10C12000002D17D02869002814D0274A0020182194
:10C13000414389180B00C9780A33A14207D1286806
:10C14000006E008B0009401C0126188002E0401C94
:10C150000228ECDB300094E7F1B582B0F4F7BAFACC
:10C1600000901A491A480EF019F8FFF706F80190E6
:10C17000029814F04CFB174F0024260001202506DE
:10C1800038602D0E0299280023F0A7FF029928009D
:10C1900024F059F8641C042C3E60EFDB01A8FFF783
:10C1A00017F80098F4F79BFAFEBD0B4800880028AA
:10C1B00005D00A480178032901D104210170704794
:10C1C0003448000454670500284900041111FFFF9A
:10C1D000BBBBBBBB2865050060860500C9690500BF
:10C1E000FFB583B0040016000F00911C0C980022CC
:10C1F0000291130069460CC10122F979BB79090249
:10C200001943E92900D00022797BC907C90FF9F742
:10C2100049FE0500F879B97900020843EA2803D1FC
:10C22000797B082211437973312109016218237A3D
:10C23000012721003F039C31012B18D0062B1CD174
:10C240000B0006993000F9F7FEFD1B204001201875
:10C250000088002800D100273D430298062205806F
:10C2600030001A30694648F032EC07B0F0BD0B00E0
:10C2700006993000F9F7E7FD23E0637A022B15D128
:10C28000069B0A0006999B1D3000F9F7DCFD012092
:10C2900040020543B079C007DFD10221200006F03B
:10C2A000A7FB0128D9D140030543D6E7E62801D1F1
:10C2B0000B0000E0069B3000F9F7C5FDFF20401C95
:10C2C0000543FF4800680079C3E7FE490020886005
:10C2D0007047F3B581B00600FA4CA06800285DD124
:10C2E0000298FDF7FDFE002858D0FF21F6480022F5
:10C2F0002D3148F0E4EB050050D00120B80A14D0ED
:10C300000100000040BF00000004000026AE60F8FD
:10C310000221A06029736E61697B0143F048697353
:10C32000A861B0202881FF209130825BE94800920B
:10C330000068320003793120000131189C32280056
:10C34000F9F763FD07001C202C18288174212000B8
:10C3500048F0DEEB3000276624F07BFEA070E14859
:10C36000A06020F083FA002804D1A068012109030D
:10C370000843A060DC48007E800607D4A07800282F
:10C3800004D0A068012189070843A060FCF731FFB1
:10C39000002802D0FDF719FF00E00320603420736D
:10C3A000280024F071FD002804D1280048F064EB37
:10C3B0000020FEBD0298FDF70CFF0120FEBDC6491E
:10C3C0000020C8607047FFB585B0070005D0002188
:10C3D000380032F0A9FE002802D1002009B0F0BDDB
:10C3E0000898002819D0BC48C168002915D0BF4959
:10C3F0000A6949698A420BD041680722491C416099
:10C40000BB4801210068F8F779FF22200CF06EFC90
:10C4100010E10120F8F716FF01E0FF242D34210080
:10C42000380004F0A3FD0500F3D028894619380030
:10C4300013F0EAFE002801D00C2000E00420312196
:10C440000290387A09013A0079189C320628019244
:10C4500000910AD11300029AEE3302213000F9F75D
:10C4600011FDF0784008400008E01300029A022114
:10C470003000F9F707FDF07801210843F070F178FA
:10C48000EF20014006982C00C007C00F0490000167
:10C490000143FF20F170C01C3071000A7071002050
:10C4A000307070701C20288102201C342873742185
:10C4B000200048F02EEB200060300F99039041736C
:10C4C0002666089800280AD00120C007A06082488C
:10C4D0000121C160687B084368738648A861002019
:10C4E000208002980C281FD10799380013F075FF9F
:10C4F00041072078490FC008C00008434107207059
:10C50000490F380014F0BCF80101206E028B1207AD
:10C51000120F0A430283206E017E09090901017688
:10C5200020789F2108402070079A210038000023BE
:10C5300013F063FF0E986C4E002821D1FDF706FE24
:10C54000002807D00698002804D003990720087314
:10C5500009200EE00298042805D118F0ACF8002854
:10C5600001D0072000E0042003990873380024F06C
:10C5700070FDA070A068012109030843A0601EE0BF
:10C58000002138002EF0B7FE0328A07017D9307EA6
:10C59000C00604D554486030807A40060AD5787ABF
:10C5A00002280CD1032000023918896A0818007982
:10C5B000000704D50321380024F011FDD9E7307EAF
:10C5C000800607D4A078002804D0A068012189073C
:10C5D0000843A06020F091F9002811D00E9800289F
:10C5E0000ED0280021F0ACF9280024F06AFE0028C3
:10C5F00002D020F0A2F91DE0280021F0BAF913E0E2
:10C60000380032F08AFE002809D0380011F0DAFC38
:10C61000816904229143049A9200114381612800A8
:10C6200024F032FC002805D1280013F045FF280033
:10C6300048F022EA0120D1E6FFB5FF212D310600A6
:10C6400085B004F093FC070001D10120C6E630005C
:10C65000FF30317A8B300129049002D0707A0228A1
:10C6600004D10499300012F065FF02E0300013F0AD
:10C67000CBFD6B46197EF322114008310028197654
:10C6800003D00807000FC03002E00807000F403059
:10C690006B46187638893200C519312000019C326A
:10C6A0003118019200911C7E049B20092107020091
:10C6B0000390890F2800F9F7E5FBFF20C01C2871C3
:10C6C000054A000A687150880101401C5080687E4C
:10C6D0002A7E11E0986D0500583601C0480D00040F
:10C6E0000FBF0000020400001067000400A00080DB
:10C6F000A06C0500EFBF0000000210430007000F10
:10C7000008432876000A68766B46AC70630206160A
:10C71000010000003CC30000000400002457B8EEF4
:10C72000587EE870707A02280DD10221300006F0A0
:10C7300073F9E9788A06D20F1043C007DF22800E12
:10C7400011400143E9701C2038813C183800FD6716
:10C7500008997C3041730E99017303980C2823D1FA
:10C760006B46988B2080707A03281DD1300013F01F
:10C77000C5FC0100300013F03AFE41072078490F54
:10C78000C008C000084341072070490F300013F073
:10C7900081FF0101206E028B1207120F0A430283F0
:10C7A00020789F2108402070002130002EF0ADFD40
:10C7B000A070380024F072FB012803D0380048F044
:10C7C00066E94CE7002013E60200744810B50068E3
:10C7D00004210023F8F789FD002804D10220FEF788
:10C7E0006AFC002010BD012010BD6D490968087168
:10C7F0006C49486170476A4800680079704710B515
:10C800000CF0D1F9002801D1012010BD002010BD8D
:10C81000654870B50124006B400713D524F04EFF26
:10C82000624D00212E1F0AE0CA0053191B6892199D
:10C830001268934200D00024491C012C08D1814287
:10C84000F2D905E05A48816AC06A814200D00024CA
:10C85000200070BD10B5FFF7DBFF002801D0F9F70D
:10C8600075FA10BD534870B5007800283BD1524886
:10C8700000220068082148F002E9002833D1FFF7C0
:10C88000E9FF00282FD04D4848F0C8E904004B4884
:10C89000082148F0FCE905004848102148F0F6E975
:10C8A000281884421FD1464848F0B8E9040044489B
:10C8B000082148F0ECE905004148102148F0E6E97C
:10C8C000281884420FD13F4848F0A8E904003D48A9
:10C8D000082148F0DCE905003A48102148F0D6E983
:10C8E0002818844201D0002070BD012070BD70B5B1
:10C8F000012012F050FC00284ED1334C2D4D2E4E0D
:10C9000008E02078401C20700120FEF7D4FB0120B5
:10C91000F8F7A2FC28780028F3D13068002208211B
:10C9200048F0ACE80028ECD102E00120F8F794FCD4
:10C93000FFF790FF0028F8D0204848F070E9040085
:10C940001E48082148F0A2E905001C48102148F0C3
:10C950009EE928188442E8D1194848F060E90400AB
:10C960001748082148F092E905001548102148F0C1
:10C970008EE928188442D8D1124848F050E90400C2
:10C980001048082148F082E905000E48102148F0BF
:10C990007EE928188442C8D170BD00006067050098
:10C9A000986D050040A6008040A3008034A9008057
:10C9B00000A00080940C0004286405000C0D000405
:10C9C000480D0004D80D0004583601C0FF30A130D6
:10C9D0000E2210B51DF093FC10BD70B505000C00C3
:10C9E0001600F3F78BFE00212560A171E671083473
:10C9F0000A0006C4F3F787FE012070BD10B50400DD
:10CA00000C235843F549401800210A000B000EC0C2
:10CA1000200048F040E9200048F040E9200048F0BC
:10CA200042E910BDF7B584B015000400EC4A0020BF
:10CA3000009203900598290003AA02ABF9F74EF97A
:10CA40006B46187B052801D0062850D12D062D0EE7
:10CA50002800FBF7F4FEFBF703FF0600607A0328CB
:10CA600006D16B461B7A32002900200013F055FBDB
:10CA7000F3F744FE0700FEF794FBD8496B4601909C
:10CA8000D84A187B3839F9F7CAF86B46197B187AF7
:10CA90001CF082FB6B46187BFFF7B1FA6B46187BE4
:10CAA0002A003100230013F0AAFF6B46197A3000E8
:10CAB0001CF0A0FA6B46187B310023F08DFB6B460F
:10CAC000187B310023F0A0FB01A8FEF795FB38008E
:10CAD000F3F719FE6B46197A059A200025F0DCFE63
:10CAE0006B46187AFFF78AFF012007B0F0BD0020DF
:10CAF000FBE7F0B585B014000600B94A0F0000202E
:10CB0000009203902100380003AA02ABF9F7E6F87F
:10CB1000B64DB54928000DF055FB6B46840557808E
:10CB20000100000038C7000000040000778D6B8210
:10CB3000187B052801D006283FD1B24928000DF006
:10CB40004BFB2006000EFBF784FEFBF793FEF3F78A
:10CB5000DFFD0400FEF72FFBA5496B460190A64AB6
:10CB6000187B3839F9F765F86B46197B187A1CF091
:10CB70001DFB6B46187BFFF777FA300013F065FE5C
:10CB80006B46187A1CF0CDFA6B46187B002123F017
:10CB9000C2FA6B46187B002123F073FB01A8FEF755
:10CBA00035FB2000F3F7B9FD6B46197A3A003000E7
:10CBB00025F07CFE012005B0F0BD0020FBE7F8B5B4
:10CBC0000D0006000024F3F7A3FD8A4A070029069A
:10CBD000090E30323000F8F7BDFE0A280DD2854A22
:10CBE00000210001303211548018C160290030004A
:10CBF0001CF0FDFB12F053FA01243800F3F78DFD11
:10CC00002000F8BDF0B505000C00087885B00007DD
:10CC1000400F12D1784802AA03A9F9F73FF801287A
:10CC20000BD003986B460206187A120E0106090E05
:10CC300020001CF089F9002801D10020BBE70398EF
:10CC400022000106090E1432280025F018FE6B465A
:10CC5000187A1CF058FB08206B4618561CF044FB51
:10CC600008206B461856624B01218200383B9950D0
:10CC70000306604A0398009202061B0E120E210062
:10CC80002800F8F705FF6B46187AFFF7A6F9201D74
:10CC900047F04EEF0006000EFBF7DBFDFBF7EAFD69
:10CCA0000700687A03280FD1201D47F042EF0106E4
:10CCB00003986B460606187A360E0206090E120E07
:10CCC0003300280013F033FAF3F722FD0600FEF7D5
:10CCD00072FA0190201D47F02CEF02066B46187A7D
:10CCE000120E0106090E2B00380013F092FE201DD3
:10CCF00047F01EEF02066B46187A2B00FF338B338A
:10CD0000120E1D00390023F07AFA201D47F010EFB3
:10CD100002066B46187A120E2B00390023F038FBFE
:10CD200001A8FEF773FA3000F3F7F7FC012042E7A1
:10CD3000F8B500252F4F18206843395C002927D00B
:10CD4000C419201D12F093F8060021D0617800224A
:10CD5000300012F015FC6B46198800010907090F15
:10CD6000014300911878000900011870A07800991B
:10CD70001CF0BCF86B461988200009090C30618151
:10CD80000021821E030021736178300022F0DCFC58
:10CD90006D1C2D062D0E022DCDD3F8BD70B50500EE
:10CDA0000C0047F086EF0C216943114B5A581218BA
:10CDB0005A50226070BD70B505000C0047F074EF4A
:10CDC0000C226A430A4951188A6812188A60226044
:10CDD00070BD70B505000C0047F06EEF0C226A4381
:10CDE000034951184A6812184A60226070BD000059
:10CDF000304A000428490004906705006666FFFF7A
:10CE0000BBBBBBBB7777FFFF30B50020FF4D0D21CB
:10CE1000040003008901691814E0E868401CE86018
:10CE20001000526B8A62002A00D1CB620279052A77
:10CE30000BD12A69521C2A618362036003710020AE
:10CE4000002C02D18A6A002AE7D130BD10B50A68E9
:10CE5000EE4B002A03D11868401C186010BD8A6A86
:10CE6000824203D05868401C586010BDE848002436
:10CE7000026A002A0FD08A4210D09A68521C9A6027
:10CE800004220A71C26A002A01D0516300E0816263
:10CE9000C1624C6310BD012201620A71006A07225F
:10CEA0008462DC4840210068F8F73CFA10BD10B5F8
:10CEB0000A68002A10D0D64A536B83420CD1106AFC
:10CEC000002809D0884207D100205063D1480722AA
:10CED00000688021F8F726FA10BDF0B5050085B08E
:10CEE00000F0C0FB002000F0CBFB04007ED0286BDC
:10CEF0002063C7480490416A491C4162216000F0E8
:10CF0000B9FB47F06AEE03910290206800272E00DB
:10CF100039002036002803D1049A01205062206095
:10CF200000232371307A6071A079717A5987195979
:10CF30000100000034CB00000004000083E21E3634
:10CF4000800889078000890F0843F321A0710840F9
:10CF5000B17A8907090F0843CF21A0710840F17AFF
:10CF60008907890E0843A0716969286959400843F7
:10CF70000DD02A6902986B690399121A8B410AD362
:10CF8000029A2869039B6969801A994102E0A8699D
:10CF9000002800D00700029A039B0021B8185941CD
:10CFA000E160A060E8692061286A6061686AA06148
:10CFB0002868E06168682062A8686062200020300C
:10CFC000417B327B490892074900D20F1143FD2271
:10CFD00041731140327B5207D20F5200114341730B
:10CFE00002218173317B090701D506218173327BD0
:10CFF0000121D20700D102210173827B230000E0CE
:10D000000AE00092894828333A002100F8F73BFBF8
:10D01000002806D1206001E000F036FB002005B0BA
:10D02000F0BD2068FBE7F8B505250E0000F032FBE7
:10D0300004007C48016AA14216D1A06A002803D0EE
:10D04000F8F773FB0020A062002E66610CD000226E
:10D05000230000927548283332002100F8F713FBB3
:10D060000325002800D104252800F8BD70B505254A
:10D0700000F010FB04006B48016AA14207D1A06ACE
:10D08000002804D0F8F751FB00200325A0622800F7
:10D0900070BDF8B50F00052600F0FCFA614C0500E4
:10D0A000216A814215D1606B002803D0F8F73DFB5F
:10D0B00000206063002F0CD05A4B002200925C4885
:10D0C00034333A002900F8F7DEFA0326002800D1AD
:10D0D00004263000F8BD70B5052500F0DBFA514C90
:10D0E000216A814207D1606B002803D0F8F71DFB4D
:10D0F000002060630325280070BD38B50120FDF7CE
:10D10000EEFF484C2C20236AC15C5A6A1868DB6920
:10D1100098470DF092F800F0AFFAF3F703FB216A9D
:10D1200005000020086000F0AFFAFFF777FE2062EC
:10D130002800F3F7FCFA25F0F6FA216A002908D056
:10D140002E20425C0B0000923A4A38482833F8F708
:10D150009AFA032038BDF8B505250F0000F09AFAB9
:10D1600004006ED0A06A0026002802D0F8F7DDFA8D
:10D17000A6622C4D286AA04261D100F07DFA207988
:10D18000022801D0032825D1267100F07DFA286AF3
:10D190002030072F07730BD0286A082F006B0FD1A0
:10D1A0001A22002104F00FF837200BF0BDFD47E0F4
:10D1B000286A1922006B002104F005F83620F4E7F4
:10D1C00027F0D9FC286A1822006B002103F0FBFF2E
:10D1D0003520EAE7012801D004282DD100F054FAC7
:10D1E000E369626A20680B21984726602671032450
:10D1F000F3F798FA0600FFF711FE28623000F3F704
:10D2000096FA296A002908D02E20425C0B00009271
:10D21000084A06482833F8F736FA2000F8BD10E02F
:10D22000D01E000410220004B86D050055CA00008D
:10D23000B7CA0000A086010000F026FA00E02660D0
:10D2400003252800EAE770B504000425F3F76AFA1D
:10D250000600FE48006AA04219D021792068032503
:10D26000042906D105212171E369626A0B219847DF
:10D270000DE0A06AF8F759FA012808D1E369626A5B
:10D2800020680B2198470021A162216021713000A4
:10D29000F3F74DFA280070BD70B50500042400F0C6
:10D2A000EBF9280000F0F6F9002802D0FFF7CBFFD9
:10D2B000040000F0E9F9200070BDF8B505000E008B
:10D2C00000F0DAF9E24F002438206043C019816988
:10D2D00000290ED0002D03D04521095C890705D413
:10D2E000002E06D04521095CC90702D01830FFF78F
:10D2F000AAFF641C0F2CE7D300F0C6F98EE70121CA
:10D300000020DAE710B527F078FB002801D10120D2
:10D3100010BD002010BD38B527F0B9FBCB4C16224C
:10D32000206A0021006B03F04EFF206A1522006B7B
:10D33000002103F048FF206A417900293E91E5E28F
:10D340000100000030CF000000040000D038CD5AAA
:10D3500005D08179009141790098FFF7DDFF216ABE
:10D3600003200871206A8069002808D047F048EC43
:10D37000256AAA68EB68801A9941A9690860216A40
:10D38000CB694A6A086803219847216A48690028DE
:10D3900009D08A6A002A06D100920B000200B24826
:10D3A0002833F8F77AF9032038BD70B5060027F066
:10D3B0006CFBAB4C2C20236AC15C5A6A1868DB6991
:10D3C00098470500032814D1206A002E006B05D071
:10D3D0001622002103F001FF332004E01722002170
:10D3E00003F0FBFE34200BF0A9FC216A0220087137
:10D3F00000E00225280070BDF0B585B006000F00E2
:10D400001300002502AA03A904A847F091F9049C7F
:10D41000002C08D0029A01923200002103980B00E0
:10D420000097A0470500280003E670B586B0060007
:10D43000002503AA04A905A802AB47F079F9059CC9
:10D44000002C09D0039A002101920A0000913100BA
:10D4500004980023A0470500280006B070BD80484E
:10D460002030017E491C01767D49096A00290AD0D5
:10D470000A79032A07D1427E521C4276CB694A6A56
:10D48000086809211847704710B5754C206A0028B4
:10D490000FD02030007B03280BD10CF0D8FE206A7F
:10D4A0000121203001737148072200684021F7F7FD
:10D4B0004DFF10BD70B50420694C236A002B4AD083
:10D4C0002C21C95C1868032501290CD10DF069F9DC
:10D4D000002836D001200DE0206A2030057339E0A5
:10D4E0000CF0B5FE2DE0022909D10DF05AF9002803
:10D4F00027D00020FFF759FF0328F1D1ECE70329DB
:10D5000009D1012025F0F1F8206A042120300173AF
:10D51000FFF70BFF1EE0062901D1062006E00729D0
:10D5200007D100210120FFF7D2FE0720FFF7EFFD12
:10D5300010E0082901D10820F8E75A6ADB6998470A
:10D5400008E00120F7F7A6FE4848072200684021BE
:10D55000F7F7FCFE032070BD41490420096A002949
:10D5600007D00A79032A04D1CB694A6A08680521E1
:10D5700018477047052801D2002801D100207047C4
:10D580003B4AC000801806C906C001207047F3B5A9
:10D5900087B00225079842780378100218430128C3
:10D5A00036D1079F891EBF1C30E0F8780E1FB9786E
:10D5B00000023C000843B0422ADC60782178000277
:10D5C0000843FF3864381AD1201D47F0C6EA401ED0
:10D5D00000902000083047F0C0EA7D23DB0058436C
:10D5E000019020000C3047F0B8EA7D23DB0058435F
:10D5F0000290009801A90006000EFFF7BBFFE0783B
:10D60000A17800020843311A3F1DC7190429CCD262
:10D61000FF2064306B4698810C20D881079FBF1C87
:10D6200001241348E1000E18601C7D21049030682D
:10D63000C90047F0D2EA7D2105907068C90047F023
:10D64000CCEA06901022380003A947F072EA10379E
:10D650001035641C052CE4DB280009B0F0BD000087
:10D6600010220004D01E000455CA0000B86D050049
:10D67000140100041648006A002800D001207047F9
:10D680001348006A002800D001207047104800218C
:10D6900010B5006BC943F7F770FE10BD0C4810B50C
:10D6A000006BF7F771FE10BD30B50400094D002086
:10D6B000010038224A4352199369A34201D1100054
:10D6C0001830491C002801D10F29F2D330BD0000C9
:10D6D00010220004D01E0004474810B50068002244
:10D6E000652147F0EAE9002800D0012010BD402163
:10D6F00001817047F8B50024160025000028009429
:10D7000025D13000694601F0F2FE04000DD06B46D1
:10D7100025611A88642A04D3E188032001F0C2FC41
:10D7200002E0032001F0E4FC60816B4618880028C9
:10D7300005D0402020811888001FA08007E0002C21
:10D7400005D031002000A580F3F72DFD7D520C6A35
:10D75000010000002CD30000000400006FFDE8E988
:10D7600000242000F8BDF8B51C000E000027012B96
:10D7700029D0274D042C03D00F2C20D0162C2BD1D0
:10D780000BF04EFA002804D0022011F044FA07F002
:10D790005BFF162C08D11F48310047F0B0EA1E4944
:10D7A0000868401C086004E01A4831003C3847F023
:10D7B000A6EA286807220121F7F7D2FD0CE01548F8
:10D7C00031002838F3E713483100143847F096EA5F
:10D7D000706902210CF01FFD3800F8BD10B500245F
:10D7E000202910D065290CD10A483C3847F08AEA34
:10D7F000002805D10748283847F084EA002800D0DF
:10D800000124200010BD04488260FAE72C64050062
:10D810005C670500244B00049467050070B50C009C
:10D82000150008001AF0C2FCA843010020001AF0FD
:10D83000C9FC70BD70B5002425022800FF309F3060
:10D840000004000C07211AF0E5FCFF35AD1D28048B
:10D85000000C40211AF0DEFC2006000E10222021D0
:10D86000FFF7DCFF641C012CE6DB70BD70B50C001B
:10D87000150008001AF09AFC2843010020001AF055
:10D88000A1FC70BDF3B581B007001AF087FC00243D
:10D8900025022800FF30BF300604360C80213000FE
:10D8A0001AF0ADFC802130001AF0B4FC2800FF30E3
:10D8B0009F300004000C06001AF078FCFA210840A2
:10D8C000002F01D0012108430299002901D0042131
:10D8D00008430221014330001AF074FCFF35AD1DEE
:10D8E0002804000C40211AF08AFC2006000E1022A9
:10D8F0002021FFF7BBFF641C012CC9DB1AF052FC8E
:10D90000FEBD012804D1C448405CC449400001E088
:10D910004800C349085A704770B51400C14A00282E
:10D9200011619070D470C04A137F02D1DF252B4063
:10D9300003E0012802D120252B431377220000F0B9
:10D94000AFFBBA481022022C01D0032C02D1816B0C
:10D95000114301E0816B91438163012070BDB148A7
:10D9600000697047AF4880787047AE48C07870470C
:10D97000AF4870B57D210068490147F028E9890565
:10D98000800A0843AB4900E0401E0A6B920301D4B1
:10D990000028F9DC00281BD11AF000FC1A201AF02C
:10D9A00005FCA04D84092D1D287046201AF0FEFBB1
:10D9B00068702D1F002C06D0002804D1A868012112
:10D9C00009044018A8601AF0EDFBA868401CA86084
:10D9D00070BD10B51AF0E2FB00201AF0E7FB914C85
:10D9E000207001201AF0E2FB607093481AF0F7FBF8
:10D9F000FFF720FFB2201AF0D9FBC00603D5102193
:10DA0000B2201AF0FCFB1021B3201AF0F8FB202101
:10DA10004B201AF0F4FB002060611AF0C3FB10BD2C
:10DA200010B5FFF7D6FF012022F04CFB012010BDFE
:10DA30007C48407870477B48007870477047000208
:10DA4000FF3070B5BC3004040D00240C1AF0A6FBA6
:10DA5000290020001AF0B6FB1AF0A4FB70BD10B527
:10DA60000124642018F078FE71487D210068490186
:10DA700047F0ACE88905800A08436E4900E0401E83
:10DA80000A6B920301D40028F9DC6649002805D10D
:10DA9000C868012200241204801801E0C868401CF4
:10DAA000C860200010BD70B55B49654D085C5B49DE
:10DAB00040000C5A5B48614920308C4217D95F49BD
:10DAC0001830AA318C4212D95E4918308C420ED9D6
:10DAD0005C491830AF318C4209D959491830C839DE
:10DAE0008C4204D90020AC4201D84E4898301AF03C
:10DAF00076FB18F0A7FF06280FD018F0A3FF09281F
:10DB00000BD050489138844201D8C32102E0AC4286
:10DB100003D8C52134201AF055FB70BD70B5040040
:10DB20001500002801D0012300E000230022012974
:10DB30000BD00122022908D0032906D00222002995
:10DB400003D00322042900D0121F3649980018314F
:10DB50000858511C01D1002605E019014CA7EE52CE
:10DB60000100000028D70000000400003C273B858E
:10DB7000314B9200B033C9188E581AF03AFB30007E
:10DB80001AF037FB18F068FF06280FD018F064FF72
:10DB900009280BD0002132201AF01EFB302133203F
:10DBA0001AF01AFBC32134201AF016FB012C02D103
:10DBB0002800FFF782FF70BD7047704770B5040002
:10DBC0000D0018F049FF254940000B5A290020009C
:10DBD000FFF7A1FE002219001AF031FB70BD10B54D
:10DBE0001AF0E6FAB2201AF0EBFA0400C00616D5D5
:10DBF00007201AF0E5FA800709D5022107201AF05C
:10DC000013FBFFF7BFFE022107201AF002FB0821D9
:10DC10001A201AF009FB08494869401C4861210094
:10DC2000B2201AF0D9FA1AF0C7FA10BD080600049B
:10DC30004C21F4033021F403A4670500F0660004CE
:10DC400000A10080685601C0402000805C010004F3
:10DC5000881300000C170000C81400006E5B05005C
:10DC6000002810B50DD0FA4BFA4A04E089008478F8
:10DC7000C9180C60001D01889142F7D18478FF2CEF
:10DC8000F4D110BDF44810B5C169012292051143C9
:10DC9000C161C16B01242143C163F048FFF7E0FF7C
:10DCA000EF48272144700170012010BDE849800031
:10DCB000401800680006000E7047E54A8000801892
:10DCC000016070478200E248101802681206120EC6
:10DCD0000A43026070478200DD481018026812068D
:10DCE000120E8A4302607047002000B5FFF7DEFF86
:10DCF000DB49491F487000BD012000B5FFF7D6FF82
:10DD0000D749491F887000BD0020704737280ED0C2
:10DD100005DC0A2809D014280DD1012070476E288F
:10DD200007D0DC2807D1042070470020704702206C
:10DD3000704703207047FF207047C01F030000B5E5
:10DD400046F042EF0916120E0A0614100C081800CD
:10DD5000052000BD062000BD072000BD082000BD35
:10DD6000092000BD0A2000BD0B2000BD0C2000BD15
:10DD70000D2000BDFF2000BD072907D8002801D0D5
:10DD8000173100E00E310806000E7047202901D13E
:10DD900016207047FF207047B1492331085C704757
:10DDA000AF49491F087070474042032900D1022142
:10DDB000AB4A890042328918AA4A1268012A01D165
:10DDC0008A5601E000228A5600231018A44A521FE6
:10DDD000D35602228A56C018824203DB03228A5697
:10DDE000824200DD10000006001670479D499C4AE3
:10DDF00009684042921C012901D1515601E00021DD
:10DE00005156081802215156814203DB0321515615
:10DE1000814200DD08000006001670479049027834
:10DE2000891C0A7002794A70827840310A708279BE
:10DE30004A7042780A7142794A71C2780A72C0798E
:10DE40004872704786490E20C043891C087048708C
:10DE50004031087048700871487108724872704704
:10DE6000002801DD002004E06421C943884200DA73
:10DE700008004042000600167047002801DD00201F
:10DE800004E06521C943884200DA080040420006E8
:10DE900000167047662801DD662002E0002800DADF
:10DEA0000020000600167047002070477CB56B46C6
:10DEB00000246B4E1970F61D5870009801A946F0A9
:10DEC00030EF00280BD0A5006B465979705BFFF747
:10DED000F4FEA8196B4619794088FFF7EEFE641C22
:10DEE000012CEADB7CBD7CB56B4600245C4E1970CE
:10DEF0000B365870009801A946F016EF00280BD099
:10DF0000A5006B465979705BFFF7D7FEA8196B46E1
:10DF100019794088FFF7D1FE641C012CEADB7CBD37
:10DF20007CB56B4600244E4E19700F365870009821
:10DF300001A946F0FEEE00280BD0A5006B465979EA
:10DF4000705BFFF7BAFEA8196B4619794088FFF796
:10DF5000B4FE641C012CEADB7CBD0EB56B46197067
:10DF60005870009801A946F0E8EE00286C06C7CB6F
:10DF70000100000024DB000000040000C8484E310E
:10DF800003D001A8FFF754FF0EBDFFF765FF0EBDDC
:10DF9000002800B511D1022A05D1092901D8481C51
:10DFA00000BD082000BD032A05D1052901D3C81EE4
:10DFB00000BD022000BD481E00BD022A01D0032A78
:10DFC00040D1702938D011DC8807800F38D18B10F0
:10DFD000093B46F004EE132727292935352B2B352D
:10DFE000353535353535352F2F31350088290DD06C
:10DFF0000EDC7C2922D005DC742901D078291FD1C0
:10E00000762000BD802919D0842919D1862000BD31
:10E0100095290DD099290BD09D2901D0A1290FD187
:10E020009F2000BD262000BD2E2000BD3E2000BD4B
:10E03000972000BD662000BD6E2000BD7E2000BD83
:10E04000362000BD080000BD002804D0012802D001
:10E05000054A904212D1074A921E1070002051705A
:10E060007047000000200090FFFF0000402000806B
:10E0700060030004796805007C0C00040120EFE7D0
:10E08000F84B00B51878FF281DD0012804D10421D1
:10E090007020FFF721FE03E004217020FFF725FE2A
:10E0A0005F20FFF70DFE59784018EF490006000E7B
:10E0B00008606020FFF704FE59784018EA4900061E
:10E0C000000E091D086000BDF8B504000D00160023
:10E0D00000F0AFF9E54FB86AE5490840B862786AE0
:10E0E000E4490843786280210220FFF7F5FD012012
:10E0F00018F046FB80210220FFF7F7FD012018F001
:10E100003FFB2900200023F0A9FEDB48FFF7B2FD0A
:10E110002A06120E31002000009223F0A3FB002CEF
:10E1200010D1022E05D0032E03D00E2D01D1D348DD
:10E1300006E046F010EE012801D1D14800E0D148B8
:10E14000FFF798FD23F010FCFFF79AFF3200210043
:10E150002800FFF7EFFE320021002800FFF7CDFE78
:10E16000320021002800FFF7ABFE3200210028001A
:10E17000FFF7FDFE786ABF49C943084078621AF08C
:10E1800021F82A0031002000FFF7DCFC21F0A3FF7A
:10E19000009932002000FFF7FBFE0600010020007E
:10E1A000FFF715FD2000F6F7CFFE0100200023F059
:10E1B000E5FB2000F6F7C8FE01002000FFF706FD92
:10E1C000022107201AF03AF823F030FC2000F6F77D
:10E1D000BBFE002804D0102107201AF02FF803E01E
:10E1E000102107201AF01FF820214B201AF026F8E2
:10E1F00031002000FFF7ECFC31002000FFF743FC6A
:10E2000023F026FC20214B201AF00DF82000F6F711
:10E210009BFE002821D09C48006B800319D4072066
:10E2200019F0D8FF8F498009C91E012803D1C86998
:10E23000401CC8610AE0022803D1086A401C086239
:10E2400004E0032802D1486A401C48628869401CE7
:10E2500088610221072019F0E6FF19F0B7FF2000BE
:10E2600023F0CCFB894E072031694003002C08D1F4
:10E270008143316130690521490308433061844895
:10E2800007E081433161306903214903084330616C
:10E29000804830612000F6F777FF200022F055FF1C
:10E2A000012803D12900200022F091FF290020003D
:10E2B00022F09EFF30690821084330610120F8BD3B
:10E2C00030B50024674D80012D1D2B57000C002B0D
:10E2D00000DC5C4223061B0E1F241F2B00D21C00F7
:10E2E000202905D0402905D0802905D0002304E04D
:10E2F000102302E0202300E03023674D0106090EC1
:10E300002960000A291D0860D220FFF7D9FC4009C6
:10E3100040012043002A02D14021084301E0BF21EF
:10E3200008405D4914310860802003435A48001FAB
:10E33000036030BDF3B5D2208DB0FFF7C1FC4021A2
:10E34000084203D055480926009003E0534809309D
:10E350000B2600900D98310046F004EC00252F00AC
:10E360000195CC20FFF7ACFC4006FAD5002202ABA9
:10E3700023E0CC20FFF7A4FC00090001BCAB23BACA
:10E380000100000020DF0000000400009B929D5D62
:10E390004006400E104345490006000E091F086064
:10E3A000D120FFF797FC000494001851D020FFF70C
:10E3B00091FC1959000208431851CF20FFF78AFC3D
:10E3C00019590843185101994018521C0190B24242
:10E3D000D9DB0198002818D0002413E0A10002A87E
:10E3E00040580102081A019946F01EEC0D990006EA
:10E3F000000E085541190D0600992D0E095741438D
:10E40000CF19641CB442E9DB08E00D9AFF21701EAD
:10E410000D0011540099085607023F1A0D980D9AE5
:10E420000178FF20401B09181170009A00215156F5
:10E430004143C8190E99002902D00E990012088094
:10E4400030000FB0F0BDF8B504001EF05FFA0028F0
:10E450005DD016F080F9002859D02000F6F77EFD37
:10E46000002854D01348016A054E0C07FF25240FDD
:10E470002D35114F803E28E0776805007C21009003
:10E4800000A80080FCFDFFFFC000008060030004C6
:10E49000AC070004080700040C07000440200080BB
:10E4A000C0A2008008A80000086800003423009083
:10E4B000545B05000000019000A700800A2018F0BE
:10E4C00069F91348006A0407240FF868800708D523
:10E4D000F06A400005D5052C01D0062C01D16D1E37
:10E4E000ECD2FF252D3502E00A2018F053F9F86828
:10E4F00080070CD518F0CDFC002808D0F06A400049
:10E5000005D4052C01D0062C01D16D1EECD2F8BD2E
:10E510000000019070B5FF4D6969FF488164FF49B3
:10E520000968C164FE4800248461F6F7A9FB042051
:10E53000F6F711FB0C20F6F70EFB2C6070BD10B542
:10E54000F54C0200616B206B46F056EB7D22D20049
:10E5500046F052EBE36AA26A46F052EB10BDF8B502
:10E560007D220700EC4CD200616B206B46F044EB3F
:10E5700005000E00E16AA06A3A0046F03EEB330067
:10E580002A0046F03EEBF8BD70B50600F4F70BFE2E
:10E590000400E4490025300046F036EB2B00220051
:10E5A00046F02EEB70BD10B50400F4F7FCFD210021
:10E5B00046F02AEBDB4A002346F022EB10BD70B593
:10E5C0000400D54D01206872D448816A020C1143C1
:10E5D0008162D2488038C16B820C1143C16318F04C
:10E5E0004FFAD1494000085A64235843A861604358
:10E5F000F6F795FA70BD10B50124F6F785FA2000FC
:10E6000010BD10B5F6F795FA0400F6F796FAC24970
:10E6100000220C634A638B6943438B62BF4BCA621F
:10E62000986A1C0CA04398624A7210BD70B5BA4C2F
:10E630002069FFF784FF618946F0F6EAE061050092
:10E64000BA48A16946F0F0EA0100A84201D8E069A1
:10E6500001E00800E1617D21C90046F0E6EA2062A0
:10E6600070BD0A2010B5FFF7AAFFFFF7C4FF040032
:10E6700010D0FFF7C6FFFFF7D9FFA748016A0800CF
:10E680000A2907D9FFF79BFFF6F73EFAFFF7B9FF14
:10E69000FFF7CCFF200010BD70B504009E4D012097
:10E6A00068729E48816A020C1143816218F0E8F991
:10E6B0009D494000085A64214143002CA96102D0C1
:10E6C0000800604305E0E86948437D21C90046F041
:10E6D000ACEAF6F724FA70BD8F490A6A824206D87E
:10E6E0004A7A002A03D14979002900D1D4E770473A
:10E6F000F3B583B0002788490D006B6B2A6B390096
:10E7000046F036EB02900C00E96AA86A049A46F0DB
:10E7100074EA05000E00062246F06EEA3B00052270
:10E7200046F06EEA0191AA0FB10011430090A800D3
:10E730003B00052246F064EA029A2300121A8B413C
:10E740001AD3684607C8801AA14115D307223100A1
:10E75000280046F052EA029A801861416E4C4A073E
:10E76000C0081043636B226BC90846F04AEAE162B5
:10E77000A06204986763206305B0F0BD70B5664C75
:10E780006079002811D1F6F7BFF9F6F73CC18CAEDD
:10E79000010000001CE3000000040000B30318E0C7
:10E7A000D2F90500F6F7D3F901006148826A030C3B
:10E7B0009A438262A06948432900FFF7A3FF002023
:10E7C000607270BDF8B5FF245A34584F3B68C61AC2
:10E7D000361BFF3EFF3E361F002E04DC5948816A7F
:10E7E000491C816203E0814201D8824201D20020AB
:10E7F000F8BD3000FFF7BDFE05002000FFF7DDFE8D
:10E800000400854209D92C002800FFF7C7FE301A02
:10E81000FF305A30FFF7ADFE050000222300110043
:10E820002800F6F777FA3879002806D13868FFF71C
:10E83000A0FE0004000CF6F769F90120F8BD38B518
:10E8400004006846F6F767FD3F480099006881427A
:10E8500001D0F6F745FD3D4800990068814201D09E
:10E86000F6F73EFD3A483B4D807FFF280BD10AF07A
:10E87000CCF9002807D0002C05D0354A28681E3274
:10E880000D21F6F73FFD00992868814201D0F6F787
:10E8900027FD314800990068814201D0F6F720FD3C
:10E8A00038BD294838B50068F6F720FD27480068CC
:10E8B000F6F71CFD274D2868F6F718FD2648006876
:10E8C000F6F714FD224CA17FFF2905D028686A467F
:10E8D000F6F718FDFF20A07738BD10B5FBF7E7FD70
:10E8E00004000AF0F5FC204310BD194810B5A0380B
:10E8F000007FC00705D019F079FCFFF761F819F027
:10E9000079FC10BDF8B500250E4E7560FFF7C9FF04
:10E91000124908690122D206104308610C48104FC1
:10E92000A038007FC0071DE000A50080185F01C06F
:10E930008020008040A6008040420F006E5B0500F2
:10E94000002D3101C83401C0586705009C6C0500DA
:10E9500090670004B46D0500046A05000022008081
:10E96000EFFFFFFFFC4C1FD0F1F718FF009020696C
:10E970000B21884320612069F16808432061A5616B
:10E98000F6F788F9F6F7FEF9F448C760F248C030A8
:10E990000168082211430160F148016811430160D8
:10E9A0000098F1F700FF06E0A561F6F773F9F6F7B6
:10E9B000E9F9EA48C76046F0B2E9EA48EA49806CFA
:10E9C000486120691021884320610120F6F7C1FBCE
:10E9D0000021080010F09DF9002801D0022001E07C
:10E9E000E248006823F0B3FEF6F727FFF8BDFFB555
:10E9F00083B000240500DE4F0C9E0AF001F90028C8
:10EA000000D0022010F02FF9002802D0407BC00671
:10EA1000C00FFFF714FFF1F7C1FE00220290D548A6
:10EA2000009200680822012101ABF6F7C5FC0198AD
:10EA3000002817D1D048002200684A2146F06EE82D
:10EA40000022002801D0002E0CD0C6493F23886D3B
:10EA5000C96DCA4EDB0419403040130016005940FE
:10EA600008430AD0BF48C54C826DC16D3F23224088
:10EA7000DB0419408265C1651FE0002D29D046F0F6
:10EA8000F2E8009004982A686B68101AB341009A63
:10EA90000C0019002300121A8B410AD2009A286830
:10EAA0006968801AA141069A0599FFF78BFE002834
:10EAB00006D1B3488169491C8161FFF723FF14E146
:10EAC000A8486A6829688030C260816000F014FA42
:10EAD0000400A34908680822904308609E48C0309B
:10EAE0000168914301609C4E3169A54A04200140B0
:10EAF000D16031698143316130690321084330615C
:10EB0000A048F1F7D9FD6CE09D49486A401C486275
:10EB1000781E070062D1086A0F00401C08620AF0E4
:10EB200079F8002820D0B069B06930698008800089
:10EB300030618B4801680822114301608649C03169
:10EB400008681043086030698D49C968084330611E
:10EB5000F6F773FEFFF7D6FE0298F1F724FE0120C8
:10EB60000004F1F7A9FDC3E030698008800030613E
:10EB700030698349C968084330617749C031086802
:10EB800008273843086076490868384308600298C7
:10EB9000F1F709FEB0698006800F0128CCC39450BC
:10EBA0000100000018E7000000040000E0D9CB8C51
:10EBB00007D178480169491C016100200EF0C4FEAC
:10EBC00001E00EF007FFF1F7F3FD6A4902900868D3
:10EBD000B84308606549C0310868B84308603069C7
:10EBE0000421884330613069032108433061654F57
:10EBF000012017F0E3FDB0698006800F03288DD156
:10EC000001200004F1F762FD002D0DD000F07EF927
:10EC100006990400884202D80598844204D25D49CE
:10EC2000C869401CC86166E054484169524A916411
:10EC300002214161594845F0ECEF46F076E8584929
:10EC400008690122D206904308610020F6F78BFA8A
:10EC500030691021084330614E4F3878022801D1C5
:10EC6000022600E04026002D02D000F04FF90400FB
:10EC7000002C05D0032023F074FD0120064302E0A0
:10EC8000042023F06EFD17F0FBFFF007C00F01D04A
:10EC9000F6F702F8422006401BD070060AD5102075
:10ECA000F5F767FF1020F5F770FF0420F6F77BF803
:10ECB000F6F7A0F8B0070CD5012636033000F5F7BB
:10ECC00058FF3000F5F767FF0C20F6F76CF8F6F701
:10ECD00091F801267E60002D17D000F017F90699F3
:10ECE0000400884202D8059884420ED2F8690121B6
:10ECF00009044018F861FFF70FFEFFF700FE0298C5
:10ED0000F1F75BFD002007B0F0BD2648844203D236
:10ED1000002C01D024480670FFF7E9FD002801D03F
:10ED2000102000E03020F4F709FA0298F1F745FDD1
:10ED300045F0C6EF1D49884209D00022D24312484F
:10ED4000009200680822012101ABF6F73FFB012089
:10ED5000D9E710B509F068FF002803D00D484068D6
:10ED6000002801D0FFF7D8FD10BD000040A60080AC
:10ED70008020008000A30080185F01C000A50080F3
:10ED8000806D050088130000F071050028640500FF
:10ED900018000400C83401C0F10001001000100088
:10EDA00000220080B80B0000A1640500507F050020
:10EDB0005F4810B501690B229143016101695D4A09
:10EDC0009268114301610021816119F019FAFEF77F
:10EDD00001FE19F019FA564AC0321068082108439A
:10EDE0001060554A106808431060BDE7F8B5524AF4
:10EDF000524811680826B14311604D4AC03211686B
:10EE0000B14311604A4C21694A4D04273940A96039
:10EE10002169B943216121690B2211432161401EFF
:10EE20001BD1FFF7C5FF0EF0D5FD20693840A86063
:10EE30002069B843206140490868B04308603C49F4
:10EE4000C0310868B0430860A0698006800F0128BF
:10EE500002D16869401C68613848A1698906890F38
:10EE60000329D8D1F8BDF8B530200026340035008C
:10EE7000F4F725FA45F000EF009031480F000B0041
:10EE8000C168009A8068121A8B4106D22C48009AF9
:10EE9000C1688068841AB9410D002A4A3300121BE8
:10EEA000AB4129D22648284980380068FF245A34CB
:10EEB0000E1A361BFF3EFF3E361F3000FFF763FB86
:10EEC00005002000FFF783FB0400854209D92C00D0
:10EED0002800FFF76DFB301AFF305A30FFF753FB65
:10EEE00005000022230011002800F5F71DFF102067
:10EEF000F4F724F90020F8BD0120F8BD104880384F
:10EF0000007970470E488038407A704710B5F5F7A1
:10EF100037FF0400F5F703FF201A05D50549C86A35
:10EF2000401CC86200201FE7FFF71DFB1CE7000024
:10EF300040A60080C83401C000A3008088130000F0
:10EF4000985F01C0280A0000D4170000242358430A
:10EF5000FF494018C1690905C90D81614069C900AF
:10EF60004018406870472423F0B55843F8490127FA
:10EF70004018C16942690905C90DCB00D2180023A8
:10EF80003F05FE02146805693C406D1E8D420AD1A2
:10EF9000C168090131431160C2690121090391432C
:10EFA000C161002109E0C5690835ED04C36A8F021B
:10EFB0000100000014EB00000004000014B6BE388D
:10EFC000ED0CC56185682D013543491C1560002C89
:10EFD00007D14269CC001219816104695B1C9C4213
:10EFE000DAD2C069F0BD24214143DE4A10B58C1845
:10EFF00045F0E0EEE2690100D204C9040120D20C20
:10F00000C90C8A4200D1002010BD10B502E00120D9
:10F01000F6F786F90420FFF7E6FF0028F7D102E0B3
:10F020000120F6F77DF90520FFF7DDFF0028F7D175
:10F0300002E00120F6F774F90620FFF7D4FF00285C
:10F04000F7D1C94C0BE00EF004F8002804D020687A
:10F050000022622145F076ED0120F6F761F90320E8
:10F06000FFF7C1FF0028EED110BDC048802110B5C8
:10F0700045F0BCED10BD090530B5CC0D2421514340
:10F08000B84A0005C00D8D18B84A012109E0115495
:10F090002B695B1E834201D1002002E0401C00046A
:10F0A000000CA042F3D130BDF7B582B02423070095
:10F0B0000498AC4958434618F1F784FB0190AC48DA
:10F0C0000569049A2805C40D03993800FFF7D3FF9A
:10F0D0000127A64BFF071EE07069E1004018426857
:10F0E0000021116019553169491EA14209D1F16809
:10F0F000090139430160280001252D0385430024BF
:10F1000009E0B168083509013943ED04641CED0CD0
:10F110002404240C0160185D0028DDD12804049922
:10F12000000C45F04CEE0198F1F751FB05B0F0BD35
:10F13000242358438B4930B54018C16905690B0534
:10F14000DC0D01236D1E1B03A54213D0140AE4003D
:10F150000919C904C90C1206C16101D1C16903E0D2
:10F160000831C904C90CC1610A052924120D240102
:10F17000A24201D98B43C361C06930BD24235843E7
:10F180007849F0B54018C16944690905C90DCA003C
:10F190000669A3180022751E1B6801273F053B4026
:10F1A0008D4205D1C1693F128F430021C76105E03F
:10F1B000C7690837FF04FF0C491CC761002B05D144
:10F1C000CB00E318521C96428161E5D2C069F0BDC4
:10F1D000644A674900206C32403110B5096BD2692E
:10F1E000090C13050C051B0D240DA34205D10123A9
:10F1F0001B031A4019408A4200D1012010BDF0B50E
:10F2000024238E46002158438C4656494018C16934
:10F210000905CA0D82614169D300CB180121090398
:10F2200024E01C68A50201D5E4072ED10469641E00
:10F2300094420BD1C26801241201E40722431A60F0
:10F24000C3690A009A43C26100220BE08468012569
:10F250002401ED072C431C60C3690833DB04DB0C7D
:10F26000521CC3614369D4001B198261C469056AD9
:10F2700026052F05360D3F0DBE42D2D10C400D4064
:10F28000AC42CED06146012904D1C06971460880E4
:10F290005868F0BD0020F0BD70B504002AD02500EC
:10F2A0002035287D217DC006CB09820F4906E07EEE
:10F2B000490E002A09D0012A0AD0022A01D0032AC5
:10F2C00009D11800FEF78AFD06E0FEF768FD03E0AD
:10F2D000FEF74EFD00E0FF20E076287DC006810F9E
:10F2E0000B202056FEF792FDE07207202056FEF715
:10F2F000AFFDE07170BDF8B50D000700242050434C
:10F300001849402244183900280045F058EC2800DC
:10F31000FFF7C2FF2800403045F064EC390040316F
:10F3200020220D00009045F04AEC29882269A0694E
:10F330000D00603D0026521E904207D1E0680A1D74
:10F34000824203D90500643D0E1A361D009839002B
:10F3500020302A006431009045F030EC002E0FD0B0
:10F36000009807E0007701C028640500B07801C06C
:10F3700080A30080616940194968320045F01EECA5
:10F38000F8BDF8B505000E001F0000240520FFF7AA
:10F39000E7FD4188EF4B99421AD1010040312860C6
:10F3A0003160098840390904090C09D00F239B01F9
:10F3B000994205D864302039106001244AEB078E49
:10F3C0000100000010EF000000040000476C6D54C5
:10F3D000398007E00520FFF7DAFD0004000C052165
:10F3E00045F0F6EC2000F8BD38B50400F1F7F4F96B
:10F3F0000500DE488069DE49000C48610520694649
:10F40000FFF707FF00280BD04188D74A914207D168
:10F41000D849418005222100FFF777FF012400E051
:10F4200000242800F1F7DDF9200038BD38B50400CC
:10F43000CE480069CE49000C403908630420694673
:10F44000FFF7E7FE002804D004222100FFF75DFF4C
:10F45000012038BD38B50400C448006AC449000C16
:10F46000886306206946FFF7D4FE00280BD0010010
:10F4700040310A88682A01D968220A8006222100C0
:10F48000FFF743FF012038BDB949B84854390A0095
:10F49000F0B56C324038006B040C08001430C460C6
:10F4A000B248006A2705030CB1483F0D8363CE695B
:10F4B000012031050500090DB94200D100250127C1
:10F4C0003F0301003E403C40A64200D00021D269EB
:10F4D000294315051E0504002D0D360DB54200D13A
:10F4E00000240C433A403B409A4200D00020204385
:10F4F000F0BD70B59E4D9D48543D4038006B2900CD
:10F50000000C1431C8600005C40D032045F05CEC0C
:10F510000105CA0D012300211B031840A24205D199
:10F520002E6A1E40864201D1002070BD641C532CFF
:10F5300002D2491C1029F1DB012070BD8C4810B5A6
:10F540005438C1690905C90D81614269C900521861
:10F55000C169006A0B0504051B0D240DA34205D1EA
:10F5600001231B031940184081420ED150687E4987
:10F570000068000C884208D07F490868401C086079
:10F5800000200EF0F5F9002010BD012010BDF8B5E7
:10F590000D0007007548002640380E80006B744946
:10F5A000000C4039C860FFF7C9FF00281FD00320B6
:10F5B0006946FFF72EFE040019D0402221003800D2
:10F5C00045F006EB3800FFF771FE6B461988E180C5
:10F5D00026610221200021733900403040310600AD
:10F5E00044F0B0EE3088001D28802000F8BD0020D7
:10F5F000F8BDF8B5042202275D487B02403802615D
:10F600000021836181625E4D076245625B4AC3618E
:10F6100042619A000163C262584A5A4ECB005C199B
:10F6200062600124A4021219491C0129EE50F5D38D
:10F63000534BC900CC186260524A5A504C490622BA
:10F640008A61514ACA610222FF235B1C8A624C4EC6
:10F6500000220B6220360A63CE624B628A631A0173
:10F66000494B4A4F4A630022D400A5196B60FF330F
:10F670005B1C521C012A3751F6D3414CD200203476
:10F6800015196B60414BA3500522426322001832CA
:10F69000826302220027CF6053024A602500C363C1
:10F6A000103D4F618D60D2020B600A612200354E21
:10F6B00018323900CB005C1962600124A4021219CF
:10F6C000491C0129EE50F5D32D4BC9001033CC183D
:10F6D00062605E5026490322C039CA662C4A0A6716
:10F6E0005322CA67FF22521C47604A6712018A6789
:10F6F000284DC760264E056000248260042130003A
:10F7000045F062EAE00041194E60FF361F49761C61
:10F71000641C522C2950F1D30421300045F054EAE6
:10F72000E0004119114B4E601B49403B29501F60BE
:10F7300013490E481031C161022484610B4AC10C87
:10F74000803A51620E4E4661046111622036466273
:10F75000046291625D6353201863116145F03CEBD4
:10F760000248C0308760F8BDEFBE000000A40080F2
:10F77000C07701C0BAAB0000683601C0008401C088
:10F78000C87B01C000400080008C01C000100080D8
:10F79000008E01C0307901C000000180E9481421C9
:10F7A00010B545F02EEA10BD70B505000E0001D170
:10F7B000012070BD30898419607A217A00020843E3
:10F7C00001280DD1607B217B000208432C9FB6C726
:10F7D000010000000CF3000000040000F8A948E755
:10F7E000032807D1002D11D0280001F044FA002889
:10F7F00012D001E0002D03D0E87AA073A87AE0735C
:10F80000607A217A00020843012809D131000420DE
:10F8100000F0B1FA002803D1300045F0B0E9D1E79B
:10F82000002070BD70B50D00103211040400CB48EB
:10F830001E00090C002245F0CEE90028206015D0FA
:10F8400002210173216820200881206801212030D5
:10F8500028600172002141722868310A06734173E1
:10F86000296800208872C872012070BDBC490868F0
:10F87000401C0860002070BD1CB50C000300022273
:10F88000694601A8FFF7CEFF00280FD0009800219D
:10F890000174002C417405D0019901234A7B1A435D
:10F8A0004A738C61022181720021C17201981CBDD2
:10F8B00010B5040008001100FFF7DEFF002803D098
:10F8C00001002000FFF77AFF10BD0022F0E77CB5B1
:10F8D000140005000B000222694601A8FFF7A2FFF1
:10F8E00000280BD00098210A04744174022181720F
:10F8F0000021C17201992800FFF760FF7CBD7CB533
:10F90000040015000B000822694601A8FFF78AFFD2
:10F91000002811D0009800210174417406222900AA
:10F92000123045F060E90099082088720020C87202
:10F9300001992000FFF742FF7CBDFEB51C041E00AC
:10F9400005001700240C0B002200694601A8FFF7F0
:10F9500069FF00280DD0009832003900103045F0C2
:10F9600042E90098210A8472C17201992800FFF7C8
:10F9700025FFFEBD7CB514001E0005000B0008220B
:10F98000694601A8FFF74EFF002811D00098210A10
:10F990000474417406223100123045F024E90099C4
:10F9A000082088720020C87201992800FFF706FF1E
:10F9B0007CBD70B5060010891500841800222274E1
:10F9C000200062740622123045F00CE9E07AA17A38
:10F9D000000208430830A072000AE07229003000DB
:10F9E000FFF7ECFE70BDF0B5012089B00290F0F792
:10F9F000FDFE002706905B483C01005D00287ED09C
:10FA0000594D00236019083003C858405940084335
:10FA10007AD000F090F900287AD1FF229132592350
:10FA200004A905A8FFF7FEFE002806D14C49486846
:10FA3000401C4860002002906AE04B480059049C3A
:10FA40000190002010343D00039050E045482E0105
:10FA5000805D00284AD044480023301808900830C0
:10FA6000079003C85840594008433FD03E48019A88
:10FA70008059927A817A914238D10199C07AC97AB3
:10FA8000884233D1FF209A302070000A60703548D8
:10FA900006223618F11C201D45F0A4E87078A072EB
:10FAA0000020E0720898082280882073000A6073A2
:10FAB0000020A273E07320000799103045F092E80F
:10FAC000079800210A0006C0E07BA17B00020843E2
:10FAD0000C300004000C010AA070E1700399241D91
:10FAE000091D41180904090C041903916D1C0A2D04
:10FAF000ACD3049903988872000AC87200E003E04E
:10FB000005990198FFF75AFE7F1C0A2F00D272E771
:10FB10000698F0F770FE029809B0F0BDFEB51D0022
:10FB200006000F0014000B000322694601A8FFF72E
:10FB300079FE00280ED0742F0CD10098E5210174B5
:10FB400044740321857481720021C17201993000CF
:10FB5000FFF734FEFEBD00000C8405008C0D000490
:10FB6000CC68050058490004484A000470B50500F7
:10FB70000089441909F0A4F8002808D0607B217B93
:10FB8000000208430B2802D0052009F031F9FB4B95
:10FB9000F9481C680022290000680223A04770BDB4
:10FBA000F74801000C394860F648012141700021F6
:10FBB00001707047F24900200C394860F1494870E3
:10FBC0000870704730B5040085B001A845F00EE814
:10FBD0006B465879C10601D480061DD591C26C418F
:10FBE0000100000008F7000000040000AB739B8BCD
:10FBF0006B4618790007000F012817D1F0F700FEB7
:10FC00000500E648007801280DD002A945F000E87B
:10FC10006B46187901210207120F0092220000237F
:10FC200002A8F5F74DFA2800F0F7EFFD05B030BD5A
:10FC3000DB48D84900680C390028886001D10120D0
:10FC4000CAE77047D348D6490C38806809688842AB
:10FC500000D0C1E77047CF4AD1480C3AD17800684C
:10FC6000052905D2022101235156D356994203DCBE
:10FC7000002809D0002006E00023D356994203DD76
:10FC8000002801D10120A7E77047C2490C398870CC
:10FC9000E1E7C0490C39C870DDE710B5BE4C6078AB
:10FCA000002809D001202070A06D002802D044F067
:10FCB000ACEF6065FFF7BCFF10BD10B5B94844F06C
:10FCC000CCEF002802D0FFF75BFFF7E710BD70B55F
:10FCD000F0F796FDB04C05006078002809D0AD49DA
:10FCE00004200856411C04D0811C02D0012117F0C9
:10FCF000DFFFAD480078012802D1142009F06EF82A
:10FD0000002020720420FBF758FAA848002200685F
:10FD10000C2144F036EFFFF7D0FF2800F0F775FD17
:10FD200070BD10B5FFF7D3FF9B49002008704870E5
:10FD300048659F490860FFF785FF10BD9648017A26
:10FD4000032901D0032101727047924900200C3928
:10FD50004968002904D090490978002900D0012081
:10FD60007047FF2800D008407047924910B50968D5
:10FD700044F086EF7D22D20044F07AEF8905800AB4
:10FD8000084301D044F078EE10BDF8B5002504001A
:10FD90000E002A00002901D030898219FFF7D5FF13
:10FDA00000287ED07C49087A03287BD00228FCD02A
:10FDB000600721D5002E28D0507B117B05020D4312
:10FDC0000A2D0ED006DC032D11D0082D0FD0092DE1
:10FDD00014D10CE00B2D04D0102D08D0122D0DD114
:10FDE00005E07548754900880978084301D0FF246B
:10FDF00004E00420844301E0002E06D0A006800F1A
:10FE000003D0507B117B05020D43624F0C3F786895
:10FE100044F006EF01002000FFF7A3FF00286BD09D
:10FE2000674C002D1AD0208800280DD05949042095
:10FE30000856401C08D178684079FFF796FFFFF715
:10FE400070FF0020208053E0F0F7DAFC05005548F1
:10FE5000310044F0AEEF2800F0F7D7FC78680426B4
:10FE60008657FFF772FF002811D04B4D686D0028B0
:10FE70000DD0A86D00280AD002E0524816F0C6FC4A
:10FE800044F0C2EE696D401AA96D8842F5D342482C
:10FE900002210172701C08D0B01C06D00021300075
:10FEA00001E01FE015E017F003FF78684079FF28B4
:10FEB00021D0FFF75AFF208800281CD0FFF745FF0C
:10FEC000002804D0FFF72DFF0020208013E02088B9
:10FED00011E060070FD5002E0DD03248310044F0FC
:10FEE00068EF08E0600706D5002E04D0FFF7E5FEB6
:10FEF0003000FFF745FE0120F8BD27485C2110B512
:10FF000044F092EE10BDF8B500220400224F0D001F
:10FF1000BA82BA651DE06078217800020843FF3894
:10FF2000163819D0A1280AD12000062D07DB417907
:10FF3000027908027D231043DB005843B865E1785D
:10FF4000A27808021043291A091F0D042D14241D3C
:10FF50000419042DDFDCF8BDE178A2780902114311
:10FF6000CE082000F2009142E9D1121D11040914BB
:10FF7000A942E4DC0821082E00D23100CA00011D8C
:10FF80000548143044F038EE25E000002C640500EC
:10FF90009C670500E06805002084050058650500A1
:10FFA0007C0C00040C840500B06D0500286405007D
:10FFB000143501C0685601C060860500C869050097
:10FFC000CC69050088130000F000C019002114302E
:10FFD0000A0006C0761C082EF6DBB0E7F3B585B044
:10FFE00000250700554804950390388984DC0A0AE7
:10FFF0000100000004FB0000000400005F1CEE3F55
:020000021000EC
:100000003900C419243140188446E0782E00C00716
:1000100001D1A01D01E020001230A2781307990F32
:10002000012903D1100908287ED018E09A0F01D1C8
:10003000402514E00388474A934208D143889342FD
:1000400005D18388934202D101252E0007E0007874
:10005000C00702D00825032601E002252E00022950
:100060002FD10698002101706046801D04903A4807
:10007000406844F0E0ED002806DA0498022203A963
:1000800044F0B1F800285ED07F69002F19D0380005
:10009000F2F79DFD002802D0387B400704D43800D9
:1000A00012F0D5FE00280CD02C48019004980222B2
:1000B00001A944F098F8002803D10699012008709E
:1000C00041E02548406844F0B6ED28423BD0A07896
:1000D0000007800F022839D1214FB88A002835D077
:1000E000C120C0000025029028E0B04202D019498A
:1000F000884220D1E08A1749884207D0210004981D
:100100001631022244F06FF8002814D1A069401C77
:100110001CD00498022202A944F065F800280AD1F4
:1001200004981A30210000E010E01831042244F055
:100130005AF800280AD06D1C082D04DAE800C4190A
:10014000A08A0028D1D1002007B0F0BD0120FBE734
:1001500086DD0000FFFF0000D4680500888E0000E7
:1001600020840500A14900208880091F086070478D
:10017000F8B50C00F0F74EFB0090200044F05AED6B
:100180009A4944F0FEE8607921790002974F0843CC
:100190000228B88004D90098F0F741FB0020F8BD90
:1001A000A41D934E002511E0682068432178315446
:1001B000617880194170801CA11C00F0DFF8E078A4
:1001C000A17800020843241D04196D1CB888A842B8
:1001D000EADC0098F0F723FB0120F8BD10B504001D
:1001E000824844F028ED204000D0012010BDF7B532
:1001F00082B006007E4F002464E0F0F70BFB68211C
:1002000061430500785C049A824303D02800F0F72C
:1002100006FB56E0764AC919D03210704878507003
:10022000891C901C00F0AAF82800F0F7F8FA3000BA
:1002300000F0ADF8002844D06D4D0024D03568782A
:1002400001270009012803D1300000F041F825E022
:10025000022823D1318970698919009144F0DEEDBB
:10026000040001D13C0017E0200044F0DCED010067
:10027000604B300001AA19F09FFB002803D1200039
:1002800044F0D4EDEEE700996B469B8800221231D2
:10029000200044F0D0ED0024002C02D16878C00783
:1002A00004D00398002C076008D102E003980021D5
:1002B00001606878800701D40020B080012005B07B
:1002C000F0BD641C49488088A04296DC0020F6E717
:1002D000FEB5FF210022F53101904669464844F001
:1002E0008EEC04001FD0B020251820811221280098
:1002F00044F088EC1420287100202F001437687116
:10030000009700980E2144F07EEC31200001321855
:10031000390001980E31029219F0ECFA070003D16E
:10032000200044F040ECFEBD009802990622801D9A
:1003300044F06CEC390000980622123144F066EC6F
:100340000099C120C0000873000A48730198042175
:100350008088A0800820207330696061F07A68701E
:10036000B07A28700220A8710020E8712A20A870B5
:100370000020E8702000F1F7C1FFFEBD10B54A78FB
:100380000B7812021A43921C44F040EC10BD10B5D9
:1003900001890400243009188AB00E390E2206A8FB
:1003A00044F034EC114844F046EC0100200004AA6B
:1003B00019F099FB002816D019F069F90C4C04A922
:1003C000D034A01C19F0F5F9002805D0A01C01A913
:1003D00019F038F9029C00E0002405980E2206A9C5
:1003E00044F014EC20000AB010BD0000EC680500D9
:1003F0007C8405004C060000D80D00041B78317584
:100400000100000000FF0000000400000CC63D5386
:1004100010B5040073D06321200044F0FEEB0820E7
:10042000207000206070FF20401DA070000AE07066
:100430000221002021716071FF20801D2072000ABE
:1004400060720020A172E072FF20C01DA073000A3C
:10045000E073002021746074FF2008302075000ACA
:100460006075080AA175E0753C202076FF201730E2
:10047000A076000AE076080A21776077FF22200044
:10048000183220300270120A42700A0A8170C2705B
:10049000FF2227328271120AC2710A0A0172427265
:1004A000FF2228320273120A42730A0A8173C2734E
:1004B000FF22293210308270120AC2700A0A0171BA
:1004C0004271FF222A320272120A42720A0A8172B1
:1004D000C272FF2225328273120AC27310301022B8
:1004E0000270002203004270FF204A305034A07096
:1004F000000AE070080A217132216071997510BDFF
:100500000B21890140188089002800D00120704704
:10051000FFB581B01D000F00C878897806020E4330
:1005200001980B21890141188C68002C04D1FF48E7
:1005300088600400FFF76CFF6078217800020843B0
:10054000012D03D1F878B978000205E0022D05D11C
:10055000F978BA7809021143084306E0032D07D160
:10056000F978BA780902114388432070000A607054
:1005700003983F1D001F0297070401983F0C40306D
:100580000090CEE0042F73D30299C8788A780002D5
:1005900010434A780B7811021943001DFF23000411
:1005A0002533000CCA1A994273D025DCE04BCA1AD5
:1005B00099425ED011DCFF39491F44D001294CD04B
:1005C000022967D1012D03D0022D3BD1710739D506
:1005D000220060322100123188E00F2A5BD0102AFD
:1005E000EFD1012D03D0022DEFD1B106EFD52200BE
:1005F0005B322100243179E0042A62D00EDC022A29
:1006000054D0032ADDD1012D03D0022D7FD1310634
:100610007DD522005E322100303167E0052A5BD0B3
:10062000252A73D1012D03D0022D70D131056ED54D
:1006300021000298002256311AF0ACFB009A562194
:10064000095D917663E0012D03D0022D5FD1F107A2
:100650005DD022005832A11D48E0012D03D0022DAB
:1006600055D1B10753D522005A3221000C313DE05B
:100670005AE0012D03D0022D49D1310747D5210081
:100680000298002218311AF085FB009A217E5176DB
:100690003DE02FE03AE0012D03D0022D37D1F106E5
:1006A00035D52200593221001E311FE0012D03D023
:1006B000022D2CD171062AD522005C3221002A316C
:1006C00014E0012D03D0022D21D1F1051FD5220008
:1006D0005D322100363109E0012D03D0022D16D103
:1006E000B10514D522005F3221003C3102981AF086
:1006F00051FB0CE0012D03D0022D08D1710506D568
:100700002100029842311AF063FB00E03800874272
:1007100003D3391A0F043F0C00E000270299081890
:100720000290002F00D02DE705B0F0BD0A000B218C
:100730008901401810B58168901C002904D0582206
:1007400044F06EEA562010BD002010BD70B50500C3
:10075000059E049C0020002905D05178002900D175
:100760000121197070BD19780029FBD0491E0906B6
:10077000090E1970F6D15078002801D018700FE0DA
:10078000B00041190B20800108188068002807D0AC
:100790004178027809021143A1430170090A4170AE
:1007A000012070BDF1B584B0049809F011FA070476
:1007B00004983F1409F006FA000400140026039080
:1007C0000499B00040180B21890140188468002C5E
:1007D0007BD060782178000200250843800712D57D
:1007E000217B0120B94200DD00200221009123007D
:1007F0002200010004985A330C320196FFF7A6FF3D
:10080000002800D002256078217800026394562EDB
:1008100001000000FC020100000400000E903B7A81
:100820000843800614D52421095D0120B94200DA6D
:1008300000202021009123002200010004985B3356
:1008400024320196FFF78CFF002801D020200543B9
:100850006078217800020843C00714D0A179039A78
:1008600001204942914200DD002001210091230036
:10087000010004985833A21D0196FFF771FF00286C
:1008800001D0012005436078217800020843C006AA
:1008900015D5A17F039A01204942914200DA002038
:1008A00010210091230022000100049859331E32C8
:1008B0000196FFF755FF002801D010200543002DB9
:1008C0000DD0002E0BD104980B218901401881898D
:1008D0002943818101210498C90609F014FD761C81
:1008E0003606360E012E00D274E727E7F1B56120F7
:1008F000C04384B00027039002900498B900081800
:100900000B21890140188468002C7ED06078217802
:1009100006020F200E4380010640F6D00520C001DC
:10092000064208D00398623005D1049809F06EF9A8
:10093000000400140390FF20413006420DD003E074
:10094000A80C0004070100000298623005D1049849
:1009500009F03CF90004001402900025300614D57B
:100960003021095D039A0120914200DD00208021A1
:10097000009123002200010004985E333032019779
:10098000FFF7EEFE002800D08025B00517D53C21EA
:10099000095D039A0120914200DA002001214902F9
:1009A000009123002200010004985F333C3201973C
:1009B000FFF7D6FE002802D0012040020543700652
:1009C00016D52A21095D029A01204942914200DD93
:1009D00000204021009123002200010004985C3394
:1009E0002A320197FFF7BCFE002801D040200543C2
:1009F000F00518D53621095D029A0120494291423D
:100A000000DA0020FF26761C00E01CE02300220014
:100A1000010004985D33363201970096FFF7A0FE7F
:100A2000002800D03543002D0DD0002F0BD10498A5
:100A30000B21890140188189294381810121049872
:100A4000C90609F060FC7F1C3F063F0E012F00D253
:100A500053E773E6F3B5002405000B26B60181B019
:100A6000A000401980198068002848D04178027899
:100A700009021143490742D50299096900290CD19D
:100A80000100603100224A708A70C07C0B00012195
:100A9000002800D00100197031E0010060318A782F
:100AA0004B7812021A43521C1204120C130A4A7099
:100AB0008B700B78002B22D0877CBA421FD35B1E31
:100AC0001A06120E0A701AD14A708A70C27C002A65
:100AD00001D00A7008E0417802780902114304222B
:100AE00091430170090A4170002C08D1A81981892D
:100AF0000422114381815106280009F004FC641C82
:100B00002406240E012CABD3FEBDAF49C868401C9F
:100B1000C8607047AC480022C168002903D1417801
:100B2000491C417000E04270C2607047F8B5070090
:100B30000B2080013D18AC68002C34D060782178FF
:100B40000002084340052ED5380009F04BF801009B
:100B50004034E078A37802029B4E1A430020914271
:100B600022DC7188491C0904090C7180627923799F
:100B700012021A438A4216D871788A4202D9318900
:100B8000012910D104007080EFF758FE7470EFF760
:100B90005AFE3481A889012189020843A8814904A9
:100BA000380009F0B0FBF8BD70803081F8BD0B2231
:100BB0009201801810B58468002C1FD060782278CC
:100BC00000021043400519D5487D44F04CE94034FB
:100BD000E179A2790B0213437B49002298420ED897
:100BE0008888401C0004000C8880637A247A1B02E9
:100BF0002343834202D8012008818A8010BD0A81E4
:100C0000FBE7F0B51D001FB40020C04384B0009086
:100C1000019004980B2189014618B468CA2E97B236
:100C200001000000F8060100000400005D4AE8161B
:100C3000002C3ED06078217800020843400538D56A
:100C400044F06AE8069A0F002B00121A8B410290BA
:100C500005D2069A02983900801AA94107E0069A3F
:100C600000980199801A029AA941801879410700D9
:100C700020000D004A3043F0FCEF00212B003A1A0F
:100C80008B4118D3554FF888401C05042D0C2000CB
:100C90004E30FD8043F0ECEFA8420AD80020F880E7
:100CA000B089012189020843B0810498490409F000
:100CB00034FB09B0F0BD49490020C880F9E710B500
:100CC0000400EFF7C5FD0B21890161188C89002212
:100CD0008A81EFF7C2FD200010BD0B2102008901BF
:100CE000511889680020002906D04A780B78110233
:100CF0001943090700D5012070470B2189014018CD
:100D00008068002803D000216030417081707047F6
:100D100070B5002031490400087048808880C88080
:100D200008810D00C8601035487063206043401989
:100D3000FFF782FB641C012CF7D370BD002010B5B7
:100D40000DF041FA0B2189014018806800280ED06F
:100D500041780278090211430122D20291430170C5
:100D6000090A41701D48017849084900017010BD09
:100D70000B218901421810B59168002911D04B78D8
:100D80000C781902214309050BD514490978C907C4
:100D900007D091890123DB0219439181190409F0DD
:100DA000BCFA10BD0B218901411810B58A898A81CE
:100DB0000121C90609F0B1FA10BD0B2189014218C1
:100DC0009168002902D10549103191600A7E4030B6
:100DD00040314276897D817670470000980C00048E
:100DE00038B505000C000021684623F0ECFE6B4688
:100DF000187880070ED1012020F0CCF9012C01D108
:100E0000092400E0142420F0CBF9200044F038E855
:100E1000002403E0022020F0BDF9F1E721002800C2
:100E20000FF091FC0100200020F068FD641C2406F6
:100E3000240E082CF2D338BDFD4A106BFD494863DF
:100E4000506B8863704770B5040031200D000001BD
:100E5000211820009C3018F0C5FEFFF7EDFF44F08C
:100E600014E88034217E280018F0B8FE280018F01D
:100E7000F7FE70BD002010B518F058FF00210620C5
:100E80000EF053FB44F004E8012106200EF01AFB9B
:100E900044F002E817F0E2FD10BD10B544F000E8A0
:100EA00010BDF8B505000E00170043F0FEEF04007A
:100EB000E148C069C06900280CD03A003100280020
:100EC00029F01AFDA04212DA3A003100280029F078
:100ED00013FD0DE03A003100280029F0DBFCA042B0
:100EE00005DA3A003100280029F0D4FC00E02000A7
:100EF000D24A1168884200DB08005168884200DB52
:100F00000800F8BD10B5FCF7ACFD0006000E10BDE2
:100F100010B5FCF7A9FD10BD10B50400FCF7A7FD46
:100F2000CF22F321002806D0022811D003282078F0
:100F300013D0084002E020780840001D10402070C7
:100F4000FCF792FD012820780BD0800880000BE090
:100F50002078084010401030F1E708403021084365
:100F6000EDE780088000401C207010BD10B5FFF731
:100F7000C9FF00220100100029F045FB10BDAF4A57
:100F80001368834203D00029106000D0EEE7704759
:100F9000AA4A5368834203D00029506000D0E5E795
:100FA0007047A64840680006000E704710B5140050
:100FB00002688A4201D1FF2909D101600EF08FFC3D
:100FC0009E494968884202D02100FFF7E1FF10BD29
:100FD000F8B50500080000210091697B1600FF2488
:100FE000C90716D069461DF0D9F9012811D16B4601
:100FF00093481978401840300479687B800708D5F9
:101000000320000228180079A04201DA241A00E027
:1010100000246120C000320021002818FFF7C6FF1D
:10102000F8BD10B503789B079B0F0B70EA25E350C2
:1010300001000000F40A010000040000A9259DA29F
:10104000110018F08EFE10BD3EB50500080000210D
:101050001400009101AA02A9FFF7EDFF43F032EF5F
:10106000002C1FD07C48694620F088F8002819D150
:101070000098774C800605D4A068401CA060002032
:101080000CF0BCFC0098C00606D4A068012109043D
:101090004018A0600CF0F8FC43F014EF0020694603
:1010A00020F06CF86B461A79187A2900FCF7C0FC1E
:1010B000FFF766FF20F06DF843F008EF3EBD10B576
:1010C0000400FCF7D8FC0006000E01222100FFF707
:1010D000BBFF10BD10B517F0C5FC10BD10B5FCF777
:1010E000CAFC0006000E10BD70B50E040500360CDB
:1010F0005A480022310043F0AAED040006D15848B6
:101100000022310043F0A2ED04000AD00220207337
:101110001C20656120812018742143F09CEDB020D3
:101120002081200070BDF7B5FF212D310700FFF7AA
:10113000DBFF05002BD01C202E18288102982C00E4
:10114000B03406602021200043F084EDA078F32124
:10115000800880000840001D01070198090F000168
:10116000014331200001A1703918200006220C3003
:1011700043F074ED3900FF3106228B31A01D43F09E
:101180006EED03216C20346681550520B070280077
:10119000FEBDFFB583B01400018945690E181C21FE
:1011A000471801817421380043F070ED2D480699ED
:1011B00000680C9B02790192009104992200300092
:1011C00018F0E3FD218828480022814206D1618879
:1011D000814203D1A188814200D1012206992800D1
:1011E0002AF0CEF9B870287A03280ED10698052186
:1011F000042809D0052802D00D2806D104E0687A19
:10120000022801D0012800D1B970380007B0F0BD24
:1012100010B50400FBF78CFB012805D1200043F03A
:10122000EAEC0020C04310BD002010BDFFB581B026
:101230006425FF275D370A9E01983900FFF754FFA8
:1012400004001CE000A5008040A30080546300045B
:10125000F4680500DC220004204E0000480D000464
:10126000D80D0004986D0500FFFF00000120F4F781
:10127000A7F801983900FFF737FF04006D1E002C16
:1012800007D1002D01DD132EF0D00020C04305B0A2
:10129000F0BD2089039A05190B980A2300280092B3
:1012A00000D10C230198312109014118029A200034
:1012B000FFF76FFF02202870002068700498203527
:1012C0002870000A68702189892021810655200034
:1012D000FFF79EFFDBE77CB50C00150006990022A6
:1012E000019200912A002100FFF7A0FF7CBD7CB590
:1012F0000C00150006990122019200912A0021009C
:10130000FFF794FF7CBDF0B5140007000E000A0043
:1013100085B000252100684618F06DFD00281DD11C
:10132000292C1BD00FDC202C18D007DC1D2C15D04D
:101330001E2C10D130786B4618730FE0222C0DD084
:10134000262C0BD007E02A2C08D0302C06D0312CCC
:1013500004D0322C02D00025ED4303E0380069466A
:1013600022F0F3FB280092E7F0B5130087B006AA3D
:1013700000921A00002505AB43F0ACED06990598E4
:1013800088422AD01FF0A4F920F072F9FD4E30688F
:10139000B10C88433060059800281ED0002401AFAE
:1013A00001200599A04008420BD0A00078556D1C83
:1013B000042C06D1012043F092ED3068E10208438D
:1013C0003060641C0D2CEBDD002D06DDFF20785510
:1013D00001A843F088ED43F08AED17E70A000121E8
:1013E00010B5FFF7C1FF012010BD10B58A781407B2
:1013F000A30F022B07D101282AD1C878C10727D112
:10140000800725D422E0A40F15D1130943F05EEC28
:101410000E080808081E1E20201E1E081E1E0A2078
:10142000022010BD012811D0032811D120310878E5
:1014300004280DD10AE0012B0AD113091B3FD6D590
:1014400001000000F00E010000040000FAFF4ECE83
:10145000083B43F046EC08070707050505050507A7
:10146000012010BD032010BD010070B50A008C786A
:10147000123225070020AE0F931F022E0CD1CC781C
:10148000E50705D1A00701D4100070BD180070BD9C
:10149000A207FCD4881D70BDAD0FF5D0012EFAD186
:1014A00022090A2AF6D00E2AF0D00F2AEED070BDFB
:1014B00010B504000CF0C9FC617A022904D1603037
:1014C0000078022807D203E0032904D0012902D0C2
:1014D000207A012801D1012010BD002010BD002874
:1014E00010B509D00CF042FE002805D01D2149019D
:1014F0004018007C012800D0002010BDF0B5050088
:1015000085B00026012001900C00370028000096CD
:101510000CF02CFEA079C00774D1002D0ED0687B92
:10152000C0067CD4687A032801D1012000902800ED
:10153000FFF7BEFF00285ED002205DE0A078010723
:10154000890F2CD10009042829D102200CF04FFE6C
:101550000600312000010DE0312000013118062283
:10156000A01D42F072FE002859D0022130000DF07B
:10157000EFFB0600002EEFD103200CF038FE0CE04C
:101580003120000131180622A01D42F05EFE002825
:1015900045D0032130000DF0DBFB0600F0D1200028
:1015A000FFF762FF060015D030000EF0FEF90500CF
:1015B00003D103200CF01BFE0500287A002801D07F
:1015C000062807D1A0780007800F022802D1E07812
:1015D000800715D5002D13D0287A022804D12800C1
:1015E000FFF77DFF00280BD0287A032805D1687A01
:1015F000002805D001E001200190207BC00702D027
:1016000001273EE00BE0A0780107890F09D100090E
:101610000D2806D1E078C10703D1800701D400204E
:101620003FE6287A2100FFF7EAFE0199884228D98F
:1016300001270721032800D0062120000291697AA2
:101640000C300229039005D1029A0399280027F053
:101650006EF816E0300001F0FBF9002811D1009877
:10166000002808D0A0780007810F012901D0800F41
:1016700001D1012015E6029A03992800002343F0C6
:1016800044EC38000DE670B50400EFF7F5F80500FE
:10169000E17AA07A0CF02AFC0FE0607BC00607D547
:1016A00020001DF00EFB0200012120002AF004F8AA
:1016B000E27AA17A20000CF0D8FC0400EDD12800D9
:1016C000EFF7DFF870BD10B504000CF04FFD416C72
:1016D000002908D031490300020041186433483220
:1016E000200018F0BDFC10BD10B504002B482018D8
:1016F00018F008FD032000210002201801728172F9
:10170000016110BD70B504000CF030FD0500200033
:101710000CF09BFB007AB7218900691883079B0FA7
:101720000A0020321500127910000DD0002B0BD1C9
:10173000253118F09BFB200028F0A6FB287A000733
:10174000C10F207A1EF0A4FF70BD10B504000CF08C
:101750000DFDB7218900401800222D210A542530A3
:1017600018F09BFB2000FFF7CDFF10BDF8B505007A
:101770000CF0FCFC0321090241180C781723DF222E
:10178000EF265B01022C0BD10F79C01837400F7187
:10179000017E002411401EE000A300800103000030
:1017A0000B24A40104196479E40702D18C78002C7D
:1017B00000D001240F793740E607F60E3743002C9E
:1017C0000F7104D1C118097E2022114302E0C11813
:1017D000097E1140C0180176280028F055FB28002A
:1017E00028F0D4FB200016F0FFFFF8BD10B5040070
:1017F0000CF0BCFC03221202002180188170200032
:10180000FFF7B4FF10BDFEB507000CF0AFFC019070
:1018100038000CF01AFB0400387A3D000C34803597
:1018200003282ED17D20C00000906068002806D0DB
:10183000698B009843F070EA21680E1A00E0266870
:10184000698B009843F068EAB0420BD367D754F134
:1018500001000000EC12010000040000453A6B7D1D
:10186000200002F0FFFE002806D1FF209130C15B6E
:101870000022380001F0B6F95420005D012811D98A
:1018800000206060217E012080020129019905D19C
:101890000818806A04E053480090DAE70818406AA4
:1018A0002060FEBD0128FCD1687E4000401CF7E7A7
:1018B00070B504000CF064FC0321090243181A7887
:1018C0001721FB254901022A01D1002202E0002A4A
:1018D00005D101224018417E294041760FE0DA7897
:1018E000002A00D00122002A04D143185B7E04257F
:1018F0002B4302E043185B7E2B40401843760121C6
:10190000002A00D000212000FFF788FA200028F0EC
:1019100047FB70BD10B504000CF032FC032212022C
:1019200000218018C1702000FFF7C2FF10BD2E4AB1
:10193000831A90420ED005DC2C4A801A0AD0072860
:101940000ED107E02A48181808D07D22D200801A4C
:1019500006D101E000207047012070470220704747
:101960000E29F9D8F6E701280AD002280AD0002962
:1019700003D00E2901D11C4870471B48C01F704777
:10198000184870477D204001704710B504000800DA
:101990001100FFF7E8FF2070000A6070012BE27071
:1019A00001D10A2004E0022B01D1282000E01420FC
:1019B000A07010BD10B504000DF0E2FF012801DD9C
:1019C000012000E00020002C06D0012C07D0022CC2
:1019D00001D143F07CEA10BD1FF073FF10BD1FF072
:1019E0007EFF10BD881300006E0900006009000032
:1019F000CEF9FFFF3EB5002104000A000B00684647
:101A00000EC00622FF49684643F03CE9FD4A002526
:101A1000CB3A507B012100280CD0012807D00428A4
:101A200003D180206B46987106E0002C02D06B46F3
:101A3000997101E06B469D716B46117398799073B3
:101A4000F04869460B38C06B21F057FB3EBDF0B53E
:101A500091B0EC4C0B3CE06B0CF0A4FC0500402179
:101A600001A843F028E9E749062201A843F00AE962
:101A7000200020300100427C03A80F39801C43F075
:101A800002E920002030C17C6B469972007DD8723B
:101A9000DD480021008826009881A37AC03E01AA73
:101AA0000AE07018A030007F571820374006400E1B
:101AB000491C0906090EB8728B42F2D80420307313
:101AC000E06BEF22417B11402822525DD207D20EFB
:101AD00011434173CB480FA9173818F069FB10ABBD
:101AE0001880E06B417BC90604D4C6494B390969AB
:101AF000002905D02A00002301A921F085F902E080
:101B000001A921F050F9E06B1022417B1143417390
:101B100011B0F0BD7CB504000CF044FC05002000C1
:101B2000F1F796F9A17BC8073FD101200143B548E1
:101B3000A173AB38007900280BD0032000022018D5
:101B4000006A2030007BC00703D0012120001EF076
:101B500044FA0021200000F0D1FF402120000BF0CA
:101B6000A6FA20002EF03EFAA6484B3880690028DD
:101B700010D0A448CB38C16900290BD07D23DB00ED
:101B800059430022019200910322290020000023E2
:101B900021F090FC9D480088002806D007F0ADF8A1
:101BA000002802D0200007F00BFD7CBDF8B506220E
:101BB0000700944839000B38C56B2800FF308B3084
:101BC00043F060E82800062239009C3043F05AE8D0
:101BD000280078302021060043F06CE83C002034D7
:101BE000A279B91D300043F04EE8A1799820415503
:101BF00084490020CB390871032000022E18316A75
:101C0000E2792031087B520740084000D20F104390
